:0407000039EF9FF03E
:08070800046ED8CF05F0E0CF2C
:1007100006F00001E9CF0CF0EACF07F0E1CF08F0D6
:10072000E2CF09F0D9CF0AF0DACF0BF0F3CF12F015
:10073000F4CF13F0FACF14F0F5CF15F0F6CF16F092
:10074000F7CF17F0F8CF18F0FBCF19F000C00EF07C
:1007500001C00FF002C010F003C011F0A3AAB4EF63
:1007600003F0A4BAE2EF0FF09DAABAEF03F09EBA2D
:100770002BEF0FF09DA2C0EF03F09EB23CEF11F003
:100780000EC000F00FC001F010C002F011C003F065
:100790000CC0E9FF07C0EAFF078E08C0E1FF09C0EF
:1007A000E2FF0AC0D9FF0BC0DAFF12C0F3FF13C08B
:1007B000F4FF14C0FAFF15C0F5FF16C0F6FF17C00E
:1007C000F7FF18C0F8FF19C0FBFF045006C0E0FF98
:1007D00005C0D8FF1000F76AEA0FF66E070EF72281
:1007E000000EF86E0900F5501200280C0106F76A99
:1007F000020FF66E080EF722000EF86E0900F55093
:1008000012002020466F726D6174207361766564FA
:1008100020200000F76A280FF66E080EF722000E5F
:10082000F86E0900F550120020204F757470757431
:1008300020736176656420200000F76A4E0FF66E23
:10084000080EF722000EF86E0900F5501200202065
:10085000457869742053657475702020202000004D
:10086000F76A740FF66E080EF722000EF86E090094
:10087000F5501200204E69676874204D6F64652042
:10088000497269730000F76A9A0FF66E080EF72234
:10089000000EF86E0900F550120020204D616E75B3
:1008A000616C20497269732020200000F76AC00F34
:1008B000F66E080EF722000EF86E0900F5501200D1
:1008C000202020204175746F2049726973202020F8
:1008D0000000F76AE60FF66E080EF722000EF86EBB
:1008E0000900F55012002020204F6E6520507573CE
:1008F0006857422020200000F76A0C0FF66E090EA0
:10090000F722000EF86E0900F55012002020204159
:1009100057422F4142422053657420200000F76A5D
:10092000320FF66E090EF722000EF86E0900F55030
:100930001200202020414242204661696C20202084
:1009400020200000F76A580FF66E090EF722000EFD
:10095000F86E0900F5501200202020415742204631
:1009600061696C20202020200000F76A7E0FF66E5F
:10097000090EF722000EF86E0900F55012004D61C5
:100980006E75616C20576869746542616C20000067
:10099000F76AA40FF66E090EF722000EF86E090032
:1009A000F550120020205742205072657365742064
:1009B000412020200000F76ACA0FF66E090EF722C8
:1009C000000EF86E0900F550120020205742204119
:1009D00075746F202020202020200000F76AF00F7F
:1009E000F66E090EF722000EF86E0900F55012009F
:1009F00020204175746F2041637469766520202042
:100A00000000F76A160FF66E0A0EF722000EF86E57
:100A10000900F5501200204F50574220416374697D
:100A20007665202020200000F76A3C0FF66E0A0E43
:100A3000F722000EF86E0900F55012002053686985
:100A40006674204B4E454520202020200000F76A88
:100A5000620FF66E0A0EF722000EF86E0900F550CE
:100A600012002053686966742041637469766520BA
:100A700020200000F76A880FF66E0A0EF722000E9B
:100A8000F86E0900F550120020536869667420451D
:100A900078697420202020200000F76AAE0FF66EDF
:100AA0000A0EF722000EF86E0900F5501200204FD2
:100AB00050574220436F6D706C65746520200000B4
:100AC000F76AD40FF66E0A0EF722000EF86E0900D0
:100AD000F550120020204175746F205768697465C5
:100AE00042616C200000F76AFA0FF66E0A0EF722D8
:100AF000000EF86E0900F5501200205363656E6514
:100B000020412053746F726564200000F76A200F43
:100B1000F66E0B0EF722000EF86E0900F55012006B
:100B2000205363656E652041204C6F6164656420CD
:100B30000000F76A460FF66E0B0EF722000EF86EF5
:100B40000900F55012002020204E6F205363656E7F
:100B50006520412020200000F76A6C0FF66E0B0E16
:100B6000F722000EF86E0900F5501200205363655D
:100B70006E6520422053746F726564200000F76A2E
:100B8000920FF66E0B0EF722000EF86E0900F5506C
:100B90001200205363656E6520432053746F7265A5
:100BA00064200000F76AB80FF66E0B0EF722000EF5
:100BB000F86E0900F5501200205363656E652042FF
:100BC000204C6F61646564200000F76ADE0FF66EEA
:100BD0000B0EF722000EF86E0900F550120020539C
:100BE00063656E652043204C6F616465642000007E
:100BF000F76A040FF66E0C0EF722000EF86E09006D
:100C0000F55012002020204E6F205363656E652042
:100C1000422020200000F76A2A0FF66E0C0EF72201
:100C2000000EF86E0900F55012002020204E6F20B3
:100C30005363656E6520432020200000F76A500F43
:100C4000F66E0C0EF722000EF86E0900F550120039
:100C5000205363656E65204220436C656172656454
:100C60000000F76A760FF66E0C0EF722000EF86E93
:100C70000900F5501200205363656E652041204342
:100C80006C65617265640000F76A9C0FF66E0C0E6D
:100C9000F722000EF86E0900F5501200205363652C
:100CA0006E65204320436C65617265640000F76ADD
:100CB000C20FF66E0C0EF722000EF86E0900F5500A
:100CC00012002020466F726D61742F4F757470751D
:100CD00074200000F76AE80FF66E0C0EF722000E83
:100CE000F86E0900F55012002046696E64696E675F
:100CF0002043616D657261200000F76A0E0FF66E89
:100D00000D0EF722000EF86E0900F5501200204E6D
:100D10006F2063616D65726120466F756E640000BF
:100D2000F76A340FF66E0D0EF722000EF86E09000A
:100D3000F55012002046696E64696E67204845319F
:100D4000303020200000F76A5A0FF66E0D0EF722A1
:100D5000000EF86E0900F5501200202041572D4872
:100D6000453130302020202020200000F76A800FFD
:100D7000F66E0D0EF722000EF86E0900F550120007
:100D80002046696E64696E672043616E6F6E202035
:100D90000000F76AA60FF66E0D0EF722000EF86E31
:100DA0000900F5501200202056414444494F204884
:100DB000442D313820200000F76ACC0FF66E0D0E5E
:100DC000F722000EF86E0900F5501200202056415F
:100DD0004444494F2052455645414C200000F76A93
:100DE000F20FF66E0D0EF722000EF86E0900F550A8
:100DF00012004365696C696E67564945572048443F
:100E000031380000F76A180FF66E0E0EF722000E4A
:100E1000F86E0900F5501200202056414444494F15
:100E20002048442D323020200000F76A3E0FF66E35
:100E30000E0EF722000EF86E0900F5501200202069
:100E400056414444494F2048442D31392020000068
:100E5000F76A640FF66E0E0EF722000EF86E0900A8
:100E6000F550120020202020204556492D443330D3
:100E7000202020200000F76A8A0FF66E0E0EF7225F
:100E8000000EF86E0900F550120020202020455673
:100E9000492D44313030202020200000F76AB00F67
:100EA000F66E0E0EF722000EF86E0900F5501200D5
:100EB00020202020204556492D4437302020202056
:100EC0000000F76AD60FF66E0E0EF722000EF86ECF
:100ED0000900F5501200202020204252432D4837AF
:100EE0003030202020200000F76AFC0FF66E0E0E36
:100EF000F722000EF86E0900F55012002020202085
:100F00002020456C6D6F2020202020200000F76AF3
:100F1000220FF66E0F0EF722000EF86E0900F55044
:100F2000120020202020204252432D333030202038
:100F300020200000F76A480FF66E0F0EF722000E11
:100F4000F86E0900F5501200202020204252432D57
:100F50005A373030202020200000F76A6E0FF66EDE
:100F60000F0EF722000EF86E0900F5501200202037
:100F700020204252432D5A333330202020200000BD
:100F8000F76A940FF66E0F0EF722000EF86E090046
:100F9000F550120020202020204556492D4844318C
:100FA000202020200000F76ABA0FF66E0F0EF722FD
:100FB000000EF86E0900F55012002020202020437A
:100FC000562F48442020202020200000F76AE00F00
:100FD000F66E0F0EF722000EF86E0900F5501200A3
:100FE000202020202043562F534420202020202042
:100FF0000000F76A060FF66E100EF722000EF86E6C
:101000000900F55012002020556E6B6E6F776E2030
:1010100043616D6572610000F76A2C0FF66E100E69
:10102000F722000EF86E0900F55012002020496EDC
:1010300076616C69642043616D6572610000F76AD6
:10104000520FF66E100EF722000EF86E0900F550E2
:101050001200205363656E652041205361766564FC
:1010600020200000F76A780FF66E100EF722000EAF
:10107000F86E0900F5501200205363656E6520423A
:1010800020536176656420200000F76A9E0FF66E9B
:10109000100EF722000EF86E0900F55012002053D2
:1010A00063656E65204320536176656420200000EF
:1010B000F76AC40FF66E100EF722000EF86E0900E4
:1010C000F550120020202020202020202020202049
:1010D000202020200000F76AEA0FF66E100EF7229B
:1010E000000EF86E0900F550120020202020205537
:1010F0006E6B6E6F776E202020200000F76A100F55
:10110000F66E110EF722000EF86E0900F55012006F
:101110002020556E6B6E6F776E2056414444494FC8
:101120000000F76A360FF66E110EF722000EF86E09
:101130000900F55012002020496E69742045455081
:10114000726F6D2020200000F76A5C0FF66E110EA2
:10115000F722000EF86E0900F5501200204C6F6166
:10116000642044656661756C7473202000004F75BF
:10117000747075743E25730020497269732047614D
:10118000696E3E2573002049726973204761696E5C
:101190003E2573002049726973204761696E3E25C0
:1011A00073002049726973204147433E2573000054
:1011B0002049726973204761696E3E25756442005B
:1011C0002049726973204761696E3E257300497238
:1011D0006973204761696E3E257300002050656485
:1011E000657374616C203E20256400002047454EE5
:1011F0004C4F434B203E20256400204972697320E8
:101200004761696E3E202575000020204972697390
:1012100020506F733E25730020204972697320505F
:101220006F733E25730020204972697320506F73DD
:101230003E25730020204972697320506F733E254C
:10124000730020204972697320506F733E2573002C
:1012500020204972697320506F733E25730020204F
:101260004972697320506F733E25730020204972C4
:10127000697320506F733E25730020204972697393
:1012800020506F733E2573004972697320566F6C4E
:101290003E2025344C6400002020204972697320D0
:1012A0002575202020200000204145204C657665D2
:1012B0006C20257520200000202049726973205081
:1012C0006F733E2025750000202057422053686927
:1012D00066743E202564000020472D456E68616ECF
:1012E00063653E2030202020000020472D456E6899
:1012F000616E63653E202564000020427269676864
:10130000743E2025750047616D6D613E2025750096
:10131000204E6F697365205265647563204F4646A1
:101320000000204E6F697365205265647563204F1D
:101330004E20000047616D6D613E20257300204204
:101340006C7565204761696E3E202564000020535E
:101350006875742053706420312F342020200000E1
:1013600020536875742053706420312F313520204C
:10137000000020536875742053706420312F36307C
:101380002020000020536875742053706420312F92
:101390003130302000002053687574205370642071
:1013A000312F31303030000020436F6C6F72204796
:1013B00061696E3E2025640020422D456E68616E95
:1013C00063653E2025640000204368726F6D613EB6
:1013D0002025750020536875747465723E2025734E
:1013E0000000204368726F6D613E2025640020205C
:1013F000526564204761696E3E2025640000204EDE
:10140000442046696C746572204F464620200000D7
:10141000204E442046696C74657220312F3620209E
:101420000000204E442046696C74657220312F33D1
:1014300032200000202041706572747572653E2074
:101440002575000020436F6C6F72204875653E2043
:101450002564000020522D456E68616E63653E2054
:1014600030202020000020522D456E68616E63659B
:101470003E202564000020506564657374616C3EF5
:1014800020257500204B6E65653E2025750047615F
:101490006D6D6120312E3030200047616D6D61200F
:1014A000302E2532642000002053746162696C691B
:1014B0007A6572204F4646200000205374616269AD
:1014C0006C697A6572204F4E2020000020506564C0
:1014D000657374616C3E202564004D6173746572A0
:1014E000204761696E3E2573000020537461626974
:1014F0006C697A6572204F46462000002053746163
:1015000062696C697A6572204F4E2020000020428B
:101510006C7565204761696E3E2025640000204B94
:101520006E656520506F696E74204155544F000000
:10153000204B6E656520506F696E7420484947489E
:101540000000204B6E656520506F696E74204D4918
:1015500044200000204B6E656520506F696E74203A
:101560004C4F5720000020436F6C6F722048554548
:101570003E202564000020426C7565204761696E3D
:101580003E202564000020426C7565204761696E2D
:101590003E20254C640020426C7565204761696ED1
:1015A0003E20254C6400426C7565204761696E3EA3
:1015B00020254C64000020426C7565204761696EEF
:1015C0003E202564000020426C7565204761696EED
:1015D0003E20254C640020426C7565204761696E91
:1015E0003E20254C640020426C7565204761696E81
:1015F0003E202564000020426C7565204761696EBD
:101600003E202564000020426C7565204761696EAC
:101610003E202564000020526564204761696E3ECB
:101620002025640020426C61636B20535452455462
:1016300043482020000020426C61636B204D4944E8
:10164000444C45202020000020426C61636B2050F8
:101650005245535320202020000020436F6C6F72AE
:10166000204D58204E4F524D414C000020436F6C8E
:101670006F72204D582043494E45312000002043D1
:101680006F6C6F72204D582043494E453220000048
:101690002020526564204761696E3E202564000069
:1016A0002020526564204761696E3E20254C64000D
:1016B0002020526564204761696E3E20254C6400FD
:1016C00020526564204761696E3E20254C6400000D
:1016D0002020526564204761696E3E202564000029
:1016E0002020526564204761696E3E20254C6400CD
:1016F0002020526564204761696E3E20254C6400BD
:101700002020526564204761696E3E2025640000F8
:101710002020526564204761696E3E2025640000E8
:101720002020526564204761696E3E2025640000D8
:1017300020202044657461696C203E2025750000DE
:101740002044657461696C3E202564002047616D0A
:101750006D61204E4F524D414C202020000020470B
:10176000616D6D612043494E4531202020200000ED
:101770002047616D6D612043494E45322020202075
:10178000000020486F722044657461696C204849EC
:101790004748000020486F722044657461696C20DE
:1017A0004D494420000020486F72204465746169EF
:1017B0006C204C4F572000000A0D55345F4953529E
:1017C00020253278202532780A0D000052646163AA
:1017D0005F30203E20256C752000526461635F30CD
:1017E000203E20256C752000526461635F31203EED
:1017F00020256C752000526461635F31203E2025F6
:101800006C752000526461635F32203E2025752094
:101810000000526461635F32203E20257520000085
:1018200055345F4953522D45727220254C5820255E
:101830004C580A0D00005363656E652041205072BC
:1018400065736574204C6F616465640A0D004844DB
:101850002D3138205363656E6520412050726573C9
:101860006574204C6F616465640A0D0042616420F8
:101870006F72204E6F205072657365740A0D000000
:101880000D0A41572D48453130300D0A00004261A4
:1018900064206F72204E6F205072657365740A0D5C
:1018A0000000426164206F72204E6F205072657399
:1018B00065740A0D00000A0D2043616D6572615464
:1018C00079706520000054696D656F75740A0D208C
:1018D00000000D0A56414444494F2048442D3138F8
:1018E0000D0A00000D0A56414444494F2052455606
:1018F00045414C2048442D31380D0A000D0A56410F
:101900004444494F204365696C696E6756494557A1
:101910002048442D31380D0A00000D0A5641444438
:10192000494F2048442D32300D0A00000D0A56411F
:101930004444494F2048442D31390D0A00000D0A16
:10194000536F6E79204556492D4433300D0A0000FF
:101950000D0A536F6E79204556492D443130300DB4
:101960000A000D0A56414444494F2048442D31385D
:101970000D0A00000D0A536F6E79204556492D441B
:1019800037300D0A00000D0A536F6E792042524322
:101990002D483730300D0A000D0A456C6D6F20431D
:1019A000616D6572610D0A000D0A536F6E792042F8
:1019B00052432D3330300D0A00000D0A536F6E79FB
:1019C000204252432D5A3730300D0A000D0A536F12
:1019D0006E79204252432D5A3333300D0A000D0ADE
:1019E000536F6E79204556492D4844310D0A000049
:1019F0000D0A56616464696F204365696C696E679E
:101A0000564945572048440D0A000D0A5661646442
:101A1000696F204365696C696E6756494557205365
:101A2000440D0A00556E6B6E6F776E2043616D65D5
:101A300072610D0A0000556E6B6E6F776E20436108
:101A40006D6572610D0A0000496E76616C696420F3
:101A500043616D6572610D0A00000D0A20576169CE
:101A600074536F6E7941636B00000D0A20576169F2
:101A700074536F6E79002A57616974536F6E7900E1
:101A8000202D2054696D656F757420256C75202894
:101A90006D73290D0A00202D2054696D656F7574D2
:101AA00020256C7520286D73290D0A00202D2054E7
:101AB000696D656F757420256C7520286D73290D0F
:101AC0000A00205761697450616E61736F6E6963BB
:101AD000496E71526573702000000D0A20576169CC
:101AE0007450616E61736F6E69630000202D205425
:101AF000696D656F757420256C7520286D73290DCF
:101B00000A00202D2054696D656F757420256C7551
:101B100020286D73290D0A00202D2054696D656FF2
:101B2000757420256C7520286D73290D0A000D0A27
:101B300020676574382054696D656F757420256C55
:101B40007520286D73290D0A00000A0D20202067DA
:101B5000657438200000204572726F720A0D000013
:101B60000D0A2067657431362054696D656F757490
:101B700020256C7520286D73290D0A000A0D202080
:101B80002067657431362000204572726F720A0D2D
:101B900000000A0D476574556E736F6C6963697454
:101BA0006564205B2025780048442D31382053633C
:101BB000656E6520412050726573657420436C65C5
:101BC000617265640A0D000048442D31382053636A
:101BD000656E6520422050726573657420436C65A4
:101BE000617265640A0D000048442D31382053634A
:101BF000656E6520432050726573657420436C6583
:101C0000617265640A0D000048442D313820536329
:101C1000656E65204120507265736574205361764E
:101C20006564000048442D3138205363656E65209B
:101C300042205072657365742053617665640000BC
:101C400048442D3138205363656E6520432050721F
:101C500065736574205361766564000048442D31D6
:101C600038205363656E652041205072657365743A
:101C7000204C6F616465640A0D0048442D313820A2
:101C80005363656E65204220507265736574204C05
:101C90006F616465640A0D0048442D313820536338
:101CA000656E65204320507265736574204C6F61CA
:101CB0006465640A0D00526564204761696E2052B4
:101CC000657472792044656C6179203130306D73B0
:101CD000205361766528254C782920576F726B2830
:101CE000254C78290A0D0000426C75652047616912
:101CF0006E2052657472792044656C6179203130B0
:101D0000306D73205361766528254C782920576FF4
:101D1000726B28254C78290A0D000A0D2043616D4D
:101D200065726154797065200000496E76616C6956
:101D3000642043616D6572610D0A0000496E766131
:101D40006C69642043616D6572610D0A00000A0DC3
:101D500020506F776572204F6E2052657472792023
:101D60000000496E76616C69642043616D65726143
:101D70000D0A0000496E76616C69642043616D65EF
:101D800072610D0A00000D0A43616E6F6E20000043
:101D9000556E6B6E6F776E2043616D6572610D0AD3
:101DA0000000496E76616C69642043616D65726103
:101DB0000D0A0000202D2054696D656F7574202573
:101DC0007520286D73290D0A0000205D0A0D0000A2
:101DD000202D2054696D656F757420257520286D40
:101DE00073290D0A0000202D2054696D656F7574EC
:101DF00020257520286D73290D0A00000D0A205733
:101E000061697443616E6F6E00000D0A205761694D
:101E10007443616E6F6E4E6F744275737900202D3E
:101E20002054696D656F757420256C7520286D735D
:101E3000290D0A000D0A20436865636B43616E6FCC
:101E40006E4175746F574253746174757300A4A822
:101E5000FED76D6E12000D01C06B000E9EBA010E12
:101E6000000AD8B4A7D0ABA408D0AECFC0FD000EF6
:101E70009EBA010E000A01E19DD0ABA20BD0AB9837
:101E8000AB9E0000AB88AB8E000E9EBA010E000A1E
:101E900001E190D09EAAFED7AECFC0FD07016051F0
:101EA0000E082DE081A207D030840D01C051000141
:101EB000CEDF23D00701780E09016C25E96E070EED
:101EC0006D21EA6EC0CDEFFF010E6C250D01C16FD3
:101ED000000E09016D210D01C26F010809E303E144
:101EE000C151F30805E309016C2BD8B46D2B03D065
:101EF00009016D6B6C6B308A00015AD0070150B339
:101F00002FD00D01C051F00825E107015083780E54
:101F100009016C25E96E070E6D21EA6EC0CDEFFF59
:101F2000010E6C250D01C16F000E09016D210D011F
:101F3000C26F010809E303E1C151F30805E3090198
:101F40006C2BD8B46D2B03D009016D6B6C6B308A90
:101F500005D00D01C05100017ADF090129D0070128
:101F6000780E09016C25E96E070E6D21EA6EC0CD71
:101F7000EFFF010E6C250D01C16F000E09016D21EF
:101F80000D01C26F010809E303E1C151F30805E344
:101F900009016C2BD8B46D2B03D009016D6B6C6BF0
:101FA000308A0D01C03D03D0070150930D01090196
:101FB0000D0153D79E9A0001C0EF03F09EA8FED7F3
:101FC000AD6E12000D01C06B000EA4BA010E000A26
:101FD00051E06BA408D06ECFC0FD000EA4BA010E74
:101FE000000A01E147D06BA20BD06B986B9E0000FA
:101FF0006B886B8E000EA4BA010E000A01E13AD084
:10200000A4AAFED76ECFC0FD070160510E082CE0D8
:1020100081A206D00D01C0510001D0DF23D00701FD
:10202000710E0B016525E96E090E6621EA6EC0CDC1
:10203000EFFF010E65250D01C16F000E0B0166213A
:102040000D01C26F010809E303E1C151F30805E383
:102050000B01652BD8B4662B03D00B01666B656B47
:10206000308C000105D007010D01C0510001A6DF31
:102070000D01AAD7A49A0001C0EF03F00D01C56BB2
:10208000C66BC76BD890C235016EC3CD00F001524C
:1020900004E0D8900032012EFCD70050030BC56F2E
:1020A000D890C235016EC4CD00F0015204E0D89042
:1020B0000032012EFCD70050030BC66FC551FC0F38
:1020C0002DE2040F00019BEF10F00D01C65302E159
:1020D000C70704D0C651030801E1C72B1FD00D016B
:1020E000C651020802E1C70703D0C62D01D0C72B95
:1020F00015D00D01C651030802E1C70703D0C6532E
:1021000001E1C72B0BD00D01C62D02D0C70704D0AB
:10211000C651020801E1C72B01D00D01036AC2516B
:102120003F0FE96E000E0320EA6EC751EF24EF6EF9
:10213000000151EF11F0E824F76AF736570FF66EF9
:10214000210EF722000EF86EFB6E0A00F550FA6EB3
:102150000800F550F96E0621F220CA20DE200D019C
:10216000C56BC66BC76B040EC25D006ED89000369F
:1021700000C001F0C3CD00F0015204E0D89000325D
:10218000012EFCD70050030BC56F040EC25D006E1C
:10219000D890003600C001F0C4CD00F0015204E038
:1021A000D8900032012EFCD70050030BC66FC551EA
:1021B000FC0F2DE2040F000128EF11F00D01C653B2
:1021C00002E1C70704D0C651030801E1C72B1FD0A5
:1021D0000D01C651020802E1C70703D0C62D01D088
:1021E000C72B15D00D01C651030802E1C70703D064
:1021F000C65301E1C72B0BD00D01C62D02D0C70776
:1022000004D0C651020801E1C72B01D00D01036AB9
:10221000C251370FE96E000E0320EA6EEF50C75D22
:102220000BE1036AC2513F0FE96E000E0320EA6E14
:10223000C751EF24EF6E09D0036AC251370FE96E20
:10224000000E0320EA6EC7CDEFFF000170EF11F022
:10225000E824F76AF736710FF66E220EF722000EA9
:10226000F86EFB6E0A00F550FA6E0800F550F96E34
:10227000F821E421BC21D0210D01C06BC16B96680F
:1022800084CFC0FD3550C05D15E0C16BC15103085E
:102290000BE3C1CDC2FDC0CDC3FD35C0C4FD0001FF
:1022A000EDD60D01C12BF2D7C0CD35F0326A316ABF
:1022B000308603D0312AD8B4322A976885CFC0FD42
:1022C0003650C05D16E0040EC16FC15107080BE324
:1022D000C1CDC2FDC0CDC3FD36C0C4FD00013FD796
:1022E0000D01C12BF2D7C0CD36F0346A336A308885
:1022F00003D0332AD8B4342A9E929E920001C0EFB4
:1023000003F04343552020257300080E016E040E90
:10231000006E002EFED78B969496040E006E002E53
:10232000FED70B01CA378B98D8B09488D8A0949860
:10233000948682A6FED7012E01D002D00001E7D7F5
:10234000040E006E002EFED78B96949600009488A3
:10235000040E006E002EFED7040E006E002EFED777
:10236000948682A6FED7016A040E006E002EFED768
:1023700082B801808B9694968B98949800011200F5
:102380009488040E006E002EFED79486040E006E14
:10239000002EFED78B989498040E006E002EFED768
:1023A0008B9694960D0E006E002EFED70B01C65133
:1023B000FE0BC96FCA6F0001A8DF0D0E006E002E64
:1023C000FED7C7CBCAFBA1DF0D0E006E002EFED7D5
:1023D000C8CBCAFB9ADF0D0E006E002EFED7949874
:1023E0000000948682A6FED7040E006E002EFED753
:1023F00000D000009488040E006E002EFED70F0E51
:10240000006E002EFED700D01200080E0B01BE6F2A
:1024100000C0BFFB9488040E006E002EFED7948689
:1024200082A6FED782B8D88082A8D8900136040E42
:10243000006E002EFED794968B96BE2FEBD7948815
:10244000040E006E002EFED78B98BF51D8A494982E
:102450000000948682A6FED7040E006E002EFED7E2
:102460008B969496040E006E002EFED78B9894984F
:10247000000112000B019D6B9488040E006E002E6B
:10248000FED79486040E006E002EFED78B9894988B
:10249000040E006E002EFED78B9694960D0E006EE5
:1024A000002EFED79B51FE0B9E6FCA6F00012DDFE1
:1024B0000D0E006E002EFED79CCBCAFB26DF0D0E44
:1024C000006E002EFED79488040E006E002EFED7FC
:1024D0009486040E006E002EFED782A6FED78B983F
:1024E0009498040E006E002EFED78B9694960D0ED7
:1024F000006E002EFED70B019B5101099E6FCA6F23
:10250000000103DF0D0E006E002EFED7006A7DDF96
:1025100001C09DFB0D0E006E002EFED794980000AA
:10252000948682A6FED7040E006E002EFED700D041
:1025300000009488040E006E002EFED70F0E006E71
:10254000002EFED700D00B019DCB01F00001120040
:102550000B01816B400EC66F180EC76F7F0EC86FE0
:1025600000010EDF400E0B01C66F190EC76FC86960
:10257000000106DF400E0B01C66F1A0EC76FC86B55
:102580000001FEDE400E0B01C66F1B0EC76FC86B4D
:102590000001F6DE400E0B01C66F1C0EC76FC86B44
:1025A0000001EEDE400E0B01C66F200EC76F800EDD
:1025B000C86F0001E5DE400E0B01C66F210EC76F2C
:1025C000C86B0001DDDE400E0B01C66F220EC76F27
:1025D000C8690001D5DE400E0B01C66F230EC76F20
:1025E000C8690001CDDE400E0B01C66F240EC76F17
:1025F000C8690001C5DE400E0B01C66F0C0EC76F27
:10260000C8690001BDDE4F68400E0B019B6F9C6BDB
:10261000000130DF01C081FB400E0B019B6F010EFA
:102620009C6F000127DF01C081FB2CEFABF00D0E8A
:10263000EA6EB60EE96EEF500EE0050E016E006A0E
:10264000002EFED7012EFBD72E0E006E002EFED7D9
:1026500000D0EF2EF2D712000C01A039F00B006E63
:102660000F0E8C1400108C6E00008C80020E006E19
:10267000002EFED700008C90000112008350006EE7
:1026800000380F0B016E12000F0E9514F009956EB5
:102690008C8400008C800000F1DF01C0A0FC8C90D5
:1026A00000008C8000D000D0E9DF01C09FFC8C903E
:1026B0000F0E9514956E0C01A039006EF00E0016E9
:1026C00000509F11016E000168EF13F08C92DCD76F
:1026D00001C09FFC0C0101AE02D00001F8D78C9222
:1026E0009DB18C8200008C9400008C909E399F6F6D
:1026F0000F0E9F179FCCA0FC0001AEDF0C019E5176
:102700000F0B9F6FA06F0001A7DF12000F0E951433
:10271000956E9590959295948C928C948C900F0ECA
:102720000D01B66F000183DF010E0B01816F815136
:1027300003080DE3030E0C01A06F00018DDF050EF1
:102740000D01B66F000173DF0B01812BF0D7020E74
:102750000C01A06F000180DF0B01816B8151030828
:102760000FE3036A81510001EBEC03F00B01826F70
:102770000C019D6B9E6F0001A9DF0B01812BEED731
:10278000000134EFABF06BCBEAFF6ACBE9FF0B0142
:10279000A6CBEFFFE92AD8B4EA2AEF6A6A2BD8B4AD
:1027A0006B2B000112000900F6CF9EFBF7CF9FFBB9
:1027B000F8CFA0FBF5CFA6FBE6DF9ECBF6FF9FCBC5
:1027C000F7FFA0CBF8FF0B019D2F01D002D0000135
:1027D000EAD700011200EF520FE0EACF9EFBE9CFEB
:1027E0009DFBEFCFA6FBCFDF9ECBEAFF9DCBE9FFA2
:1027F000E92AD8B4EA2AEFD712000C019A2D01D0A9
:1028000003D0400E9B6F01D09B6B010E995D9B27FF
:102810009B5180099C6F9D6B9E6F000157DF1200DA
:102820000C0198510C0A000105E0060A0FE0020AAB
:1028300015E01BD00C019D6B010E9E6F000146DF61
:10284000020E0D01B66F0001F2DE17D0010E0C0171
:10285000996F020E9A6F0001D0DF0FD00C019D6BB3
:10286000100E9E6F000132DF08D0010E0C019D6F2B
:1028700098CC9EFC00012ADF00D0120098CC9AFC74
:1028800097CC99FC9ACC03F00C0199CCE9FF9ACC37
:10289000EAFFEF5206E0992BD8B49A2B0001F2D749
:1028A0000C019751995D006E98519A59036E00C0C2
:1028B00001F0000112000C01966B95CC98FC94CCB1
:1028C00097FC0001DBDF0152D8B48ED095CC98FC88
:1028D00094CC97FCD3DF01500C01965DD8B085D025
:1028E000036A96519425E96E95510320EA6EEF50E4
:1028F000010A00010DE0030A26E0010A3FE0080A90
:1029000058E0070A5EE0060A5CE0020A5AE059D085
:102910000C01965317E1010E996F9A6F00016DDF5C
:10292000200E0C01986F00017BDF010E0C01996FE6
:10293000020E9A6F000161DF200E0C01986F0001FA
:102940006FDF0C014ED00C01965317E1010E996F09
:102950009A6F000152DF3E0E0C01986F000160DF9C
:10296000010E0C01996F020E9A6F000146DF200ED6
:102970000C01986F000154DF0C0133D00C01965309
:1029800017E1010E996F9A6F000137DF200E0C01DD
:10299000986F000145DF010E0C01996F020E9A6FCE
:1029A00000012BDF3E0E0C01986F000139DF0C0196
:1029B00018D0010E0C01996F9A6F00011EDF0C01F7
:1029C00010D0036A0C0196519425E96E95510320AD
:1029D000EA6EEFCF97FC97CC98FC000121DF0C0149
:1029E00000D0962B000172D70C0100011200200EBE
:1029F0000B01D96FDA6FDB6FDC6FDD6F560EDE6FA8
:102A0000410EDF6F440EE06FE16F490EE26F4F0E33
:102A1000E36F200EE46FE56FE66FE76FE86FE96B39
:102A2000560EEA6F410EEB6F440EEC6FED6F490EE0
:102A3000EE6F4F0EEF6F200EF06F480EF16F440EE9
:102A4000F26F2D0EF36F310EF46F380EF56F200E0E
:102A5000F66F430EF76FF86F550EF96FFA6B560E5F
:102A6000FB6F410EFC6F440EFD6FFE6F490EFF6F52
:102A70004F0E0C01006F200E016F520E026F450EBB
:102A8000036F560E046F450E056F410E066F4C0E18
:102A9000076F200E086F096F0A6F0B6B430E0C6FE8
:102AA000650E0D6F690E0E6F6C0E0F6F690E106F55
:102AB0006E0E116F670E126F560E136F490E146F64
:102AC000450E156F570E166F200E176F480E186FB4
:102AD000440E196F310E1A6F380E1B6F1C6B560E99
:102AE0001D6F410E1E6F440E1F6F206F490E216F28
:102AF0004F0E226F200E236F480E246F440E256F59
:102B00002D0E266F320E276F300E286F200E296F84
:102B1000430E2A6F2B6F550E2C6F2D6B560E2E6F9A
:102B2000410E2F6F440E306F316F490E326F4F0ED2
:102B3000336F200E346F480E356F440E366F2D0EF6
:102B4000376F310E386F390E396F200E3A6F430EE2
:102B50003B6F3C6F550E3D6F3E6B3F6F6E0E406F8F
:102B60006B0E416F6E0E426F6F0E436F770E446FA8
:102B70006E0E456F200E466F560E476F410E486F22
:102B8000440E496F4A6F490E4B6F4F0E4C6F200E2B
:102B90004D6F4E6F4F6B506F516F430E526F536FAF
:102BA000550E546F200E556F430E566F6F0E576FB4
:102BB0006E0E586F740E596F720E5A6F6F0E5B6FF8
:102BC0006C0E5C6F200E5D6F5E6F5F6F606B616F90
:102BD000626F500E636F540E646F5A0E656F200E55
:102BE000666F430E676F6F0E686F6E0E696F740EBF
:102BF0006A6F720E6B6F6F0E6C6F6C0E6D6F200EC6
:102C00006E6F6F6F706F716B726F736F520E746F48
:102C1000640E756F610E766F630E776F200E786F9E
:102C2000430E796F6F0E7A6F6E0E7B6F740E7C6F32
:102C3000720E7D6F6F0E7E6F6C0E7F6F200E806F39
:102C4000816F826B836F846F430E856F610E866F19
:102C50006D0E876F650E886F720E896F610E8A6FB9
:102C6000200E8B6F530E8C6F650E8D6F740E8E6FF2
:102C7000750E8F6F700E906F200E916F926F936B29
:102C8000938681B602D02A0E806F0C0E986F0001D9
:102C9000C7DD30A208D00B0E0C01956FD90E946FD2
:102CA000000109DE87D0070151AF09D00C0E0C01DD
:102CB000956F720E946F0001FEDD7CD00701482DE8
:102CC00009D00C0E0C01956F830E946F0001F3DD9B
:102CD00071D0070160510E085BE15251006E5351F3
:102CE000036E010E035C04E10052000120E00701C5
:102CF000010E035C05E1010E005C000120E007010C
:102D0000010E035C05E1020E005C000120E00701FA
:102D1000020E035C04E10052000120E00701030EF3
:102D2000035C04E10052000121E0070127D00B0EF3
:102D30000C01956FEA0E946F0001BDDD27D00B0EDC
:102D40000C01956FFB0E946F0001B5DD1FD00C0ECA
:102D50000C01956F946F0001AEDD18D00C0E0C01C4
:102D6000956F1D0E946F0001A6DD10D00C0E0C01A6
:102D7000956F2E0E946F00019EDD08D00C0E0C0195
:102D8000956F3F0E946F000196DD00D013D00701C0
:102D900081B209D00C0E0C01956F500E946F00019A
:102DA0008ADD08D007010C0E0C01956F610E946F3F
:102DB000000181DD0A0E0C01986F000131DD100E5B
:102DC0000B01D725E96E000ED821EA6EEF6AD8CB49
:102DD00095FCD7CB94FC00016EDD12000B018D53E6
:102DE00002E18E5342E089CBE9FF8ACBEAFFEFCFC5
:102DF0008FFB8CCB03F08BCBE9FF8CCBEAFFEF5042
:102E00008F5D17E08ACB03F089CBE9FF8ACBEAFF1D
:102E1000EFCF8FFB8CCB03F08BCBE9FF8CCBEAFFA2
:102E2000EF508F5D02E2FF0E01D0010E016E1FD048
:102E30000BD08ACB03F089CBE9FF8ACBEAFFEF52B4
:102E400003E1000E016E13D08ACB03F08951892B68
:102E5000D8B48A2B8CCB03F08B518B2BD8B48C2B12
:102E60008D51D8B48E078D07BAD7000E016E0001C0
:102E700073EF17F00B01816B836B826B200E846FF5
:102E8000856F866F876B886B030E836FF60E826F7C
:102E9000816B815103081BE3036A8151840FE96E42
:102EA0000B0E0320EA6EF2CF8BFBF29E83CBAAFFC0
:102EB00082CBA9FFA69CA69EA680A8508BBFF28EAF
:102EC000EF6E010E8227000E8323812BE2D70B0EBB
:102ED0008A6F840E896F8C6B220E8B6F8E6B030E44
:102EE0008D6F00017BD7015204E1010E016E04D009
:102EF00003D0000E016E00D066EFABF00B01876BC4
:102F0000866B876B866B875103081BE387CBAAFF11
:102F100086CBA9FFA868A69CA69EA684F250006E48
:102F2000F29E0F01550EA76EAA0EA76EA682A6B23C
:102F3000FED7A6940050F2120B01862BD8B4872B33
:102F4000E2D70001E9EF17F00B01876B866B886B06
:102F5000896B8A6B876B200E866F886B88532EE196
:102F6000896B8951020828E38A6B8A511F0822E382
:102F70008751036E8651862BD8B4872B8B6F03C085
:102F80008CFB8CCBAAFF8BCBA9FFA86AA69CA69E24
:102F9000A684F250006EF29E0F01550EA76EAA0E87
:102FA000A76EA682A6B2FED7A6940050F2120B011D
:102FB0008A2BDBD7892BD5D7882BD0D7000114EFEC
:102FC00018F00B01826B816B846B836B856B000146
:102FD00095D7AA6A0B0EA96EA86AA69CA69EA6847F
:102FE000F250006EF29E0F01550EA76EAA0EA76E4C
:102FF000A682A6B2FED7A6940050F212AA6A0C0EC0
:10300000A96EA86AA69CA69EA684F2CF00F0F29EA6
:10301000550EA76EAA0EA76EA682A6B2FED7A694DC
:103020000050F212000190D7030E0B01826FF60ED2
:10303000816F856B8551030827E3036A8551220F51
:10304000E96E000E0320EA6EEFCF86FB82CBAAFF6B
:1030500081CBA9FF86CBA8FFA69CA69EA684F25092
:10306000006EF29E0F01550EA76EAA0EA76EA682E5
:10307000A6B2FED7A6940050F212010E0B018127D2
:10308000000E8223852BD6D7846B836B856B85518D
:10309000090843E3036A8551260FE96E000E0320F9
:1030A000EA6EEFCF86FB86512F0803E2865139087E
:1030B00002E2000E01D0010E01082DE184532BE144
:1030C0008351050828E3036A8551260FE96E000E37
:1030D0000320EA6EEFCF86FB82CBAAFF81CBA9FF4C
:1030E00086CBA8FFA69CA69EA684F250006EF29EF8
:1030F0000F01550EA76EAA0EA76EA682A6B2FED726
:10310000A6940050F2120B01832BD8B4842B010E2D
:103110008127000E8223852BBAD7000183EFABF005
:1031200007014F6B506B516B556B546B576B566B64
:10313000586B606B616B646B656B676B666B696B1F
:10314000686B6A6B6B6B6C6B6D6B6E6B6F6B706BC4
:10315000716B726B736B746B756B766B000106EF42
:103160001AF00B018151000A000104E0080AD8B4EA
:10317000A1D042D183CB03F00B018251E96E03C091
:10318000EAFFF2CF8AFBF29EAA6AA96AA69CA69ED3
:10319000A680A8508ABFF28EEC6AED52EF6E83CB08
:1031A00003F08251886F03C089FB83CB03F0825107
:1031B000E96E03C0EAFFECCF8BFBED52EFCF8AFB49
:1031C0008ACB8BFB8A6BF2CF8CFBF29EAA6A010E34
:1031D000A96EA69CA69EA680A8508CBFF28E8A11CE
:1031E000006E8B51036E00508A6F03C08BFB89CB3E
:1031F000EAFF88CBE9FF8BCBECFFED528ACBEFFFE8
:1032000085CB03F08451E96E03C0EAFFF2CF8AFB5D
:10321000F29EAA6A020EA96EA69CA69EA680A8503F
:103220008ABFF28EEC6AED52EF6E85CB03F08451CB
:10323000886F03C089FB85CB03F08451E96E03C01E
:10324000EAFFECCF8BFBED52EFCF8AFB8ACB8BFBF7
:103250008A6BF2CF8CFBF29EAA6A030EA96EA69C23
:10326000A69EA680A8508CBFF28E8A11006E8B514C
:10327000036E00508A6F03C08BFB89CBEAFF88CBBB
:10328000E9FF8BCBECFFED528ACBEFFF87CB03F04E
:103290008651E96E03C0EAFFF2CF8AFBF29EAA6A6A
:1032A000040EA96EA69CA69EA680A8508ABFF28E88
:1032B000EF6EA6D083CB03F00B018251E96E03C001
:1032C000EAFFF2CF8AFBF29EAA6A060EA96EA69CBE
:1032D000A69EA680A8508ABFF28EEC6AED52EF6ED1
:1032E00083CB03F08251886F03C089FB83CB03F04B
:1032F0008251E96E03C0EAFFECCF8BFBED52EFCFBA
:103300008AFB8ACB8BFB8A6BF2CF8CFBF29EAA6A7C
:10331000070EA96EA69CA69EA680A8508CBFF28E12
:103320008A11006E8B51036E00508A6F03C08BFBB5
:1033300089CBEAFF88CBE9FF8BCBECFFED528ACB40
:10334000EFFF85CB03F08451E96E03C0EAFFF2CFB3
:103350008AFBF29EAA6A080EA96EA69CA69EA6806B
:10336000A8508ABFF28EEC6AED52EF6E85CB03F067
:103370008451886F03C089FB85CB03F08451E96ECB
:1033800003C0EAFFECCF8BFBED52EFCF8AFB8ACB79
:103390008BFB8A6BF2CF8CFBF29EAA6A090EA96E98
:1033A000A69CA69EA680A8508CBFF28E8A11006EA5
:1033B0008B51036E00508A6F03C08BFB89CBEAFFF1
:1033C00088CBE9FF8BCBECFFED528ACBEFFF87CBAD
:1033D00003F08651E96E03C0EAFFF2CF8AFBF29E4A
:1033E000AA6A0A0EA96EA69CA69EA680A8508ABFAD
:1033F000F28EEF6E05D00001000E016E03D00B01BE
:10340000010E016E000133EF1AF08AD6F2CF81FB74
:10341000F29EAA6A0B0EA96EA69CA69EA680A85034
:103420000B0181BFF28E0701506FF2CF81FBF29E3C
:10343000AA6A0C0EA96EA69CA69EA680A8500B0197
:1034400081BFF28E07014F6F0B01816B55C783FB64
:1034500054C782FB57C785FB56C784FB876B58C789
:1034600086FB00017ED6010E016E9CEFABF0580E7C
:103470000B01A46F9488040E006E002EFED7948674
:10348000040E006E002EFED78B989498040E006EEA
:10349000002EFED78B9694960D0E006E002EFED752
:1034A000A451FE0BA56FCA6F000185EC11F00D0E43
:1034B000006E002EFED7A2CBCAFB85EC11F00D0EDC
:1034C000006E002EFED7A3CBCAFB85EC11F00D0ECB
:1034D000006E002EFED794980000948682A6FED738
:1034E000040E006E002EFED700D000009488040E5B
:1034F000006E002EFED70D0E006E002EFED71200BD
:10350000580E0B01A16F9488040E006E002EFED79A
:103510009486040E006E002EFED78B989498040EAD
:10352000006E002EFED78B9694960D0E006E002E28
:10353000FED7A151FE0BA26FCA6F000185EC11F0FE
:103540000D0E006E002EFED7A0CBCAFB85EC11F04D
:103550000D0E006E002EFED794980000948682A671
:10356000FED7040E006E002EFED700D00000948817
:10357000040E006E002EFED70F0E006E002EFED73A
:1035800000D012000B01816B826B0701556B3E0E60
:10359000546F576B450E566F580E586F0A0E0D013B
:1035A000B66F000117EC13F057C783FB0B01835173
:1035B000010B816F56C782FB0B01580EC66F81CB82
:1035C000C7FB82CBC8FB0001C0EC11F00A0E0D0155
:1035D000B66F000117EC13F0100E0B01816F58C786
:1035E00082FB0B01580EC66F81CBC7FB82CBC8FB99
:1035F0000001C0EC11F00A0E0D01B66F000117ECCE
:1036000013F055C783FB0B01846B010E8317846B8A
:1036100083511009816F54C782FB0B015E0EC66F88
:1036200081CBC7FB82CBC8FB0001C0EC11F092EF4D
:103630001BF0938681A675D00701556B300E546F31
:10364000576B310E566F120E586F040E0B01816FBF
:10365000FA0E0D01B66F000117EC13F00B01812F6C
:10366000F7D754C781FB0B01826BA26B54C7A3FB36
:103670000001FDDEC80E0D01B66F000117EC13F05E
:1036800055C781FB0B01826B010E8117826BA26F04
:1036900081CBA3FB0001EBDEC80E0D01B66F00016C
:1036A00017EC13F056C781FB0B01826B020EA26F61
:1036B00056C7A3FB0001DBDEC80E0D01B66F00018B
:1036C00017EC13F057C781FB0B01826B010E8117BA
:1036D000826B030EA26F81CBA3FB0001C8DEC80E74
:1036E0000D01B66F000117EC13F0070158517F0B65
:1036F0000B01816F040EA26F81CBA3FB0001B7DE2B
:10370000C80E0D01B66F000117EC13F00B01A06B92
:103710000001F6DE640E0D01B66F000117EC13F028
:1037200001D030D712000B01826B400E9B6F010E4F
:103730009C6F00013AEC12F001C082FB070151516D
:103740000B01825D02E1812D02D082CB51F7000195
:10375000B4EFABF0016603D0026602D007D0022AB4
:1037600000C0EEFF012EFCD7022EFAD712000D0189
:10377000B8BF10D00F0E006EB73900160A0E005CED
:1037800003E2300E002602D0B85100260050A4A853
:10379000FED76D6E0F0EB7170A0EB75D02E2300E40
:1037A00002D0B89FB851B727B751A4A8FED76D6E05
:1037B000000112000D019E6B9F6B9CCDE9FF9DCD1A
:1037C000EAFFEFCF9FFD9F534DE0070151AD08D0B9
:1037D0000D0EA4A8FED76D6E0A0EA4A8FED76D6EBE
:1037E000010E0D019E6F9E519F5D30E3070151ADAB
:1037F00016D0036A0D019E519C25E96E9D51032050
:10380000EA6EEFCFA0FDA0CDB7FD570EB86F000157
:10381000AEDF200EA4A8FED76D6E07D00701010E03
:103820000D01B66F000117EC13F0036A0D019E51F4
:103830009C25E96E9D510320EA6EEFCFA0FDA051BB
:103840000001DEEC0FF00D019E2BCDD7070151AD2D
:1038500008D00D0EA4A8FED76D6E0A0EA4A8FED740
:103860006D6E0D01000112000C01D351090805E332
:10387000300ED325016E05D004D0370ED325016E4E
:1038800000D0000112000900F55211E0F6CFACFDA6
:10389000F7CFADFDF8CFAEFDF550A4A8FED76D6E05
:1038A000ACCDF6FFADCDF7FFAECDF8FFECD71200F3
:1038B0000D01B751B903F3CF01F0F4CF00F0BA0313
:1038C000F3500026B851B903F3500020026E0001F6
:1038D00012000900F6CFB7FDF7CFB8FDF8CFB9FD5C
:1038E000F550A4A8FED76D6EB7CDF6FFB8CDF7FFA3
:1038F000B9CDF8FF0D01B62F01D002D00001E9D7F4
:1039000000011200EACFBEFDE9CFBDFD0D01B739C0
:10391000F009B96FB927E20FBA6F320FBC6FB75118
:103920000F0BBA27BA27BC27E90FBB6FBB27BB27F2
:10393000B6390F0BBB27BC27BB37BC37BC1FBC3706
:10394000B6510F0BBC27B937070EB86F0A0EBB076D
:10395000BC27FDE3BA07BB27FDE3B907BA27FDE3A0
:10396000B807B927FDE30D0EEA6EB80EE96E070E33
:10397000BD15BD9DE926BC0EE95CD8B4BD8DEF50E8
:10398000006E08E1BDBD06D0BDB90CD0BDB702D0F8
:10399000200E03D0BD87BD99300E00260050A4A88C
:1039A000FED76D6EEE50BDADE6D700011200016A84
:1039B000026A006A036A0D01BE5102E1BD5118E0BE
:1039C000100EBF6FD890BB37BC3700360336BE51E0
:1039D000035C02E1BD51005C07E3BD51005ED8A06D
:1039E0000306BE51035ED88001360236BF2FEAD7E8
:1039F00000011200780E09016E25E96E070E6F2195
:103A0000EA6EEFCFB8FD0D01010E09016E250D0123
:103A1000B96F000E09016F210D01BA6FBC6FB9CDEE
:103A2000BBFD010EBE6FF40EBD6F0001C0DF00C014
:103A30006EF9090103C06FF96C516E5D04E16D51BF
:103A40006F5D01E1309A0D01B8CD01F00001120067
:103A50000C01EA6BE96BEC6BEB6BED9130BA45D086
:103A6000EACCB8FDE9CCB7FD0D01BA6B320EB96FE7
:103A700000011EDF02C0EFFC01C0EEFC0C01E751AB
:103A8000025C28E303E1E651EE5D24E3070151AD5A
:103A90001ED0EC0EF66E1A0EF76E000EF86E0B0EC0
:103AA0000D01B66F000115DF100EE96EE7CCB7FD12
:103AB000E6CCB6FD27DFFA0EF66E1A0EF76E000E94
:103AC000F86E070E0D01B66F000103DF0701000E4F
:103AD000016EACD1320E0D01B66F000117EC13F080
:103AE0000C01E92BD8B4EA2BB9D7E4CCEAFFE3CC3C
:103AF000E9FF006A026AE5CC01F000012BDE070154
:103B000051AD0CD0200EA4A8FED76D6E2D0EA4A82A
:103B1000FED76D6E200EA4A8FED76D6E30BA1CD0F5
:103B2000EACCB8FDE9CCB7FD0D01BA6B320EB96F26
:103B30000001BEDE02C0F0FC01C0EFFC0C0102502F
:103B4000E75DD8A050D1D8B402D0070105D0E65126
:103B5000EF5DD8B048D1070130AAFBD00C01E3518A
:103B6000EB25016EE451EC21036E01C0EEFCEF6F1A
:103B7000000140DFEFCCEAFFEECCE9FF01C0EFFF30
:103B80000C01EDB1A6D0E8533AE1E351EB25E96E23
:103B9000E451EC21EA6EEF50020830E1E351EB25ED
:103BA000E96EE451EC21EA6EEFCFF0FCE4CCEAFFE1
:103BB000E3CCE9FFF0CCEFFFEC6B010EEB6F0701FC
:103BC00051AD1AD00C01E3CCE9FFE4CCEAFFEFCF12
:103BD000EEFC5B0EA4A8FED76D6E200EA4A8FED747
:103BE0006D6EEECCB7FD370E0D01B86F0001BFDD75
:103BF000200EA4A8FED76D6E0C01ED8169D0EB53A9
:103C000033E1EC5331E1E351EB25E96EE451EC2172
:103C1000EA6EEFCFF0FCE4CCEAFFE3CCE9FFF0CCB6
:103C2000EFFFEC6B010EEB6F070151AD1BD00C01E8
:103C3000E3CCE9FFE4CCEAFFEFCFEEFC5B0EA4A8F7
:103C4000FED76D6E200EA4A8FED76D6EEECCB7FD2C
:103C5000370E0D01B86F00018ADD200EA4A8FED733
:103C60006D6E070134D00C01070151AD14D00C0169
:103C7000E351EB25E96EE451EC21EA6EEFCFEEFC67
:103C8000EECCB7FD370E0D01B86F000170DD200ED0
:103C9000A4A8FED76D6E0C01E351EB25E96EE4514B
:103CA000EC21EA6EEF500D0813E1070151AD0CD085
:103CB0005D0EA4A8FED76D6E0A0EA4A8FED76D6E89
:103CC0000D0EA4A8FED76D6E010E016EAFD00C01D3
:103CD00041D0070151AD14D00C01E351EB25E96E41
:103CE000E451EC21EA6EEFCFEEFCEECCB7FD370EDF
:103CF0000D01B86F00013BDD200EA4A8FED76D6E4C
:103D00000C01E351EB25E96EE451EC21EA6EEF5032
:103D1000030813E1070151AD0CD05D0EA4A8FED736
:103D20006D6E0A0EA4A8FED76D6E0D0EA4A8FED768
:103D30006D6E010E016E7AD00C01EB2BD8B4EC2B1A
:103D4000EC5303E1E551EB5D05E3FF0E016E070166
:103D50006DD00C0130BA45D0EACCB8FDE9CCB7FD46
:103D60000D01BA6B320EB96F0001A2DD02C0EFFC8B
:103D700001C0EEFC0C01E751025C28E303E1E651CF
:103D8000EE5D24E3070151AD1ED0020EF66E1B0E50
:103D9000F76E000EF86E0B0E0D01B66F000199DD87
:103DA000100EE96EE7CCB7FDE6CCB6FDABDD100E2C
:103DB000F66E1B0EF76E000EF86E070E0D01B66F55
:103DC000000187DD0701000E016E30D0320E0D01BB
:103DD000B66F000117EC13F00C01E92BD8B4EA2BF5
:103DE000B9D707019BD6070151AD1ED0180EF66E4C
:103DF0001B0EF76E000EF86E0B0E0D01B66F000174
:103E000068DD100EE96EE7CCB7FDE6CCB6FD7ADDD5
:103E1000260EF66E1B0EF76E000EF86E070E0D01E5
:103E2000B66F000156DD0701000E016E00011200A1
:103E3000070151AD08D0DA0EF66E1A0EF76E000EBD
:103E4000F86E000120DD0C0E0C01E46FD50EE36F5F
:103E50000D0EE56FD3CCE7FCD2CCE6FCD4CCE8FC6D
:103E60000001F6DD012C08D00C01D651450803E015
:103E7000010E016E04D00001FF0E016E0C01000165
:103E800012000D019C6B30AA06D00001B3DD01C009
:103E90009CFD0D01F8D70901706B000112000B01A8
:103EA000D091080ED16F020ED26F510ED36F530E08
:103EB000D46F410ED56F3A0ED66F330ED76F300EDA
:103EC000D86F030ED96F050EDA6F020EDB6F510E3D
:103ED000DC6F470EDD6F520EDE6F030EDF6F050ED7
:103EE000E06F020EE16F510EE26F470EE36F420E7C
:103EF000E46F030EE56F050EE66F020EE76F510EDD
:103F0000E86F410EE96F570EEA6F030EEB6F050E77
:103F1000EC6F020EED6F510EEE6F540EEF6F440E0C
:103F2000F06F030EF16F050EF26F020EF36F510E7C
:103F3000F46F430EF56F470EF66F030EF76F080E22
:103F4000F86F020EF96F510EFA6F530EFB6F440EAD
:103F5000FC6F3A0EFD6F350EFE6F300EFF6F030ED5
:103F60000C01006F050E016F020E026F510E036F00
:103F7000520E046F530E056F030E066F050E076F8A
:103F8000020E086F510E096F520E0A6F560E0B6F1C
:103F9000030E0C6F050E0D6F020E0E6F510E0F6F9C
:103FA000470E106F550E116F030E126F050E136F33
:103FB000020E146F510E156F530E166F560E176FBB
:103FC000030E186F050E196F020E1A6F510E1B6F3C
:103FD000530E1C6F460E1D6F030E1E6F080E1F6FD3
:103FE000020E206F510E216F530E226F440E236F6D
:103FF0003A0E246F360E256F350E266F030E276F8F
:10400000080E286F020E296F510E2A6F530E2B6F68
:10401000410E2C6F3A0E2D6F380E2E6F370E2F6F0C
:10402000030E306F0B0E316F020E326F4F0E336F77
:10403000530E346F410E356F3A0E366F330E376FB5
:10404000300E386F3A0E396F380E3A6F3B6B030EF5
:104050003C6F080E3D6F020E3E6F4F0E3F6F520ECB
:10406000406F470E416F3A0E426F436B446B030E35
:10407000456F080E466F020E476F4F0E486F420E97
:10408000496F470E4A6F3A0E4B6F4C6B4D6B030EE8
:104090004E6F070E4F6F020E506F4F0E516F410E55
:1040A000526F570E536F3A0E546F556B030E566F87
:1040B000080E576F020E586F4F0E596F540E5A6FFD
:1040C000440E5B6F3A0E5C6F5D6B5E6B030E5F6F51
:1040D000080E606F020E616F4F0E626F430E636FCA
:1040E000470E646F3A0E656F666B676B030E686F01
:1040F0000B0E696F020E6A6F4F0E6B6F530E6C6F73
:10410000440E6D6F3A0E6E6F350E6F6F300E706F1E
:104110003A0E716F726B736B030E746F070E756FCF
:10412000020E766F4F0E776F520E786F530E796FC7
:104130003A0E7A6F7B6B030E7C6F090E7D6F020E59
:104140007E6F4F0E7F6F520E806F560E816F3A0E4C
:10415000826F836B846B856B030E866F080E876F8F
:10416000020E886F4F0E896F470E8A6F550E8B6F48
:104170003A0E8C6F8D6B8E6B030E8F6F0A0E906FE5
:10418000020E916F4F0E926F530E936F410E946F0C
:104190003A0E956F380E966F976F3A0E986F996B2F
:1041A000030E9A6F070E9B6F020E9C6F580E9D6F49
:1041B000530E9E6F460E9F6F3A0EA06FA16B030EBB
:1041C000A26F050EA36F020EA46F4F0EA56F570EC0
:1041D000A66F530EA76F030EA86F050EA96F020EF0
:1041E000AA6F4F0EAB6F410EAC6F530EAD6F030E47
:1041F000AE6F0A0EAF6F020EB06F4F0EB16F530E5F
:10420000B26F410EB36F3A0EB46F380EB56F370E02
:10421000B66F3A0EB76FB86B030EB96F0B0EBA6F6D
:10422000020EBB6F4F0EBC6F530EBD6F440EBE6FC0
:104230003A0EBF6F360EC06F350EC16F3A0EC26FA9
:10424000C36BC46B030EC56F040EC66F230EC76F1E
:104250004F0EC86F310EC96F0D0ECA6F050ECB6FB2
:10426000230ECC6F440ECD6F410ECE6FCF6B0D0E73
:10427000D06F0B01CE51010A0001D8B467D0030AF8
:10428000D8B46DD0010AD8B473D0070AD8B479D0A5
:10429000010AD8B47FD0030AD8B485D0140AD8B4A0
:1042A0008BD0180AD8B491D01E0AD8B497D0020A7D
:1042B000D8B49DD0010AD8B4A3D04D0AD8B4A9D09F
:1042C000060AD8B4AFD03D0AD8B4B5D07D0AD8B468
:1042D000BBD0010AD8B4C4D0030AD8B4CAD0010AEA
:1042E000D8B4D3D03F0AD8B4D9D0010AD8B4E2D0D8
:1042F000060AD8B4EBD00C0AD8B40BD1040AD8B44F
:1043000036D13C0AD8B461D1280AD8B49AD16B0A04
:10431000D8B4BAD1020AD8B4DAD1010AD8B4FAD1E1
:104320000E0AD8B41AD23F0AD8B42BD2230AD8B472
:104330004BD2030AD8B457D20E0AD8B463D2020AB9
:10434000D8B46FD2150AD8B478D283D20C0E0D012E
:104350009D6F130E9C6F0001DAEC1BF07CD20B0EEC
:104360000D019D6FE60E9C6F0001DAEC1BF073D21D
:104370000C0E0D019D6F010E9C6F0001DAEC1BF01D
:104380006AD20B0E0D019D6FD10E9C6F0001DAEC0D
:104390001BF061D20B0E0D019D6FDA0E9C6F0001B8
:1043A000DAEC1BF058D20B0E0D019D6FE00E9C6FE6
:1043B0000001DAEC1BF04FD20C0E0D019D6F070EC1
:1043C0009C6F0001DAEC1BF046D20C0E0D019D6FC4
:1043D0000D0E9C6F0001DAEC1BF03DD20B0E0D01AF
:1043E0009D6FEC0E9C6F0001DAEC1BF034D20B0ECB
:1043F0000D019D6FF20E9C6F0001DAEC1BF02BD2C9
:104400000B0E0D019D6FF80E9C6F0001DAEC1BF096
:1044100022D20C0E0D019D6F190E9C6F0001DAEC7B
:104420001BF019D20C0E0D019D6F280E9C6F000120
:10443000DAEC1BF010D20C0E0D019D6F1F0E9C6F5D
:104440000001DAEC1BF007D2300E0C01556F0C0E98
:104450000D019D6F4F0E9C6F0001DAEC1BF0FBD13C
:104460000C0E0D019D6FA30E9C6F0001DAEC1BF08A
:10447000F2D1310E0C01556F0C0E0D019D6F4F0ED8
:104480009C6F0001DAEC1BF0E6D10C0E0D019D6F64
:10449000A90E9C6F0001DAEC1BF0DDD1310E0C018E
:1044A0007B6F0C0E0D019D6F750E9C6F0001DAEC99
:1044B0001BF0D1D1300E0C017B6F0C0E0D019D6FE6
:1044C000750E9C6F0001DAEC1BF0C5D10701713944
:1044D000006E0F0E001600500F0B0C01D16FD36F42
:1044E000000134EC1CF001C03AFC070171510F0BC4
:1044F0000C01D16FD36F000134EC1CF001C03BFC08
:104500000C0E0D019D6F310E9C6F0001DAEC1BF05B
:10451000A2D1070167310C01D26F070166310C018E
:10452000D16FD233D133D233D133D233D1330F0E13
:10453000D217D117D26BD1CCD3FC000134EC1CF0D4
:1045400001C043FC070166510F0B0C01D16FD26B08
:10455000D36F000134EC1CF001C044FC0C0E0D01C3
:104560009D6F3D0E9C6F0001DAEC1BF074D10701CA
:1045700069310C01D26F070168310C01D16FD23360
:10458000D133D233D133D233D1330F0ED217D11727
:10459000D26BD1CCD3FC000134EC1CF001C04CFC3C
:1045A000070168510F0B0C01D16FD26BD36F000163
:1045B00034EC1CF001C04DFC0C0E0D019D6F460E3D
:1045C0009C6F0001DAEC1BF046D163C7D1FC0C01F3
:1045D000D26B0F0ED117D26BD1CCD3FC000134ECCF
:1045E0001CF001C083FC070163310C01D26F07018D
:1045F00062310C01D16FD233D133D233D133D233C4
:10460000D1330F0ED217D117D26BD1CCD3FC00010E
:1046100034EC1CF001C084FC070162510F0B0C014B
:10462000D16FD26BD36F000134EC1CF001C085FC5C
:104630000C0E0D019D6F7D0E9C6F0001DAEC1BF0DE
:104640000AD107016539006E0F0E001600500F0BDE
:104650000C01D16FD36F000134EC1CF001C08DFC54
:10466000070165510F0B0C01D16FD36F000134ECC2
:104670001CF001C08EFC0C0E0D019D6F870E9C6F0F
:104680000001DAEC1BF0E7D007017239006E0F0E63
:10469000001600500F0B0C01D16FD36F000134ECEA
:1046A0001CF001C05DFC070172510F0B0C01D16FB2
:1046B000D36F000134EC1CF001C05EFC0C0E0D0148
:1046C0009D6F570E9C6F0001DAEC1BF0C4D0070100
:1046D0007339006E0F0E001600500F0B0C01D16FD6
:1046E000D36F000134EC1CF001C066FC070173516C
:1046F0000F0B0C01D16FD36F000134EC1CF001C023
:1047000067FC0C0E0D019D6F600E9C6F0001DAECD2
:104710001BF0A1D007017439006E0F0E0016005077
:104720000F0B0C01D16FD36F000134EC1CF001C0F2
:1047300072FC070174510F0B0C01D16FD36F000194
:1047400034EC1CF001C073FC0C0E0D019D6F690E62
:104750009C6F0001DAEC1BF07ED007014B510F0B70
:104760000C01D16FD36F000134EC1CF001C0B8FC18
:104770000C0E0D019D6FAF0E9C6F0001DAEC1BF06B
:104780006AD007014C39006E0F0E001600500F0B57
:104790000C01D16FD36F000134EC1CF001C0C3FCDD
:1047A00007014C510F0B0C01D16FD36F000134EC9A
:1047B0001CF001C0C4FC0C0E0D019D6FBA0E9C6F65
:1047C0000001DAEC1BF047D0310E0C01CF6F0C0E5C
:1047D0000D019D6FCB0E9C6F0001DAEC1BF00B01FD
:1047E000D081000138D0300E0C01CF6F0C0E0D01BE
:1047F0009D6FCB0E9C6F0001DAEC1BF00B01D0819A
:10480000000129D0310E0C01C96F0C0E0D019D6FF6
:10481000C60E9C6F0001DAEC1BF00B01D081000189
:104820001AD0310E0C01996F0C0E0D019D6F900E78
:104830009C6F0001DAEC1BF00ED0340E0C01A16F5E
:104840000C0E0D019D6F9B0E9C6F0001DAEC1BF0AE
:1048500002D01BD000D00B01CF2D18D0320E0D018D
:10486000B66F000117EC13F0000E0B01D0B1010E72
:104870000C01D16F070ED36FD00ED26FD1CCD4FC08
:10488000000118EC1FF041EC1FF00B0100011200B9
:10489000580E0B01BB6FBC6B9488040E006E002E8B
:1048A000FED79486040E006E002EFED78B98949847
:1048B000040E006E002EFED78B9694960D0E006EA1
:1048C000002EFED7BB51FE0BBD6FCA6F000185ECF9
:1048D00011F00D0E006E002EFED7BACBCAFB85EC90
:1048E00011F00D0E006E002EFED79488040E006E9F
:1048F000002EFED79486040E006E002EFED782A6F0
:10490000FED78B989498040E006E002EFED78B96DF
:1049100094960D0E006E002EFED70B01BB510109BF
:10492000BD6FCA6F000185EC11F00D0E006E002EF8
:10493000FED7006A05EC12F001C0BCFB0D0E006E44
:10494000002EFED794980000948682A6FED7040E0F
:10495000006E002EFED700D000009488040E006E7A
:10496000002EFED70F0E006E002EFED700D00B01DA
:10497000BCCB01F000011200938681A67DD0B1CBA3
:1049800003F00B01B0CBB6FBB1CBB7FB010EBA6F96
:1049900000017EDFB7CBEAFFB6CBE9FFEC6AED5250
:1049A00001C0EFFF0B01B0CBB6FBB1CBB7FBB1CB76
:1049B00003F0B0CBE9FFB1CBEAFFECCFB9FBED528E
:1049C000EFCFB8FBB8CBB9FBB86BBA6B000160DFB7
:1049D0000B01B8510110B9CB03F0B7CBEAFFB6CB4E
:1049E000E9FFB9CBECFFED52EF6EB3CB03F0B2CBE6
:1049F000B6FBB3CBB7FB030EBA6F000149DFB7CBF1
:104A0000EAFFB6CBE9FFEC6AED5201C0EFFF0B0104
:104A1000B2CBB6FBB3CBB7FBB3CB03F0B2CBE9FF62
:104A2000B3CBEAFFECCFB9FBED52EFCFB8FBB8CB7D
:104A3000B9FBB86B020EBA6F00012ADF0B01B85147
:104A40000110B9CB03F0B7CBEAFFB6CBE9FFB9CB86
:104A5000ECFFED52EF6EB5CB03F0B4CBB6FBB5CBAC
:104A6000B7FB040EBA6F000113DFB7CBEAFFB6CB7A
:104A7000E9FF01C0EFFF00D01200070151AD09D0DE
:104A8000C20EF66E1A0EF76E000EF86E000143ECC1
:104A90001CF0CFCBE4FCCECBE3FCD0CBE5FCD2CBFF
:104AA000E7FCD1CBE6FCD3CBE8FC000128EC1DF001
:104AB000012C0ED0010E0B01CE25E96E000ECF2188
:104AC000EA6EEF50450803E0010E016E04D00001CC
:104AD000FF0E016E0B01000112000B01DE513908BF
:104AE00005E2370EDE5D016E05D004D0300EDE5DCE
:104AF000016E00D0000112000C012651016A255DF3
:104B000003E225CC00F00CD0006A080E276F253791
:104B100000362651005CD8B0006E0136272FF7D73B
:104B200000011200015023CC25FC640E0C01266FFD
:104B30000001E2DF00C023FC0150300E08E10C014F
:104B400024A30ED024B70CD024B9200E04D00C011D
:104B500024972499248101260150A4A8FED76D6EC4
:104B600023CC25FC0A0E266F0001C6DF00C023FC03
:104B70000150300E08E10C0124B70BD024A109D05C
:104B800024B9200E000101260150A4A8FED76D6EA5
:104B90000C01300E23272351A4A8FED76D6E00010F
:104BA00012000C01206B1F6B216B229130BA46D092
:104BB00020CCB8FD1FCCB7FD0D01BA6B320EB96F1A
:104BC000000158EC1CF002C024FC01C023FC0C01C5
:104BD000245303E11E51235D26E3070151AD20D08C
:104BE000B40EF66E1D0EF76E000EF86E0B0E0D0174
:104BF000B66F000169EC1CF01ECC23FC1B0E0C01EF
:104C0000246F00018FDFC10EF66E1D0EF76E000ED1
:104C1000F86E070E0D01B66F000169EC1CF007017C
:104C2000000E016E29D1320E0D01B66F000117EC96
:104C300013F00C011F2BD8B4202BB8D71CCCEAFFE3
:104C40001BCCE9FF006A026A1DCC01F00001AAEC4E
:104C50001BF0070151AD0CD0200EA4A8FED76D6E3D
:104C60002D0EA4A8FED76D6E200EA4A8FED76D6EE3
:104C700030AADED0036A0C0121511B25016E1C51A4
:104C8000032201C023FC03C024FC0001FAEC1CF049
:104C900024CCEAFF23CCE9FF01C0EFFF0C0122B1D5
:104CA0003ED0036A21511B25E96E1C510320EA6E98
:104CB000EF50FE0833E11CCC03F0036A21511B25A1
:104CC000E96E1C510320EA6EEFCF25FC1CCCEAFFF5
:104CD0001BCCE9FF25CCEFFF010E216F070151AD81
:104CE0001BD00C011BCCE9FF1CCCEAFFEFCF23FC4F
:104CF0005B0EA4A8FED76D6E200EA4A8FED76D6E25
:104D000023CCB7FD370E0D01B86F0001B7EC1BF0D7
:104D1000200EA4A8FED76D6E0C0122813FD00701A2
:104D200051AD17D0036A0C0121511B25E96E1C51AE
:104D30000320EA6EEFCF23FC23CCB7FD370E0D0125
:104D4000B86F0001B7EC1BF0200EA4A8FED76D6E63
:104D50000701036A0C0121511B25E96E1C51032038
:104D6000EA6EEF50EF0811E1070151AD0AD0CA0E0B
:104D7000F66E1D0EF76E000EF86E000143EC1CF08F
:104D80000701010E016E78D00C01212B1D51215D10
:104D900005E3FF0E016E07016FD00C0130BA46D05B
:104DA00020CCB8FD1FCCB7FD0D01BA6B320EB96F28
:104DB000000158EC1CF002C024FC01C023FC0C01D3
:104DC000245303E11E51235D26E3070151AD20D09A
:104DD000D00EF66E1D0EF76E000EF86E0B0E0D0166
:104DE000B66F000169EC1CF01ECC23FC1B0E0C01FD
:104DF000246F000197DEDD0EF66E1D0EF76E000EBD
:104E0000F86E070E0D01B66F000169EC1CF007018A
:104E1000000E016E31D0320E0D01B66F000117EC9D
:104E200013F00C011F2BD8B4202BB8D7070120D7C3
:104E300051AD20D0E60EF66E1D0EF76E000EF86E28
:104E40000B0E0D01B66F000169EC1CF01ECC23FCAB
:104E50001B0E0C01246F000165DEF30EF66E1D0EB5
:104E6000F76E000EF86E070E0D01B66F000169ECCB
:104E70001CF00701000E016E00011200070151AD88
:104E800009D0FC0EF66E1D0EF76E000EF86E0001D6
:104E900043EC1CF00C0E0C011C6F0D0E1B6F1D6FF4
:104EA0000BCC1EFC00017DDE015225E00C011051EF
:104EB000300A000109E0030A0BE0060A11E00C0ABF
:104EC0000FE0080A11E00CD0010E016E16D010D0D0
:104ED0000701605304E1010E016E00010ED00001D4
:104EE000FF0E016E0AD004D0010E016E06D000D074
:104EF0000701D0D70001000E016E12000B01E06B1C
:104F0000DF6B060EE16FE269300EE36FE46F010EB6
:104F1000E56F870EE66FEF0EE76F070EE86FE96942
:104F2000300EEA6FEB6F010EEC6F860EED6F300EF8
:104F3000EE6FEF0EEF6F070EF06FF169300EF26F4C
:104F4000F36F010EF46F900EF56F300EF66FEF0EEB
:104F5000F76F080EF86FF969300EFA6FFB6F010EEC
:104F6000FC6FA60EFD6F300EFE6FFF6FEF0E0C0193
:104F7000006F090E016F0269300E036F046F010E9E
:104F8000056FE10E066F300E076F380E086F300E9A
:104F9000096FEF0E0A6F0B01DD515E0A000150E050
:104FA0003E0A57E0610A5EE0080AD8B464D0010AFC
:104FB000D8B46FD0440AD8B47AD0010AD8B485D016
:104FC0006D0AD8B490D0010AD8B4A6D0460AD8B495
:104FD000BCD0500AD8B4D2D0670AD8B413D17B0A57
:104FE000D8B434D1040AD8B45AD16F0AD8B480D115
:104FF000090AD8B4A6D10E0AD8B4BAD17C0AD8B45A
:10500000CED1270AD8B4E2D1010AD8B4EDD15F0AD3
:10501000D8B4F8D1030AD8B403D2150AD8B40ED242
:10502000070AD8B422D2600AD8B436D2610AD8B4FA
:105030004AD2750AD8B45ED2410AD8B472D298D294
:105040000B0E0D019D6FF00E9C6F0001DAEC1BF052
:1050500091D20B0E0D019D6FE80E9C6F0001DAECF2
:105060001BF088D20B0E0D019D6FE10E9C6F0001AD
:10507000DAEC1BF07FD2C30E0B01ED6F310EEE6F39
:105080000B0E0D019D6FE80E9C6F0001DAEC1BF01A
:1050900071D2C30E0B01ED6F320EEE6F0B0E0D01D0
:1050A0009D6FE80E9C6F0001DAEC1BF063D2A00E3E
:1050B0000B01F56F310EF66F0B0E0D019D6FF00EAB
:1050C0009C6F0001DAEC1BF055D2A00E0B01F56FBE
:1050D000300EF66F0B0E0D019D6FF00E9C6F0001F0
:1050E000DAEC1BF047D207014E51300811E0840E74
:1050F0000B01F56F300EF66F07014E6F0B0E0D01B1
:105100009D6FF00E9C6F0001DAEC1BF004D00701DC
:105110000B01DE6B00012ED207014E51310811E068
:10512000840E0B01F56F310EF66F07014E6F0B0EFB
:105130000D019D6FF00E9C6F0001DAEC1BF004D0A6
:1051400007010B01DE6B000115D207014E51320839
:1051500011E0840E0B01F56F320EF66F07014E6FF2
:105160000B0E0D019D6FF00E9C6F0001DAEC1BF031
:1051700004D007010B01DE6B0001FCD164C7E0FB2A
:105180000B01DF6BE0CBBCFDDFCBBBFD0D01BE6BCC
:1051900077C7BDFD0001D7EC1CF002C0E0FB01C0E9
:1051A000DFFB0B01DF5302E1E05304E0020EDF27D7
:1051B000000EE023E051000802E2E06BDF69DFCB84
:1051C00000F0003A0F0E001600500F0B0C010B6F91
:1051D000D36F000134EC1CF001C0FEFB0B01DF516A
:1051E0000F0B0C010B6FD36F000134EC1CF001C0EE
:1051F000FFFB0B0E0D019D6FF80E9C6F0001DAECAA
:105200001BF0B8D1070172C700F0003A0F0E00166C
:1052100000500F0B0C010B6FD36F000134EC1CF02E
:1052200001C008FC070172510F0B0C010B6FD36F0B
:10523000000134EC1CF001C009FC0C0E0D019D6F47
:10524000010E9C6F0001DAEC1BF094D1E10E0C0111
:10525000066F310E076F070166C700F0003A0F0EA8
:10526000001600500F0B0C010B6FD36F000134ECD4
:105270001CF001C008FC070166510F0B0C010B6FFD
:10528000D36F000134EC1CF001C009FC0C0E0D01C1
:105290009D6F010E9C6F0001DAEC1BF06BD1E10EEB
:1052A0000C01066F330E076F070168C700F0003A64
:1052B0000F0E001600500F0B0C010B6FD36F000187
:1052C00034EC1CF001C008FC070168510F0B0C0105
:1052D0000B6FD36F000134EC1CF001C009FC0C0E05
:1052E0000D019D6F010E9C6F0001DAEC1BF042D1A5
:1052F000E10E0C01066F390E076F07016AC700F057
:10530000003A0F0E001600500F0B0C010B6FD36FFD
:10531000000134EC1CF001C008FC07016A510F0BBE
:105320000C010B6FD36F000134EC1CF001C009FCC1
:105330000C0E0D019D6F010E9C6F0001DAEC1BF04D
:1053400019D1AD0E0B01F56F07016F510F0B0C0159
:105350000B6FD36F000134EC1CF001C0F6FB0B0E99
:105360000D019D6FF00E9C6F0001DAEC1BF002D175
:10537000B60E0B01F56F07016E510F0B0C010B6F91
:10538000D36F000134EC1CF001C0F6FB0B0E0D01D5
:105390009D6FF00E9C6F0001DAEC1BF0EBD0AE0EAF
:1053A0000B01F56F070165510F0B0C010B6FD36FEC
:1053B000000134EC1CF001C0F6FB0B0E0D019D6FDB
:1053C000F00E9C6F0001DAEC1BF0D4D0A70E0B019D
:1053D000F56F300EF66F0B0E0D019D6FF00E9C6F8A
:1053E0000001DAEC1BF0C6D0A70E0B01F56F310EF1
:1053F000F66F0B0E0D019D6FF00E9C6F0001DAEC45
:105400001BF0B8D0B50E0B01F56F300EF66F0B0E1A
:105410000D019D6FF00E9C6F0001DAEC1BF0AAD01D
:10542000B50E0B01F56F310EF66F0B0E0D019D6F72
:10543000F00E9C6F0001DAEC1BF09CD0F10E0B011A
:10544000F56F070175510F0B0C010B6FD36F000146
:1054500034EC1CF001C0F6FB0B0E0D019D6FF00E3D
:105460009C6F0001DAEC1BF085D0F20E0B01F56F9A
:10547000070174510F0B0C010B6FD36F000134EC5B
:105480001CF001C0F6FB0B0E0D019D6FF00E9C6F22
:105490000001DAEC1BF06ED0F30E0B01F56F070183
:1054A0006B510F0B0C010B6FD36F000134EC1CF030
:1054B00001C0F6FB0B0E0D019D6FF00E9C6F0001FD
:1054C000DAEC1BF057D0F40E0B01F56F07017351A6
:1054D0000F0B0C010B6FD36F000134EC1CF001C0FB
:1054E000F6FB0B0E0D019D6FF00E9C6F0001DAECC8
:1054F0001BF040D0F50E0B01F56F070171510F0B3A
:105500000C010B6FD36F000134EC1CF001C0F6FBF3
:105510000B0E0D019D6FF00E9C6F0001DAEC1BF07D
:1055200029D0E40E0B01FD6F07016CC700F0003AB3
:105530000F0E001600500F0B0C010B6FD36F000104
:1055400034EC1CF001C0FEFB07016C510F0B0C0189
:105550000B6FD36F000134EC1CF001C0FFFB0B0E8E
:105560000D019D6FF80E9C6F0001DAEC1BF002D06C
:105570000BD000D00B01DE2D08D0070E0C010C6FF4
:10558000D00E0B6F00017ADC0B01000112000B0141
:10559000DE6BDF6BE16BE06BC9CBE9FFCACBEAFFE7
:1055A000EF6A30BA49D0E1CBB8FDE0CBB7FD0D01D1
:1055B000BA6B320EB96F000158EC1CF002C0E3FB6D
:1055C00001C0E2FB0B01CD51025C2BE303E1CC51A6
:1055D000E25D27E3070151AD21D02E0EF66E1B0EC2
:1055E000F76E000EF86E100E0D01B66F000169EC3B
:1055F0001CF0100EE96ECDCBB7FDCCCBB6FD82EC26
:105600001CF0410EF66E1B0EF76E000EF86E070EC4
:105610000D01B66F000169EC1CF00701000E016E70
:1056200055D1320E0D01B66F000117EC13F00B01CE
:10563000E02BD8B4E12BB5D70B0EEA6ECE0EE96E97
:10564000006A026A100E016E0001AAEC1BF0320E15
:105650000D01B66F000117EC13F0070151AD0AD030
:105660004A0EF66E1B0EF76E000EF86E000143EC4C
:105670001CF0070130AA58D00B01DE510F08D8B03A
:1056800002D0070151D00001FAEC1CF001C0DFFB91
:10569000070151AD0ED0DFCBB7FD570E0D01B86F2E
:1056A0000001B7EC1BF0200EA4A8FED76D6E07D04A
:1056B0000701010E0D01B66F000117EC13F0070191
:1056C0006051100814E10B01DF51FE0804E1DE6BAC
:1056D000DFCBCEFB0AD0DE2B036ADE51CE0FE96EA4
:1056E0000B0E0320EA6EDFCBEFFF16D007010B0194
:1056F000DF51900803E0DF51F00804E1DE6BDFCBFF
:10570000CEFB0AD0DE2B036ADE51CE0FE96E0B0E04
:105710000320EA6EDFCBEFFF0A0E0D01B66F00012A
:1057200017EC13F00701A6D7020E0B01CB25DE5DA7
:1057300010E2070151AD0AD0560EF66E1B0EF76E41
:10574000000EF86E000143EC1CF00701000E016E24
:10575000BDD0070160511008D8A477D0036A0B01AF
:10576000CB51CE0FE96E0B0E0320EA6EEF504008CE
:1057700012E3CACB03F0036ACB51CE0FE96E0B0ED6
:105780000320EA6EEFCFE4FBCACBEAFFC9CBE9FF07
:10579000E4CBEFFF11D0CACB03F0036ACB51CE0F9D
:1057A000E96E0B0E0320EA6EEF500F0B090FCACB08
:1057B000EAFFC9CBE9FFEF6EC9CBE9FFCACBEAFF2D
:1057C000EF38006EF00E001600C0EFFF010ECB2583
:1057D000036ACE0FE96E0B0E0320EA6EEF5040080D
:1057E00019E3CACB03F0CACBEAFFC9CBE9FFEFCF7D
:1057F000E4FB010ECB25036ACE0FE96E0B0E0320EE
:10580000EA6EEF500F0BE411CACBEAFFC9CBE9FFF8
:10581000EF6E19D0CACB03F0CACBEAFFC9CBE9FFC0
:10582000EFCFE4FB010ECB25036ACE0FE96E0B0E22
:105830000320EA6EEF500F0B090FE411CACBEAFF09
:10584000C9CBE9FFEF6E35D00701CACB03F00B01DE
:10585000036ACB51CE0FE96E0B0E0320EA6EEFCF39
:10586000E4FBCACBEAFFC9CBE9FFE4CBEFFFC9CB2E
:10587000E9FFCACBEAFFEF38006EF00E001600C059
:10588000EFFFCACB03F0CACBEAFFC9CBE9FFEFCFEA
:10589000E4FB010ECB25036ACE0FE96E0B0E03204D
:1058A000EA6EEF500F0BE411CACBEAFFC9CBE9FF58
:1058B000EF6E070151AD08D00A0EA4A8FED76D6E99
:1058C0000D0EA4A8FED76D6E010E016E0001120030
:1058D0000D01B26BB16BB46BB36BB59130BA48D0FC
:1058E000B2CDB8FDB1CDB7FDBA6B320EB96F0001C4
:1058F00058EC1CF002C0B7FD01C0B6FD0D01B0515F
:10590000025C2CE303E1AF51B65D28E3070151AD22
:1059100021D0800EF66E1A0EF76E000EF86E0B0E8A
:105920000D01B66F000169EC1CF0100EE96EB0CDF0
:10593000B7FDAFCDB6FD82EC1CF08E0EF66E1A0EE2
:10594000F76E000EF86E070E0D01B66F000169ECE0
:105950001CF00701000E016E69D10D01320EB66F09
:10596000000117EC13F00D01B12BD8B4B22BB6D750
:10597000ADCDEAFFACCDE9FF006A026AAECD01F021
:105980000001AAEC1BF0070151AD0CD0200EA4A819
:10599000FED76D6E2D0EA4A8FED76D6E200EA4A8A6
:1059A000FED76D6E30BA1DD0B2CDB8FDB1CDB7FD0A
:1059B0000D01BA6B320EB96F000158EC1CF002C039
:1059C000B8FD01C0B7FD0D010250B05DD8A008D1EF
:1059D000D8B402D0070105D0AF51B75DD8B000D11F
:1059E000070130AAB0D00D01AC51B325016EAD5105
:1059F000B421036E01C0B6FDB76F0001FAEC1CF0D4
:105A0000B7CDEAFFB6CDE9FF01C0EFFF0D01B5B19B
:105A10005BD0AC51B325E96EAD51B421EA6EEFCF46
:105A2000B6FD000EB6BF010E01084DE1AC51B32525
:105A3000E96EAD51B421EA6EEF500F0B080813E088
:105A4000AC51B325E96EAD51B421EA6EEF500F0BA6
:105A5000090809E0AC51B325E96EAD51B421EA6EF5
:105A6000EF500F0B30E1AC51B325E96EAD51B421CD
:105A7000EA6EEFCFB8FDADCDEAFFACCDE9FFB8CD12
:105A8000EFFFB46B010EB36F070151AD1AD00D01DA
:105A9000ACCDE9FFADCDEAFFEFCFB6FD5B0EA4A81C
:105AA000FED76D6E200EA4A8FED76D6EB6CDB7FDE5
:105AB000570EB86F0001B7EC1BF0200EA4A8FED75C
:105AC0006D6E0D01B58140D0070151AD14D00D01AF
:105AD000AC51B325E96EAD51B421EA6EEFCFB6FDFE
:105AE000B6CDB7FD370EB86F0001B7EC1BF0200E36
:105AF000A4A8FED76D6E0D01AC51B325E96EAD5172
:105B0000B421EA6EEF3C13D0070151AD0CD05D0E0D
:105B1000A4A8FED76D6E0A0EA4A8FED76D6E0D0E5A
:105B2000A4A8FED76D6E010E016E80D00D01B32BBF
:105B3000D8B4B42BB45303E1AE51B35D05E3FF0E0B
:105B4000016E070173D00D0130BA48D0B2CDB8FD57
:105B5000B1CDB7FDBA6B320EB96F000158EC1CF035
:105B600002C0B7FD01C0B6FD0D01B051025C2CE3CF
:105B700003E1AF51B65D28E3070151AD21D0960E88
:105B8000F66E1A0EF76E000EF86E0B0E0D01B66F64
:105B9000000169EC1CF0100EE96EB0CDB7FDAFCD81
:105BA000B6FD82EC1CF0A40EF66E1A0EF76E000E17
:105BB000F86E070E0D01B66F000169EC1CF00701CD
:105BC000000E016E33D00D01320EB66F000117ECDE
:105BD00013F00D01B12BD8B4B22BB6D70701E2D622
:105BE000070151AD21D0AC0EF66E1A0EF76E000E05
:105BF000F86E0B0E0D01B66F000169EC1CF0100E73
:105C0000E96EB0CDB7FDAFCDB6FD82EC1CF0BA0E9B
:105C1000F66E1A0EF76E000EF86E070E0D01B66FD7
:105C2000000169EC1CF00701000E016E000112007A
:105C3000070151AD09D06A0EF66E1A0EF76E000E0E
:105C4000F86E000143EC1CF00D0E0D01AD6F9E0EC1
:105C5000AC6F0D0EAE6F9DCDB0FD9CCDAFFD0001C4
:105C600037DE015244E00D019F51010A000113E0AB
:105C7000500A1AE0030A18E0330A1CE0030A1AE08B
:105C8000020A1FE0580A23E0790A21E0030A1FE014
:105C9000120A1DE01DD00D019E51880803E1010E7E
:105CA000016E28D0000114D0010E016E0D0122D02A
:105CB00000010ED00D01A051050802E1000108D03D
:105CC0000001FF0E016E0D0115D0000101D000D0C2
:105CD000070151AD0AD0760EF66E1A0EF76E000E61
:105CE000F86E000143EC1CF00701AED70001000E76
:105CF000016E0D0100011200050E0C01006F810EF6
:105D0000016F010E026F036B046F0569050E066FCC
:105D10000769880E086F300E096F010E0A6F0B6954
:105D2000050E0C6F810E0D6F090E0E6F0F6B020EBC
:105D3000106F1169050E126F810E136F090E146F2B
:105D4000040E156F350E166F1769050E186F810E4C
:105D5000196F090E1A6F040E1B6F390E1C6F1D6927
:105D6000050E1E6F810E1F6F090E206F040E216F2E
:105D7000420E226F2369050E246F810E256F090ED6
:105D8000266F040E276F430E286F2969050E2A6FB0
:105D9000810E2B6F090E2C6F040E2D6F440E2E6F8B
:105DA0002F69050E306F810E316F090E326F040EB0
:105DB000336F490E346F3569050E366F810E376FBC
:105DC000090E386F040E396F4B0E3A6F3B69050EA2
:105DD0003C6F810E3D6F090E3E6F040E3F6F4C0EFF
:105DE000406F4169050E426F810E436F090E446F8B
:105DF0007E0E456F590E466F4769050E486F810E3E
:105E0000496F090E4A6F040E4B6F4F0E4C6F4D6970
:105E1000050E4E6F810E4F6F090E506F060E516FBB
:105E2000230E526F5369060E546F810E556F090E83
:105E3000566F7E0E576F010E586F0A0E596F5A69D2
:105E4000060E5B6F810E5C6F090E5D6F7E0E5E6FDE
:105E5000010E5F6F2E0E606F6169060E626F810E1C
:105E6000636F090E646F7E0E656F010E666F470EDD
:105E7000676F6869060E696F810E6A6F090E6B6F36
:105E80007E0E6C6F010E6D6F480E6E6F6F69060EA1
:105E9000706F810E716F090E726F7E0E736F010E3F
:105EA000746F490E756F7669050E776F810E786F86
:105EB000090E796F7E0E7A6F530E7B6F7C69050E2B
:105EC0007D6F810E7E6F090E7F6F7E0E806F540E88
:105ED000816F8269050E836F810E846F090E856F55
:105EE0007E0E866F550E876F8869050E896F810E4D
:105EF0008A6F090E8B6F7E0E8C6F560E8D6F8E69BA
:105F0000050E8F6F810E906F090E916F7E0E926F4E
:105F1000570E936F9469050E956F810E966F090E5B
:105F2000976F7E0E986F580E996F9A69050E9B6F4A
:105F3000810E9C6F090E9D6F040E9E6F4D0E9F6F1C
:105F4000A069050EA16F810EA26F090EA36F040E4A
:105F5000A46F4A0EA56FA669050EA76F890EA86FDC
:105F6000090EA96FAA6B020EAB6FAC69060EAD6F7E
:105F7000810EAE6F010EAF6F040EB06F350EB16FB4
:105F8000B26BB369060EB46F810EB56F010EB66FBA
:105F9000040EB76F390EB86FB96BBA69060EBB6FD6
:105FA000810EBC6F010EBD6F040EBE6F020EBF6F7F
:105FB000C06BC169090EC26F810EC36F010EC46F41
:105FC000040EC56F420EC66FC76BC86BC96BCA6B38
:105FD000CB69060ECC6F810ECD6F010ECE6F040E15
:105FE000CF6F030ED06FD16BD269090ED36F810EC4
:105FF000D46F010ED56F040ED66F430ED76FD86BDA
:10600000D96BDA6BDB6BDC69060EDD6F810EDE6F40
:10601000010EDF6F040EE06FE16FE26BE369090EC2
:10602000E46F810EE56F010EE66F040EE76F440E1C
:10603000E86FE96BEA6BEB6BEC6BED69060EEE6FEC
:10604000810EEF6F010EF06F040EF16F090EF26F0B
:10605000F36BF469F56F810EF66F010EF76F040EA6
:10606000F86F490EF96FFA6BFB6BFC6BFD6BFE6909
:10607000060EFF6F810E0D01006F010E016F040E01
:10608000026F0B0E036F046B0569090E066F810E1C
:10609000076F010E086F040E096F4B0E0A6F0B6B32
:1060A0000C6B0D6B0E6B0F69060E106F810E116F6E
:1060B000010E126F040E136F0C0E146F156B166920
:1060C000090E176F810E186F010E196F040E1A6FEB
:1060D0004C0E1B6F1C6B1D6B1E6B1F6B2069060E1D
:1060E000216F810E226F010E236F7E0E246F590ED9
:1060F000256F266B2769060E286F810E296F010E0A
:106100002A6F040E2B6F0F0E2C6F2D6B2E69090E4C
:106110002F6F810E306F010E316F040E326F4F0EF4
:10612000336F346B356B366B376B3869080E396FEC
:10613000810E3A6F010E3B6F7E0E3C6F010E3D6F7C
:106140000A0E3E6F3F6B020E406F4169080E426FB0
:10615000810E436F010E446F7E0E456F010E466F38
:106160002E0E476F486B496B4A69070E4B6F810EC5
:106170004C6F010E4D6F7E0E4E6F010E4F6F3D0E38
:10618000506F516B5269080E536F810E546F010EA0
:10619000556F7E0E566F010E576F470E586F596B35
:1061A0005A6B5B69090E5C6F810E5D6F010E5E6F4D
:1061B0007E0E5F6F530E606F616B626B636B646B1F
:1061C0006569090E666F810E676F010E686F7E0E3E
:1061D000696F540E6A6F6B6B6C6B6D6B6E6B6F6976
:1061E000090E706F810E716F010E726F7E0E736FEC
:1061F000550E746F756B766B776B786B7969090EDA
:106200007A6F810E7B6F010E7C6F7E0E7D6F560E56
:106210007E6F7F6B806B816B826B8369060E846FF0
:10622000810E856F010E866F7E0E876F570E886F09
:10623000896B8A69060E8B6F810E8C6F010E8D6FD4
:106240007E0E8E6F580E8F6F906B9169090E926F54
:10625000810E936F010E946F040E956F4A0E966F28
:10626000976B986B996B9A6B9B690B01FE51000AB7
:106270000001D8B436D14A0AD8B43CD1060AD8B401
:1062800043D1070AD8B44ED14A0AD8B457D1030A29
:10629000D8B45DD1010AD8B46FD1070AD8B481D17E
:1062A000010AD8B493D1030AD8B4A5D1010AD8B44D
:1062B000B7D10F0AD8B4C9D1020AD8B4DBD1010AC8
:1062C000D8B4EDD1070AD8B4FFD16F0AD8B411D22F
:1062D0006E0AD8B423D2030AD8B435D2010AD8B48E
:1062E00047D21F0AD8B459D2010AD8B46BD2040AD3
:1062F000D8B47DD2010AD8B48FD2020AD8B4A1D2C0
:10630000010AD8B4B3D20F0AD8B4C5D2010AD8B49E
:10631000D7D2030AD8B4E9D2010AD8B4FBD2070A0B
:10632000D8B40DD3010AD8B422D3030AD8B438D3D1
:10633000010AD8B44ED33F0AD8B464D3010AD8B402
:1063400077D3030AD8B48CD3010AD8B4A0D3070AF0
:10635000D8B45EEF35F0010AD8B474EF35F0030A13
:10636000D8B48BEF35F0010AD8B4A2EF35F00F0A9C
:10637000D8B4C5EF35F0010AD8B4DBEF35F0030A25
:10638000D8B4F2EF35F0010AD8B409EF36F0070AB5
:10639000D8B43CEF36F0010AD8B452EF36F0030A15
:1063A000D8B469EF36F0010AD8B480EF36F01F0A8E
:1063B000D8B4B3EF36F0010AD8B4C9EF36F0030A07
:1063C000D8B4E0EF36F0010AD8B4F7EF36F0070A98
:1063D000D8B41AEF37F0010AD8B42EEF37F0030A19
:1063E000D8B443EF37F0010AD8B458EF37F00F0AAA
:1063F000D8B479EF37F0010AD8B48DEF37F0030A3B
:10640000D8B4A2EF37F0010AD8B4B7EF37F0070AD3
:10641000D8B4D8EF37F0010AD8B4EDEF37F0030A5B
:10642000D8B401EF38F0010AD8B416EF38F07F0A7B
:10643000D8B42BEF38F0010AD8B44CEF38F0030A87
:10644000D8B461EF38F0010AD8B476EF38F0070A13
:10645000D8B48BEF38F0010AD8B4A1EF38F0030AB2
:10646000D8B4B7EF38F0010AD8B4D1EF38F00F0A3A
:10647000D8B425EF39F0010AD8B479EF39F01A0A07
:10648000D8B4CDEF39F0010AD8B4EEEF39F0030AF1
:10649000D8B40FEF3AF0010AD8B415EF3AF0040A75
:1064A000D8B436EF3AF0010AD8B457EF3AF0030AFD
:1064B000D8B46CEF3AF0010AD8B481EF3AF00F0A81
:1064C000D8B496EF3AF0010AD8B4ABEF3AF03D0AEF
:1064D000D8B4CCEF3AF0010AD8B4D5EF3AF0E2EFF5
:1064E0003AF00C0E0D019D6F9C6B0001DAEC1BF075
:1064F000E4EF3AF00C0E0D019D6F060E9C6F00014B
:10650000DAEC1BF0E4EF3AF00C01B16B020EB26F63
:106510000C0E0D019D6FAD0E9C6F0001DAEC1BF0AF
:10652000E4EF3AF00C01166B0C0E0D019D6F120E8C
:106530009C6F0001DAEC1BF0E4EF3AF00C0E0D0159
:106540009D6F9C6F0001DAEC1BF0E4EF3AF007015D
:1065500060510E0804E1870E0C01136F03D0810E09
:106560000C01136F0C0E0D019D6F120E9C6F00013C
:10657000DAEC1BF0E4EF3AF0070160510E0804E199
:10658000870E0C01196F03D0810E0C01196F0C0ED0
:106590000D019D6F180E9C6F0001DAEC1BF0E4EF0B
:1065A0003AF0070160510E0804E1870E0C011F6FDD
:1065B00003D0810E0C011F6F0C0E0D019D6F1E0E7E
:1065C0009C6F0001DAEC1BF0E4EF3AF00701605138
:1065D0000E0804E1870E0C01256F03D0810E0C011B
:1065E000256F0C0E0D019D6F240E9C6F0001DAECDF
:1065F0001BF0E4EF3AF0070160510E0804E1870E4A
:106600000C012B6F03D0810E0C012B6F0C0E0D01B2
:106610009D6F2A0E9C6F0001DAEC1BF0E4EF3AF05C
:10662000070160510E0804E1870E0C01316F03D0A1
:10663000810E0C01316F0C0E0D019D6F300E9C6FA1
:106640000001DAEC1BF0E4EF3AF0070160510E08AC
:1066500004E1870E0C01376F03D0810E0C01376FF8
:106660000C0E0D019D6F360E9C6F0001DAEC1BF0D5
:10667000E4EF3AF0070160510E0804E1870E0C01C7
:106680003D6F03D0810E0C013D6F0C0E0D019D6F0F
:106690003C0E9C6F0001DAEC1BF0E4EF3AF00701CE
:1066A00060510E0804E1870E0C01436F03D0810E88
:1066B0000C01436F0C0E0D019D6F420E9C6F00018B
:1066C000DAEC1BF0E4EF3AF0070160510E0804E148
:1066D000870E0C01496F03D0810E0C01496F0C0E1F
:1066E0000D019D6F480E9C6F0001DAEC1BF0E4EF8A
:1066F0003AF0070160510E0804E1870E0C014F6F5C
:1067000003D0810E0C014F6F0C0E0D019D6F4E0ECC
:106710009C6F0001DAEC1BF0E4EF3AF007016051E6
:106720000E0804E1870E0C01556F03D0810E0C0199
:10673000556F0C0E0D019D6F540E9C6F0001DAEC2D
:106740001BF0E4EF3AF0070160510E0804E1870EF8
:106750000C015C6F03D0810E0C015C6F0C0E0D01FF
:106760009D6F5B0E9C6F0001DAEC1BF0E4EF3AF0DA
:10677000070160510E0804E1870E0C01636F03D01E
:10678000810E0C01636F0C0E0D019D6F620E9C6FEC
:106790000001DAEC1BF0E4EF3AF0070160510E085B
:1067A00004E1870E0C016A6F03D0810E0C016A6F41
:1067B0000C0E0D019D6F690E9C6F0001DAEC1BF051
:1067C000E4EF3AF0070160510E0804E1870E0C0176
:1067D000716F03D0810E0C01716F0C0E0D019D6F56
:1067E000700E9C6F0001DAEC1BF0E4EF3AF0070149
:1067F00060510E0804E1870E0C019C6F03D0810EDE
:106800000C019C6F0C0E0D019D6F9B0E9C6F000187
:10681000DAEC1BF0E4EF3AF0070160510E0804E1F6
:10682000870E0C01786F03D0810E0C01786F0C0E6F
:106830000D019D6F770E9C6F0001DAEC1BF0E4EF09
:106840003AF0070160510E0804E1870E0C01846FD5
:1068500003D0810E0C01846F0C0E0D019D6F830E11
:106860009C6F0001DAEC1BF0E4EF3AF00701605195
:106870000E0804E1870E0C017E6F03D0810E0C011F
:106880007E6F0C0E0D019D6F7D0E9C6F0001DAEC8A
:106890001BF0E4EF3AF0070160510E0804E1870EA7
:1068A0000C018A6F03D0810E0C018A6F0C0E0D0152
:1068B0009D6F890E9C6F0001DAEC1BF0E4EF3AF05B
:1068C000070160510E0804E1870E0C01906F03D0A0
:1068D000810E0C01906F0C0E0D019D6F8F0E9C6F41
:1068E0000001DAEC1BF0E4EF3AF0070160510E080A
:1068F00004E1870E0C01966F03D0810E0C01966F98
:106900000C0E0D019D6F950E9C6F0001DAEC1BF0D3
:10691000E4EF3AF0070160510E0804E1870E0C0124
:10692000A26F03D0810E0C01A26F0C0E0D019D6FA2
:10693000A10E9C6F0001DAEC1BF0E4EF3AF00701C6
:1069400060510E0804E1870E0C01AE6F03D0810E7A
:106950000C01AE6F350EB16FB26B0C0E0D019D6F59
:10696000AD0E9C6F0001DAEC1BF0E4EF3AF007018A
:1069700060510E0804E1870E0C01AE6F03D0810E4A
:106980000C01AE6F350EB16F030EB26F0C0E0D0120
:106990009D6FAD0E9C6F0001DAEC1BF0E4EF3AF056
:1069A000070160510E0804E1870E0C01AE6F03D0A1
:1069B000810E0C01AE6F350EB16F050EB26F0C0E6D
:1069C0000D019D6FAD0E9C6F0001DAEC1BF0E4EF42
:1069D0003AF0070160510E0804E1870E0C01AE6F1A
:1069E00003D0810E0C01AE6F100EB16F050EB26FA9
:1069F0000C0E0D019D6FAD0E9C6F0001DAEC1BF0CB
:106A0000E4EF3AF0070160510E0804E1870E0C0133
:106A1000B56F03D0810E0C01B56FB96B0C0E0D0173
:106A20009D6FB40E9C6F0001DAEC1BF0E4EF3AF0BE
:106A3000030E0C01B96F070160510E0804E1870EC7
:106A40000C01B56F03D0810E0C01B56F0C0E0D015A
:106A50009D6FB40E9C6F0001DAEC1BF0E4EF3AF08E
:106A6000070160510E0804E1870E0C01B56F03D0D9
:106A7000810E0C01B56F0B0EB96F0C0E0D019D6FE1
:106A8000B40E9C6F0001DAEC1BF0E4EF3AF0070162
:106A900060510E0804E1870E0C01B56F03D0810E22
:106AA0000C01B56F0D0EB96F0C0E0D019D6FB40E7C
:106AB0009C6F0001DAEC1BF0E4EF3AF00701605143
:106AC0000E0804E1870E0C01BC6F03D0810E0C018F
:106AD000BC6FC06B0C0E0D019D6FBB0E9C6F000157
:106AE000DAEC1BF0E4EF3AF0070160510E0804E124
:106AF000870E0C01BC6F03D0810E0C01BC6F020E1F
:106B0000C06F0C0E0D019D6FBB0E9C6F0001DAEC87
:106B10001BF0E4EF3AF0070160510E0804E1870E24
:106B20000C01BC6F03D0810E0C01BC6F030EC06F53
:106B30000C0E0D019D6FBB0E9C6F0001DAEC1BF07B
:106B4000E4EF3AF0070160510E0804E1870E0C01F2
:106B5000C36F03D0810E0C01C36F07017139006E42
:106B60000F0E001600500F0B0C01C96F0701715179
:106B70000F0B0C01CA6F0C0E0D019D6FC20E9C6FA6
:106B80000001DAEC1BF0E4EF3AF0070160510E0867
:106B900004E1870E0C01CD6F03D0810E0C01CD6F87
:106BA000D16B0C0E0D019D6FCC0E9C6F0001DAECC9
:106BB0001BF0E4EF3AF0070160510E0804E1870E84
:106BC0000C01CD6F03D0810E0C01CD6F020ED16F81
:106BD0000C0E0D019D6FCC0E9C6F0001DAEC1BF0CA
:106BE000E4EF3AF0070160510E0804E1870E0C0152
:106BF000CD6F03D0810E0C01CD6F030ED16F0C0E43
:106C00000D019D6FCC0E9C6F0001DAEC1BF0E4EFE0
:106C10003AF0070160510E0804E1870E0C01D46FB1
:106C200003D0810E0C01D46F070167510F0B0C01CB
:106C3000D96F070167310D019D6F070166310D01A5
:106C40009C6F9D339C339D339C339D339C330F0E3F
:106C50009D179C510F0B0C01DA6F070166510F0B4A
:106C60000C01DB6F0C0E0D019D6FD30E9C6F0001AC
:106C7000DAEC1BF0E4EF3AF0070160510E0804E192
:106C8000870E0C01DE6F03D0810E0C01DE6FE26B0C
:106C90000C0E0D019D6FDD0E9C6F0001DAEC1BF0F8
:106CA000E4EF3AF0070160510E0804E1870E0C0191
:106CB000DE6F03D0810E0C01DE6F020EE26F0C0E50
:106CC0000D019D6FDD0E9C6F0001DAEC1BF0E4EF0F
:106CD0003AF0070160510E0804E1870E0C01DE6FE7
:106CE00003D0810E0C01DE6F030EE26F0C0E0D015E
:106CF0009D6FDD0E9C6F0001DAEC1BF0E4EF3AF0C3
:106D0000070160510E0804E1870E0C01E56F03D006
:106D1000810E0C01E56F070169510F0B0C01EA6F41
:106D2000070169310D019D6F070168310D019C6FED
:106D30009D339C339D339C339D339C330F0E9D17A5
:106D40009C510F0B0C01EB6F070168510F0B0C01ED
:106D5000EC6F0C0E0D019D6FE40E9C6F0001DAECE0
:106D60001BF0E4EF3AF0070160510E0804E1870ED2
:106D70000C01EF6F03D0810E0C01EF6FF36B0C0E63
:106D80000D019D6FEE0E9C6F0001DAEC1BF0E4EF3D
:106D90003AF0070160510E0804E1870E0C01EF6F15
:106DA00003D0810E0C01EF6F020EF36F0C0E0D017C
:106DB0009D6FEE0E9C6F0001DAEC1BF0E4EF3AF0F1
:106DC000070160510E0804E1870E0C01EF6F03D03C
:106DD000810E0C01EF6F030EF36F0C0E0D019D6F12
:106DE000EE0E9C6F0001DAEC1BF0E4EF3AF00701C5
:106DF00060510E0804E1870E0C01F66F03D0810E7E
:106E00000C01F66F07016B39006E0F0E0016005073
:106E10000F0B0C01FC6F07016B510F0B0C01FD6F89
:106E20000C0E0D019D6FF50E9C6F0001DAEC1BF04E
:106E3000E4EF3AF0070160510E0804E1870E0D01FE
:106E4000006F03D0810E0D01006F046B0C0E9D6F5F
:106E50009C690001DAEC1BF0E4EF3AF007016051A5
:106E60000E0804E1870E0D01006F03D0810E0D01A5
:106E7000006F020E046F0C0E9D6F9C690001DAEC2E
:106E80001BF0E4EF3AF0070160510E0804E1870EB1
:106E90000D01006F03D0810E0D01006F030E046F12
:106EA0000C0E9D6F9C690001DAEC1BF0E4EF3AF0E8
:106EB000070160510E0804E1870E0D01076F03D032
:106EC000810E0D01076F07016439006E0F0E001669
:106ED00000500F0B0D010D6F070164510F0B0D01D9
:106EE0000E6F0D0E9D6F060E9C6F0001DAEC1BF00D
:106EF0006BD3070160510E0804E1870E0D01116F7D
:106F000003D0810E0D01116F156B0D0E9D6F100ECC
:106F10009C6F0001DAEC1BF057D3070160510E089B
:106F200004E1870E0D01116F03D0810E0D01116F69
:106F3000020E156F0D0E9D6F100E9C6F0001DAECA6
:106F40001BF042D3070160510E0804E1870E0D01CA
:106F5000116F03D0810E0D01116F030E156F0D0E11
:106F60009D6F100E9C6F0001DAEC1BF02DD3070112
:106F700060510E0804E1870E0D01186F03D0810ED9
:106F80000D01186F07016539006E0F0E00160050D5
:106F90000F0B0D011E6F070165510F0B0D011F6FC8
:106FA0000D0E9D6F170E9C6F0001DAEC1BF00CD3D9
:106FB000070160510E0804E1870E0D01226F03D016
:106FC000810E0D01226F65C726FD0D0E9D6F210EEE
:106FD0009C6F0001DAEC1BF0F7D2070160510E083C
:106FE00004E1870E0D01296F03D0810E0D01296F79
:106FF0002D6B0D0E9D6F280E9C6F0001DAEC1BF0BF
:10700000E3D2070160510E0804E1870E0D01296FDC
:1070100003D0810E0D01296F020E2D6F0D0E9D6F95
:10702000280E9C6F0001DAEC1BF0CED207016051F4
:107030000E0804E1870E0D01296F03D0810E0D01AA
:10704000296F030E2D6F0D0E9D6F280E9C6F000192
:10705000DAEC1BF0B9D2070160510E0804E1870E8B
:107060000D01306F03D0810E0D01306F07016A39B9
:10707000006E0F0E001600500F0B0D01366F07014A
:107080006A510F0B0D01376F0D0E9D6F2F0E9C6F08
:107090000001DAEC1BF098D2070160510E0804E100
:1070A000870E0D013A6F03D0810E0D013A6F020E6B
:1070B000406F0D0E9D6F390E9C6F0001DAEC1BF0D6
:1070C00083D2070160510E0804E1870E0D013A6F6B
:1070D00003D0810E0D013A6F030E406F0D0E9D6FB0
:1070E000390E9C6F0001DAEC1BF06ED20701605183
:1070F0000E0804E1870E0D01436F03D0810E0D01D0
:10710000436F486B496B0D0E9D6F420E9C6F0001E3
:10711000DAEC1BF059D2070160510E0804E1870E2A
:107120000D01436F03D0810E0D01436F486B020EBA
:10713000496F0D0E9D6F420E9C6F0001DAEC1BF043
:1071400043D2070160510E0804E1870E0D01436F21
:1071500003D0810E0D01436F486B030E496F0D0E76
:107160009D6F420E9C6F0001DAEC1BF02DD20701DF
:1071700060510E0804E1870E0D01436F03D0810EAC
:107180000D01436F010E486F07016C510F0B0D018C
:10719000496F0D0E9D6F420E9C6F0001DAEC1BF0E3
:1071A00013D207016D5317E1020E0D01516F0D0E41
:1071B0009D6F4B0E9C6F0001DAEC1BF0010E070176
:1071C0006D6F030E0D019D6FE80E9C6F000118ECB2
:1071D0002EF041EC1FF0470E0D01586F07016E397C
:1071E000006E0F0E001600500F0B0D01596F0701B6
:1071F0006E510F0B0D015A6F0D0E9D6F530E9C6F4C
:107200000001DAEC1BF007016E510A081CE1705115
:107210000A0819E16F510A0816E1030E0D019D6F6E
:10722000E80E9C6F000118EC2EF041EC1FF0030EED
:107230000D01516F0D0E9D6F4B0E9C6F0001DAEC2E
:107240001BF007016D6B0001BFD107016D5317E102
:10725000020E0D01516F0D0E9D6F4B0E9C6F0001C4
:10726000DAEC1BF0010E07016D6F030E0D019D6F2F
:10727000E80E9C6F000118EC2EF041EC1FF0480E58
:107280000D01586F07017039006E0F0E0016005087
:107290000F0B0D01596F070170510F0B0D015A6F44
:1072A0000D0E9D6F530E9C6F0001DAEC1BF0070171
:1072B0006E510A081CE170510A0819E16F510A0861
:1072C00016E1030E0D019D6FE80E9C6F000118EC96
:1072D0002EF041EC1FF0030E0D01516F0D0E9D6F4E
:1072E0004B0E9C6F0001DAEC1BF007016D6B000187
:1072F0006BD107016D5317E1020E0D01516F0D0E99
:107300009D6F4B0E9C6F0001DAEC1BF0010E070124
:107310006D6F030E0D019D6FE80E9C6F000118EC60
:107320002EF041EC1FF0490E0D01586F07016F3927
:10733000006E0F0E001600500F0B0D01596F070164
:107340006F510F0B0D015A6F0D0E9D6F530E9C6FF9
:107350000001DAEC1BF007016E510A081CE17051C4
:107360000A0819E16F510A0816E1030E0D019D6F1D
:10737000E80E9C6F000118EC2EF041EC1FF0030E9C
:107380000D01516F0D0E9D6F4B0E9C6F0001DAECDD
:107390001BF007016D6B000117D1070160510E084A
:1073A00004E1870E0D01676F03D0810E0D01676F39
:1073B00007017439006E0F0E001600500F0B0D01FF
:1073C0006D6F070174510F0B0D016E6F0D0E9D6FE8
:1073D000660E9C6F0001DAEC1BF0F6D007016051DD
:1073E0000E0804E1870E0D01716F03D0810E0D01AF
:1073F000716F07017339006E0F0E001600500F0BEE
:107400000D01776F070173510F0B0D01786F0D0E92
:107410009D6F700E9C6F0001DAEC1BF0D5D0040E4E
:107420000D015F6F4D0E606F0001070160510E0886
:1074300004E1870E0D015D6F03D0810E0D015D6FBC
:1074400007017239006E0F0E001600500F0B0D0170
:10745000636F070172510F0B0D01646F0D0E9D6F6D
:107460005C0E9C6F0001DAEC1BF0AED0070160519E
:107470000E0804E1870E0D017B6F03D0810E0D0114
:107480007B6F07017539006E0F0E001600500F0B51
:107490000D01816F070175510F0B0D01826F0D0EEC
:1074A0009D6F7A0E9C6F0001DAEC1BF08DD0070106
:1074B00060510E0804E1870E0D01856F03D0810E27
:1074C0000D01856F020E896F0D0E9D6F840E9C6FEE
:1074D0000001DAEC1BF078D0070160510E0804E1DE
:1074E000870E0D01856F03D0810E0D01856F030E90
:1074F000896F0D0E9D6F840E9C6F0001DAEC1BF0FE
:1075000063D0070160510E0804E1870E0D018C6FF6
:1075100003D0810E0D018C6F020E906F0D0E9D6FCA
:107520008B0E9C6F0001DAEC1BF04ED0070160510E
:107530000E0804E1870E0D018C6F03D0810E0D0142
:107540008C6F030E906F0D0E9D6F8B0E9C6F000164
:10755000DAEC1BF039D0070160510E0804E1870E08
:107560000D01936F03D0810E0D01936F07017639E2
:10757000006E0F0E001600500F0B0D01996F0701E2
:1075800076510F0B0D019A6F0D0E9D6F920E9C6F31
:107590000001DAEC1BF018D00C0E0D019D6FA70E48
:1075A0009C6F0001DAEC1BF00FD0080E0C010F6F7E
:1075B0000E0E106F0C0E0D019D6F9C6F0001DAEC2A
:1075C0001BF002D021D000D00B01FF2D1ED0320EB7
:1075D0000D01B66F000117EC13F0070160510E08A2
:1075E00009E13A0E0D019D6F980E9C6F000118EC99
:1075F0002EF008D0070E0D019D6FD00E9C6F00017C
:1076000018EC2EF041EC1FF00B01000112000B01F1
:10761000B26BB16BC76BC86B070151A347D00001B8
:1076200041EC1FF0120E0B01CE6FCF6B00014FEC3F
:107630001FF00701636B626B0B0E0B01CF6FB30E74
:10764000CE6F130ED06F070ED26FD00ED16FD36BEB
:1076500000013DEC25F0012C23D0B8CBDEFB6DEC16
:1076600025F001C0C9FBB9CBDEFB6DEC25F001387C
:107670000B01CA6FF00ECA17BACBDEFB00016DEC2E
:1076800025F001500B01CA13C9CBB2FBCACBB1FB29
:10769000B2CB63F7B1CB62F7010E016E83D000016C
:1076A000FF0E016E0B017ED07BD0070151A527D0C4
:1076B000000141EC1FF0080E0B01DD6FDE6B0001D5
:1076C0007EEC27F00B0E0B01CA6FC70EC96F050EBB
:1076D000CB6F070ECD6FD00ECC6F0001C7EC2AF038
:1076E000012C07D0C7CB64F7010E016E0B015AD0F5
:1076F0000001FF0E016E0B0155D052D007010001B1
:1077000041EC1FF0080E0B01FE6FFF6B00017CECDB
:107710002EF00B0E0B01CA6FC70EC96F040ECB6F94
:10772000070ECD6FD00ECC6F0001C7EC2AF0012CF4
:1077300033D0070160510E0828E1C7CBC8FB000118
:1077400041EC1FF0080E0B01FE6FFF6B00017CEC9B
:107750002EF00B0E0B01CA6FC70EC96F040ECB6F54
:10776000070ECD6FD00ECC6F0001C7EC2AF0012CB4
:107770000AD00B01C751C85D05E1C7CB64F7010E04
:10778000016E10D0000108D00701C7CB64F7010ECD
:10779000016E0B0107D00001FF0E016E0B0102D03C
:1077A000FF0E016E000112000B01B26BB16BB36BE7
:1077B000B05303E0B051030803E2000E016E34D071
:1077C000B26B600EB16F200EB127000EB223010E16
:1077D000B05D200DF350036AB1270350B223B251BC
:1077E000036EB151B12BD8B4B22BB46F03C0B5FB4B
:1077F000F2CFB6FBF29EB5CBAAFFB4CBA9FFA69CF5
:10780000A69EA680A850B6BFF28EB36FB35309E010
:10781000070160510B01B35D04E1010E016E04D05C
:1078200003D0000E016E00D0000112000B01B46BFA
:10783000B36BB56BB25303E0B251030803E2000E21
:10784000016E5ED2B46B600EB36F200EB327000ED4
:10785000B423010EB25D200DF350036AB327035029
:10786000B423B451036EB351B32BD8B4B42BB86F57
:1078700003C0B9FBF2CFBAFBF29EB9CBAAFFB8CBDB
:10788000A9FFA69CA69EA680A850BABFF28EB56F8F
:10789000B553D8B432D2070160510B01B55DD8A4FD
:1078A0002CD2B5CB60F7B451036EB351B32BD8B41F
:1078B000B42BB86F03C0B9FBF2CFBAFBF29EB9CBC1
:1078C000AAFFB8CBA9FFA69CA69EA680A850BABFC7
:1078D000F28E0701616F0B01B451036EB351B32BEC
:1078E000D8B4B42BB86F03C0B9FBF2CFBAFBF29E89
:1078F000B9CBAAFFB8CBA9FFA69CA69EA680A8508C
:10790000BABFF28EB76FB451036EB351B32BD8B474
:10791000B42BB86F03C0B9FBF2CFBAFBF29EB9CB60
:10792000AAFFB8CBA9FFA69CA69EA680A850BABF66
:10793000F28EB66FB7CB63F7B6CB62F7B451036E76
:10794000B351B32BD8B4B42BB86F03C0B9FBF2CF8B
:10795000BAFBF29EB9CBAAFFB8CBA9FFA69CA69E04
:10796000A680A850BABFF28E0701646F0B01B45114
:10797000036EB351B32BD8B4B42BB86F03C0B9FBAB
:10798000F2CFBAFBF29EB9CBAAFFB8CBA9FFA69C57
:10799000A69EA680A850BABFF28E0701656F0B01A4
:1079A000B451036EB351B32BD8B4B42BB86F03C02A
:1079B000B9FBF2CFBAFBF29EB9CBAAFFB8CBA9FFB5
:1079C000A69CA69EA680A850BABFF28EB76FB451EF
:1079D000036EB351B32BD8B4B42BB86F03C0B9FB4B
:1079E000F2CFBAFBF29EB9CBAAFFB8CBA9FFA69CF7
:1079F000A69EA680A850BABFF28EB66FB7CB67F727
:107A0000B6CB66F7B451036EB351B32BD8B4B42BD5
:107A1000B86F03C0B9FBF2CFBAFBF29EB9CBAAFF95
:107A2000B8CBA9FFA69CA69EA680A850BABFF28E8E
:107A3000B76FB451036EB351B32BD8B4B42BB86F36
:107A400003C0B9FBF2CFBAFBF29EB9CBAAFFB8CB09
:107A5000A9FFA69CA69EA680A850BABFF28EB66FBC
:107A6000B7CB69F7B6CB68F7B451036EB351B32BFC
:107A7000D8B4B42BB86F03C0B9FBF2CFBAFBF29EF7
:107A8000B9CBAAFFB8CBA9FFA69CA69EA680A850FA
:107A9000BABFF28E07016A6F0B01B451036EB35186
:107AA000B32BD8B4B42BB86F03C0B9FBF2CFBAFB79
:107AB000F29EB9CBAAFFB8CBA9FFA69CA69EA68032
:107AC000A850BABFF28E07016B6F0B01B451036E61
:107AD000B351B32BD8B4B42BB86F03C0B9FBF2CFFA
:107AE000BAFBF29EB9CBAAFFB8CBA9FFA69CA69E73
:107AF000A680A850BABFF28E07016C6F0B01B4517B
:107B0000036EB351B32BD8B4B42BB86F03C0B9FB19
:107B1000F2CFBAFBF29EB9CBAAFFB8CBA9FFA69CC5
:107B2000A69EA680A850BABFF28E07016D6F0B010A
:107B3000B451036EB351B32BD8B4B42BB86F03C098
:107B4000B9FBF2CFBAFBF29EB9CBAAFFB8CBA9FF23
:107B5000A69CA69EA680A850BABFF28E07016E6FA3
:107B60000B01B451036EB351B32BD8B4B42BB86F1F
:107B700003C0B9FBF2CFBAFBF29EB9CBAAFFB8CBD8
:107B8000A9FFA69CA69EA680A850BABFF28E0701A8
:107B90006F6F0B01B451036EB351B32BD8B4B42B38
:107BA000B86F03C0B9FBF2CFBAFBF29EB9CBAAFF04
:107BB000B8CBA9FFA69CA69EA680A850BABFF28EFD
:107BC0000701706F0B01B451036EB351B32BD8B4DE
:107BD000B42BB86F03C0B9FBF2CFBAFBF29EB9CB9E
:107BE000AAFFB8CBA9FFA69CA69EA680A850BABFA4
:107BF000F28E0701716F0B01B451036EB351B32BB9
:107C0000D8B4B42BB86F03C0B9FBF2CFBAFBF29E65
:107C1000B9CBAAFFB8CBA9FFA69CA69EA680A85068
:107C2000BABFF28E0701726F0B01B451036EB351EC
:107C3000B32BD8B4B42BB86F03C0B9FBF2CFBAFBE7
:107C4000F29EB9CBAAFFB8CBA9FFA69CA69EA680A0
:107C5000A850BABFF28E0701736F0B01B451036EC7
:107C6000B351B32BD8B4B42BB86F03C0B9FBF2CF68
:107C7000BAFBF29EB9CBAAFFB8CBA9FFA69CA69EE1
:107C8000A680A850BABFF28E0701746F0B01B451E1
:107C9000036EB351B32BD8B4B42BB86F03C0B9FB88
:107CA000F2CFBAFBF29EB9CBAAFFB8CBA9FFA69C34
:107CB000A69EA680A850BABFF28E0701756F0B0171
:107CC000B451036EB351B32BD8B4B42BB86F03C007
:107CD000B9FBF2CFBAFBF29EB9CBAAFFB8CBA9FF92
:107CE000A69CA69EA680A850BABFF28E0701766F0A
:107CF000010E016E0B0104D003D0000E016E00D006
:107D00000001D7EF42F0070151AD0CD0200EA4A81E
:107D1000FED76D6E2D0EA4A8FED76D6E200EA4A802
:107D2000FED76D6EDECB1CFCDDCB1BFCDFCB1DFC60
:107D3000E0CB1EFC0001D1EC25F001521EE0030E49
:107D40000B01DD25E96E000EDE21EA6EEF50300AF0
:107D5000000107E0050A09E00C0A07E0080A09E04B
:107D600004D0010E016E0BD005D0FF0E016E07D0BE
:107D700001D000D00701D6D70001000E016E12001D
:107D80000B01E16BE16BDF51E15D0FE2036AE15151
:107D9000DD25E96EDE510320EA6EE051EF5C03E180
:107DA000E1CB01F004D0E12BEED7000E016E000113
:107DB00012000B01C96BC86BC76BC66BDC6B07018C
:107DC00051AD09D0340EF66E1E0EF76E000EF86E31
:107DD000000143EC1CF0000141EC1FF0600E0B01B0
:107DE000DD6FDE6B00017EEC27F00B0E0B01DE6F0A
:107DF000CA0EDD6F0D0EDF6F070EE16FD00EE06F64
:107E0000000181DF01C0DCFB0B01DC2D4FD00B0E2C
:107E1000DE6FCA0EDD6F0D0EDF6FEF0EE06F00013B
:107E2000AFDF0150090843E2CFCBDEFB6DEC25F05C
:107E300001500F0B0B01D86FD0CBDEFB00016DECB6
:107E400025F00138006EF00E00160050F00B0B010B
:107E5000DD6FD1CBDEFB00016DEC25F001500F0B87
:107E60000B01DD11D96FD2CBDEFB00016DEC25F0EB
:107E70000138006EF00E00160050F00B0B01DD6FA4
:107E8000D3CBDEFB00016DEC25F001500F0B0B0195
:107E9000DD11DA6FC96BD8CBC8FBD9CBC7FBDACB06
:107EA000C6FBC7AB03D0000E016E04D00001010E6B
:107EB000016E0B01000112000B01E36BE46BE66B3A
:107EC000E56BCECBE9FFCFCBEAFFEC6AED52EF6A70
:107ED00030BA49D0E6CBB8FDE5CBB7FD0D01BA6BA2
:107EE000320EB96F000158EC1CF002C0EAFB01C071
:107EF000E9FB0B01D251025C2BE303E1D151E95DB7
:107F000027E3070151AD21D0600EF66E1B0EF76E10
:107F1000000EF86E110E0D01B66F000169EC1CF039
:107F2000100EE96ED2CBB7FDD1CBB6FD82EC1CF0C2
:107F3000740EF66E1B0EF76E000EF86E070E0D0136
:107F4000B66F000169EC1CF00701000E016EC6D08F
:107F5000320E0D01B66F000117EC13F00B01E52B8B
:107F6000D8B4E62BB5D70B0EEA6ED30EE96E006AD5
:107F7000026A100E016E0001AAEC1BF0320E0D0118
:107F8000B66F000117EC13F0070151AD0AD07C0E5B
:107F9000F66E1B0EF76E000EF86E000143EC1CF03F
:107FA000070130AA40D00B01E3510F08D8B002D02E
:107FB000070139D00001FAEC1CF001C0E4FB070115
:107FC00051AD0ED0E4CBB7FD570E0D01B86F0001D7
:107FD000B7EC1BF0200EA4A8FED76D6E07D00701EA
:107FE000010E0D01B66F000117EC13F00B01E45107
:107FF000900803E0E451F00804E1E36BE4CBD3FB29
:108000000AD0E32B036AE351D30FE96E0B0E032072
:10801000EA6EE4CBEFFF0A0E0D01B66F000117EC1C
:1080200013F00701BED7020E0B01D025E35D11E26C
:10803000070151AD0AD0880EF66E1B0EF76E000ECA
:10804000F86E000143EC1CF00701000E016E46D0F3
:108050000B01036AD051D30FE96E0B0E0320EA6EB9
:10806000EFCFE7FBE73BF00EE717010ED025036AE1
:10807000D30FE96E0B0E0320EA6EEF500F0BE713E0
:10808000020ED025036AD30FE96E0B0E0320EA6EB1
:10809000EFCFE8FBE83BF00EE817030ED025036AAC
:1080A000D30FE96E0B0E0320EA6EEF500F0BE813AF
:1080B000CECBE9FFCFCBEAFFE7CBECFFED52E8CB2D
:1080C000EFFF070151AD08D00A0EA4A8FED76D6ED0
:1080D0000D0EA4A8FED76D6E010E016E00011200F8
:1080E0000B01CD6BCC6B000141EC1FF0070151A3DC
:1080F00033D0050E0B01CE6FCF6B00014FEC1FF09C
:108100000701676B1E0E666F0B0E0B01CF6FB80E6B
:10811000CE6F130ED06F070ED26FD00ED16FD36B10
:1081200000013DEC25F0012C15D0BDCBDEFB6DEC44
:1081300025F001380B01CE6FF00ECE17BECBDEFB63
:1081400000016DEC25F00B01CE5101100701666FA7
:10815000676B000151D0070151A502D04CD04BD024
:10816000050E0B01FE6FFF6B00017CEC2EF00B0E79
:108170000B01CF6FCC0ECE6F020ED06F070ED26FF9
:10818000D00ED16F000198DE012C36D0070160516E
:108190000E082DE10B01CC510701665D06E10B01D4
:1081A000CD510701675D01E126D0640E0D01B66F68
:1081B000000117EC13F0050E0B01FE6FFF6B0001C1
:1081C0007CEC2EF00B0E0B01CF6FCC0ECE6F020E9F
:1081D000D06F070ED26FD00ED16F00016DDE012C73
:1081E00004D0CDCB67F7CCCB66F706D00701CDCB5B
:1081F00067F7CCCB66F7000112000900F6CFB9FB98
:10820000F7CFBAFBF8CFBBFBF5509EA8FED7AD6EFB
:10821000B9CBF6FFBACBF7FFBBCBF8FF0B01B82FFA
:1082200001D002D00001E9D7000112000B01B9BF53
:1082300010D00F0E006EB83900160A0E005C03E273
:10824000300E002602D0B951002600509EA8FED75D
:10825000AD6E0F0EB8170A0EB85D02E2300E02D0F6
:10826000B99FB951B827B8519EA8FED7AD6E00018D
:1082700012000B01B36BB26BB56BB46BB66BB791FD
:1082800067C7B5FB66C7B4FBB7B176D0B451B25D72
:1082900004E1B551B35DD8B46CD0000121DF67C7EC
:1082A000B3FB66C7B2FB0B01B451B25D03E1B5513C
:1082B000B35D54E0B5CB67F7B4CB66F72B0EFE6F1A
:1082C000010EFF6F00017CEC2EF0070151AD3ED096
:1082D000B60EF66E1C0EF76E000EF86E200E0B0139
:1082E000B86F00018ADFB5CBB8FB570E0B01B96F31
:1082F00000019CDFB4CBB8FB570E0B01B96F000136
:1083000095DFD90EF66E1C0EF76E000EF86E070E96
:108310000B01B86F000171DFB3CBB8FB570E0B0137
:10832000B96F000183DFB2CBB8FB570E0B01B96FF9
:1083300000017CDF290E9EA8FED7AD6E0A0E9EA816
:10834000FED7AD6E0D0E9EA8FED7AD6E640E0D016C
:10835000B66F000117EC13F00AD00B01B62BB65123
:10836000010802E2B78102D0B36BB26B000102D008
:108370000B01B7810B0188D7000112000B01CD6BF7
:10838000CC6B000141EC1FF0070151A333D0060E66
:108390000B01CE6FCF6B00014FEC1FF00701696B33
:1083A0001E0E686F0B0E0B01CF6FB80ECE6F130E43
:1083B000D06F070ED26FD00ED16FD36B00013DECA2
:1083C00025F0012C15D0BDCBDEFB6DEC25F001387E
:1083D0000B01CE6FF00ECE17BECBDEFB00016DECB5
:1083E00025F00B01CE5101100701686F696B000188
:1083F00051D0070151A502D04CD04BD0060E0B0135
:10840000FE6FFF6B00017CEC2EF00B0E0B01CF6FAB
:10841000CC0ECE6F020ED06F070ED26FD00ED16F82
:1084200000014ADD012C36D0070160510E082DE114
:108430000B01CC510701685D06E10B01CD5107012D
:10844000695D01E126D0640E0D01B66F000117ECE5
:1084500013F0060E0B01FE6FFF6B00017CEC2EF09B
:108460000B0E0B01CF6FCC0ECE6F020ED06F070E2E
:10847000D26FD00ED16F00011FDD012C04D0CDCB07
:1084800069F7CCCB68F706D00701CDCB69F7CCCB29
:1084900068F7000112000B01B36BB26BB56BB46BE4
:1084A000B66BB79169C7B5FB68C7B4FBB7B176D0F7
:1084B000B451B25D04E1B551B35DD8B46CD00001E4
:1084C0005DDF69C7B3FB68C7B2FB0B01B451B25D96
:1084D00003E1B551B35D54E0B5CB69F7B4CB68F7B0
:1084E0002F0EFE6F010EFF6F00017CEC2EF00701D6
:1084F00051AD3ED0E80EF66E1C0EF76E000EF86E13
:10850000210E0B01B86F000178DEB5CBB8FB570E1A
:108510000B01B96F00018ADEB4CBB8FB570E0B011B
:10852000B96F000183DE0C0EF66E1D0EF76E000EA5
:10853000F86E070E0B01B86F00015FDEB3CBB8FB1E
:10854000570E0B01B96F000171DEB2CBB8FB570EAD
:108550000B01B96F00016ADE290E9EA8FED7AD6E31
:108560000A0E9EA8FED7AD6E0D0E9EA8FED7AD6E6C
:10857000640E0D01B66F000117EC13F00AD00B0169
:10858000B62BB651010802E2B78102D0B36BB26BD1
:10859000000102D00B01B7810B0188D70001120046
:1085A0000B01B16BB0CBB2FB000116EF3CF0012C1C
:1085B000D7D2070161B5ECD04F8051A31AD0210E5C
:1085C0000B01CE6F010ECF6F00014FEC1FF0130EA9
:1085D0000B01CE6F010ECF6F00014FEC1FF03B0E71
:1085E0000B01CE6F010ECF6F00014FEC1FF0CCD00E
:1085F000070151A5A0D0210E0B01DD6F010EDE6F2A
:1086000000017EEC27F0640E0D01B66F000117EC3F
:1086100013F007016D5309E1420E0B01DD6F010EEE
:10862000DE6F00017EEC27F008D0410E0B01DD6FFC
:10863000010EDE6F00017EEC27F0470E0B01DD6FAF
:10864000010EDE6F00017EEC27F0490E0B01DD6F9D
:10865000010EDE6F00017EEC27F0370E0B01DD6F9F
:10866000010EDE6F00017EEC27F03B0E0B01DD6F8B
:10867000010EDE6F00017EEC27F02B0E0B01DD6F8B
:10868000010EDE6F00017EEC27F02F0E0B01DD6F77
:10869000010EDE6F00017EEC27F0500E0B01DD6F46
:1086A000010EDE6F00017EEC27F0400E0B01DD6F46
:1086B000010EDE6F00017EEC27F0540E0B01DD6F22
:1086C000010EDE6F00017EEC27F0530E0B01DD6F13
:1086D000010EDE6F00017EEC27F0330E0B01DD6F23
:1086E000010EDE6F00017EEC27F0520E0B01DD6FF4
:1086F000010EDE6F00017EEC27F0270E0B01DD6F0F
:10870000010EDE6F00017EEC27F0660E0B01DD6FBF
:10871000010EDE6F00017EEC27F0D9EC3EF001C0C7
:10872000B1FB0B01B15304E14FB201D04F8201D034
:108730004F922CD00701210E0B01FE6F010EFF6F2F
:1087400000017CEC2EF0370E0B01FE6F010EFF6F67
:1087500000017CEC2EF03B0E0B01FE6F010EFF6F53
:1087600000017CEC2EF0070160510E080EE152531F
:108770000CE15351030809E1590E0B01FE6F010E84
:10878000FF6F00017CEC2EF007010B0172D0070196
:108790004F9051A30AD0200E0B01CE6F010ECF6F68
:1087A00000014FEC1FF065D0070151A55AD04F9240
:1087B00061B718D0200E0B01DD6F010EDE6F0001D6
:1087C0007EEC27F0640E0D01B66F000117EC13F07C
:1087D000370E0B01DD6F010EDE6F00017EEC27F01E
:1087E0001AD007014E6B670E0B01DD6FDE6B0001C7
:1087F0007EEC27F0030E0C010C6FE80E0B6F0001EE
:108800003EEC27F001C0B1FB0B01B12D01D003D02C
:10881000070161970B0107016D5309E1420E0B013E
:10882000DD6F010EDE6F00017EEC27F008D0410EF7
:108830000B01DD6F010EDE6F00017EEC27F0470EAD
:108840000B01DD6F010EDE6F00017EEC27F0660E7E
:108850000B01DD6F010EDE6F00017EEC27F009D009
:108860000701200E0B01FE6F010EFF6F00017CEC73
:108870002EF00701605109081AE1330E0B01FE6F5B
:10888000010EFF6F00017CEC2EF0400E0B01FE6F1D
:10889000010EFF6F00017CEC2EF0270E0B01FE6F26
:1088A000010EFF6F00017CEC2EF03FD007016051FC
:1088B000070803E060510F0822E1470E0B01FE6F2D
:1088C000010EFF6F00017CEC2EF0480E0B01FE6FD5
:1088D000010EFF6F00017CEC2EF0490E0B01FE6FC4
:1088E000010EFF6F00017CEC2EF0270E0B01FE6FD6
:1088F000010EFF6F00017CEC2EF017D0070151A391
:108900000AD0270E0B01CE6F010ECF6F00014FEC86
:108910001FF00BD0070151B509D0270E0B01FE6FD8
:10892000010EFF6F00017CEC2EF0070151B58CD0D9
:1089300061B14ED04F844F8251A31AD01E0E0B014D
:10894000CE6F010ECF6F00014FEC1FF02B0E0B010D
:10895000CE6F010ECF6F00014FEC1FF02F0E0B01F9
:10896000CE6F010ECF6F00014FEC1FF02FD007012B
:108970001E0E0B01FE6F010EFF6F00017CEC2EF04E
:108980002B0E0B01FE6F010EFF6F00017CEC2EF031
:10899000070160510E0807E1525305E153510308E6
:1089A00002E1000166DC2F0E0B01FE6F010EFF6F6E
:1089B00000017CEC2EF0070160510E0808E15253D3
:1089C00006E15351030803E1000165DD07013CD0D6
:1089D0004F944F8251A321D0676B1E0E666F2B0EF2
:1089E0000B01CE6F010ECF6F00014FEC1FF007019E
:1089F000696B1E0E686F2F0E0B01CE6F010ECF6FCD
:108A000000014FEC1FF01C0E0B01CE6F010ECF6F5B
:108A100000014FEC1FF00BD0070151B509D01C0E1F
:108A20000B01FE6F010EFF6F00017CEC2EF00701C1
:108A30006051090809E1460E0B01FE6F010EFF6F40
:108A400000017CEC2EF0070160510D081AE1500E78
:108A50000B01CE6F010ECF6F00014FEC1FF0520ED5
:108A60000B01CE6F010ECF6F00014FEC1FF0530EC4
:108A70000B01CE6F010ECF6F00014FEC1FF062D0E3
:108A8000070160510E085EE1525303E153510308A0
:108A90000AE0500E0B01FE6F010EFF6F00017CEC2F
:108AA0002EF009D00701510E0B01FE6F010EFF6F72
:108AB00000017CEC2EF0520E0B01FE6F010EFF6FD9
:108AC00000017CEC2EF0530E0B01FE6F010EFF6FC8
:108AD00000017CEC2EF00701525303E153510308CF
:108AE0000AE0540E0B01FE6F010EFF6F00017CECDB
:108AF0002EF028D007016D5309E1560E0B01FE6FD1
:108B0000010EFF6F00017CEC2EF008D0550E0B011A
:108B1000FE6F010EFF6F00017CEC2EF007016E531B
:108B200009E1580E0B01FE6F010EFF6F00017CEC96
:108B30002EF008D0570E0B01FE6F010EFF6F0001E3
:108B40007CEC2EF0400E0B01C66F0C0EC76F4FC0B1
:108B5000C8FB0001C0EC11F0010E016E04D003D07F
:108B6000000E016E00D012000B01C56B070151A36E
:108B700031D0040E0B01CE6FCF6B00014FEC1FF014
:108B8000800E0701716F0B0E0B01CF6FB10ECE6F10
:108B9000130ED06F070ED26FD00ED16FD36B0001C2
:108BA0003DEC25F0012C14D0B9CBDEFB6DEC25F0AB
:108BB00001380B01C66FF00EC617BACBDEFB000101
:108BC0006DEC25F00B01C65101100701716F00011A
:108BD00021D0070151A502D01ED01DD0000141ECCB
:108BE0001FF0040E0B01FE6FFF6B00017CEC2EF0FA
:108BF0000B0E0B01CA6FC50EC96F040ECB6F070EAB
:108C0000CD6FD00ECC6F0001C7EC2AF0012C02D042
:108C1000C5CB71F7070100011200070151AD0CD05F
:108C2000200EA4A8FED76D6E2D0EA4A8FED76D6EE3
:108C3000200EA4A8FED76D6EFFCBADFDFECBACFD24
:108C400000CCAEFD02CCB0FD01CCAFFD000168EC64
:108C50002CF0015228E0010E0B01FE25E96E000EFA
:108C6000FF21EA6EEF50500A000111E0300A13E0D4
:108C7000010A11E0030A0FE05A0A11E0790A0FE035
:108C8000030A0DE0130A0BE0030A09E009D0010E04
:108C9000016E0BD005D0FF0E016E07D001D000D0C1
:108CA0000701CAD70001000E016E12000B01BB6B59
:108CB000000141EC1FF0070151A340D0020E0B014F
:108CC000CE6FCF6B00014FEC1FF00B0E0B01CF6F7F
:108CD000B10ECE6F130ED06F070ED26FD00ED16FC4
:108CE000D36B00013DEC25F0012C26D0B6CBDEFB8A
:108CF0006DEC25F001C0BBFB0B01BB51FC0F0CE27E
:108D0000040F0001F9EF46F0070161810B0104D067
:108D1000070161910B0100D0070161A102D04F94BE
:108D200001D04F84400E0B01C66F0C0EC76F4FC0B1
:108D3000C8FB0001C0EC11F059D0070151A502D0C9
:108D400056D055D0020E0B01FE6FFF6B00017CEC7C
:108D50002EF0140E0D01B66F000117EC13F00B0E80
:108D60000B01FF6FB10EFE6F0A0E0C01006F070EB4
:108D7000026FD00E016F000150DF012C37D00B01C4
:108D8000B43D1ED0B351000A000109E0010A0BE016
:108D9000030A09E0010A0AE0060A0CE00FD0070105
:108DA000618161930DD0070161930AD00701619140
:108DB000618306D007016191619302D0070100D061
:108DC000070161A103D04F944F8206D04F8461A365
:108DD00002D04F9201D04F82400E0B01C66F0C0E95
:108DE000C76F4FC0C8FB0001C0EC11F007010001C4
:108DF0001200E824F76AF736130FF66E8E0EF7228C
:108E0000000EF86EFB6E0A00F550FA6E0800F55081
:108E1000F96E088D108D108D108D0B01C56B000142
:108E200041EC1FF0070151A331D0140E0B01CE6F9E
:108E3000CF6B00014FEC1FF01E0E0701726F0B0E7F
:108E40000B01CF6FB10ECE6F130ED06F070ED26F26
:108E5000D00ED16FD36B00013DEC25F0012C14D066
:108E6000B6CBDEFB6DEC25F001380B01C66FF00EC2
:108E7000C617B7CBDEFB00016DEC25F00B01C65128
:108E800001100701726F000190D0070151A502D0B7
:108E90008BD08AD060510E0843E1525341E15351C7
:108EA00003083EE1150E0B01FE6FFF6B00017CEC29
:108EB0002EF00B0E0B01CA6FC50EC96F040ECB6FDF
:108EC000070ECD6FD00ECC6F0001C7EC2AF0012C3D
:108ED00025D00B01C5510701725D01E165D0640E1B
:108EE0000D01B66F000117EC13F0150E0B01FE6FAC
:108EF000FF6B00017CEC2EF00B0E0B01CA6FC50E50
:108F0000C96F040ECB6F070ECD6FD00ECC6F000172
:108F1000C7EC2AF0012C02D0C5CB72F746D007016E
:108F2000140E0B01FE6FFF6B00017CEC2EF00B0E9C
:108F30000B01CA6FC50EC96F040ECB6F070ECD6F44
:108F4000D00ECC6F0001C7EC2AF0012C2ED0070107
:108F500060510E0827E10B01C5510701725D01E167
:108F600023D0640E0D01B66F000117EC13F0140E40
:108F70000B01FE6FFF6B00017CEC2EF00B0E0B0162
:108F8000CA6FC50EC96F040ECB6F070ECD6FD00E22
:108F9000CC6F0001C7EC2AF0012C02D0C5CB72F7D0
:108FA00004D00701C5CB72F7000112000B01C56B9D
:108FB000000141EC1FF0070151B347D0160E0B0121
:108FC000FE6FFF6B00017CEC2EF00B0E0B01CA6FE5
:108FD000C50EC96F040ECB6F070ECD6FD00ECC6FD0
:108FE0000001C7EC2AF0012C2ED0070160510E08B9
:108FF00027E10B01C5510701735D01E154D0640EF7
:109000000D01B66F000117EC13F0160E0B01FE6F89
:10901000FF6B00017CEC2EF00B0E0B01CA6FC50E2E
:10902000C96F040ECB6F070ECD6FD00ECC6F000151
:10903000C7EC2AF0012C02D0C5CB73F704D007018E
:10904000C5CB73F7000130D00701160E0B01CE6FB0
:10905000CF6B00014FEC1FF0030E0701736F0B0E77
:109060000B01CF6FB10ECE6F130ED06F070ED26F04
:10907000D00ED16FD36B00013DEC25F0012C14D044
:10908000B6CBDEFB6DEC25F001380B01C66FF00EA0
:10909000C617B7CBDEFB00016DEC25F00B01C65106
:1090A00001100701736F000112000B01C56B000175
:1090B00041EC1FF0070151B347D0170E0B01FE6FB3
:1090C000FF6B00017CEC2EF00B0E0B01CA6FC50E7E
:1090D000C96F040ECB6F070ECD6FD00ECC6F0001A1
:1090E000C7EC2AF0012C2ED0070160510E0827E1B1
:1090F0000B01C5510701745D01E154D0640E0D01EF
:10910000B66F000117EC13F0170E0B01FE6FFF6B2B
:1091100000017CEC2EF00B0E0B01CA6FC50EC96F5F
:10912000040ECB6F070ECD6FD00ECC6F0001C7ECD5
:109130002AF0012C02D0C5CB74F704D00701C5CBAF
:1091400074F7000130D00701170E0B01CE6FCF6B03
:1091500000014FEC1FF0020E0701746F0B0E0B01A4
:10916000CF6FB10ECE6F130ED06F070ED26FD00E31
:10917000D16FD36B00013DEC25F0012C14D0B9CB9D
:10918000DEFB6DEC25F001380B01C66FF00EC61743
:10919000BACBDEFB00016DEC25F00B01C6510110CE
:1091A0000701746F000112000B01C56B000141EC57
:1091B0001FF0070151A33DD0030E0B01CE6FCF6B03
:1091C00000014FEC1FF00B0E0B01CF6FB10ECE6FF5
:1091D000130ED06F070ED26FD00ED16FD36B00017C
:1091E0003DEC25F0012C23D0B6CBDEFB6DEC25F059
:1091F00001C0C5FB0B01C551010A000103E0010AD2
:1092000004E003D00701618503D00701619500D018
:1092100061A502D04F9001D04F80400E0B01C66F68
:109220000C0EC76F4FC0C8FB0001C0EC11F04FD14E
:10923000070151A500D14FB052D0618561B718D058
:10924000200E0B01DD6F010EDE6F00017EEC27F0BA
:10925000640E0D01B66F000117EC13F0370E0B0111
:10926000DD6F010EDE6F00017EEC27F01AD00701E2
:109270004E6B670E0B01DD6FDE6B00017EEC27F09D
:10928000030E0C010C6FE80E0B6F00013EEC27F093
:1092900001C0C5FB0B01C52D01D003D007016197AB
:1092A0000B0107016D5309E1420E0B01DD6F010E49
:1092B000DE6F00017EEC27F008D0410E0B01DD6F60
:1092C000010EDE6F00017EEC27F0470E0B01DD6F13
:1092D000010EDE6F00017EEC27F08CD00701619556
:1092E000210E0B01DD6F010EDE6F00017EEC27F019
:1092F000640E0D01B66F000117EC13F007016D53FA
:1093000009E1420E0B01DD6F010EDE6F00017EEC04
:1093100027F008D0410E0B01DD6F010EDE6F00015A
:109320007EEC27F0470E0B01DD6F010EDE6F0001B2
:109330007EEC27F0490E0B01DD6F010EDE6F0001A0
:109340007EEC27F0370E0B01DD6F010EDE6F0001A2
:109350007EEC27F03B0E0B01DD6F010EDE6F00018E
:109360007EEC27F02B0E0B01DD6F010EDE6F00018E
:109370007EEC27F02F0E0B01DD6F010EDE6F00017A
:109380007EEC27F0500E0B01DD6F010EDE6F000149
:109390007EEC27F0400E0B01DD6F010EDE6F000149
:1093A0007EEC27F0540E0B01DD6F010EDE6F000125
:1093B0007EEC27F0530E0B01DD6F010EDE6F000116
:1093C0007EEC27F0330E0B01DD6F010EDE6F000126
:1093D0007EEC27F0520E0B01DD6F010EDE6F0001F7
:1093E0007EEC27F0270E0B01DD6F010EDE6F000112
:1093F0007EEC27F0070161A503D04F904F920ED06D
:109400004F800001D9EC3EF001C0C5FB0B01C553F4
:1094100004E14FB201D04F8201D04F92400E0B01B8
:10942000C66F0C0EC76F4FC0C8FB0001C0EC11F037
:109430004ED04DD00701030E0B01FE6FFF6B0001F4
:109440007CEC2EF0140E0D01B66F000117EC13F03A
:109450000B0E0B01FF6FB10EFE6F0A0E0C01006FB9
:10946000070E026FD00E016F00010DEC46F0012CCB
:109470002ED00B01B43D1BD0B351000A000109E00E
:10948000030A0AE0090A0BE0010A0BE0050A0BE0F7
:109490000CD0070161850BD00701619508D0070149
:1094A00006D0070104D0070102D0070100D0070150
:1094B00061A502D04F9001D04F80400E0B01C66FC6
:1094C0000C0EC76F4FC0C8FB0001C0EC11F01200BA
:1094D0000B01C56B000141EC1FF0070151A330D017
:1094E0000A0E0B01CE6FCF6B00014FEC1FF007018E
:1094F000656B0B0E0B01CF6FB10ECE6F130ED06FDD
:10950000070ED26FD00ED16FD36B00013DEC25F06A
:10951000012C14D0B6CBDEFB6DEC25F001380B012D
:10952000C66FF00EC617B7CBDEFB00016DEC25F061
:109530000B01C65101100701656F00014AD00701F8
:1095400051A502D045D044D00A0E0B01FE6FFF6B2F
:1095500000017CEC2EF00B0E0B01CA6FC50EC96F1B
:10956000040ECB6F070ECD6FD00ECC6F0001C7EC91
:109570002AF0012C2ED0070160510E0827E10B01C3
:10958000C5510701655D01E123D0640E0D01B66F81
:10959000000117EC13F00A0E0B01FE6FFF6B0001C8
:1095A0007CEC2EF00B0E0B01CA6FC50EC96F040EBA
:1095B000CB6F070ECD6FD00ECC6F0001C7EC2AF039
:1095C000012C02D0C5CB65F704D00701C5CB65F7E8
:1095D000000112000B01AD6BAE6BAF919D920B0EB3
:1095E000EA6E9B0EE96E006A026A120E016E0001BD
:1095F000AAEC1BF00B0EEA6E9B0EE96E000E90ECCF
:1096000006F00A000900F550EE6E0009FBE10B0EB2
:109610000B01D86F9B0ED76F0001F7EC14F0070118
:10962000606B080E0B01B06FFA0E0D01B66F0001F2
:1096300017EC13F00B01B02FF7D74C0ECE6FCF6B9A
:1096400000014FEC1FF03A0E0C01D36F980ED26F51
:10965000010ED46F000118EC1FF001C0ADFB0B012F
:10966000AD2D9BD04E0ECE6F010ECF6F00014FEC93
:109670001FF05B0E0B01CE6F010ECF6F00014FECA0
:109680001FF00D0E0701606F51AD0AD0800EF66E0F
:10969000180EF76E000EF86E000143EC1CF0070187
:1096A0000B0EEA6E9B0EE96E000E0001A3EC06F0B5
:1096B0000A000900F550EE6E0009FBE10B0E0B01EC
:1096C000D86F9B0ED76F0001F7EC14F0070151AF74
:1096D00019D0320E0D01B66F000117EC13F0070E12
:1096E0000B01B16F540EB06F070EB36F560EB26F11
:1096F000070EB56F580EB46F0001BCEC24F09D82CC
:1097000062D00701000107EC3BF0012C01D007D02B
:10971000640E0D01B66F000117EC13F0F4D7010EC3
:109720000B01B06F0001D4EC3BF0012C15D0010E01
:109730000B01B06F0001D0EC42F04F984F86400E05
:109740000B01C66F0C0EC76F4FC0C8FB0001C0EC09
:1097500011F030800B01AF810B01AFB11ED00701BA
:1097600051AD09D08E0EF66E180EF76E000EF86E23
:10977000000143EC1CF00001B4EC45F070EC40F04B
:10978000BEEC41F056EC46F00DEC47F00FDC8DDC02
:109790000BDD07EC3BF09CDE0B01966884CF35F0C7
:1097A000976885CF36F0AE6BAE5107080AE3036ABF
:1097B000AE513F0FE96E000E0320EA6EEF6AAE2B4A
:1097C000F3D79D8200011200EF5210E0EACFD8FBE0
:1097D000E9CFD7FBEF50A4A8FED76D6ED8CBEAFF38
:1097E000D7CBE9FFE92AD8B4EA2AEED771EF4DF0DA
:1097F0000B01D56BD66B0B0EEA6EB00EE96E006AEC
:10980000026A110E016E0001AAEC1BF00B0EEA6E4B
:10981000C10EE96E006A026A140E016EAAEC1BF01A
:1098200007012F6B2E6B010E0B01DD6FDE6B00014C
:109830007EEC27F0070151AD09D01A0EF66E1D0E11
:10984000F76E000EF86E000143EC1CF00B0E0C01DD
:109850001C6FC10E1B6F130E1D6FE80E1E6F0001F3
:10986000D1EC25F001C0D5FB0B01D551FF0826E155
:10987000070151AD0AD02A0EF66E1D0EF76E000ECE
:10988000F86E000143EC1CF00701606B0B0EEA6EF2
:10989000B00EE96E000E00010CEC08F00A000900A1
:1098A000F550EE6E0009FBE10B0E0B01D86FB00E08
:1098B000D76F0001F7EC14F09CD10B01C4513908AB
:1098C000D8A488D04C0EDD6FDE6B00017EEC27F053
:1098D0000B0E0C011C6FC10E1B6F130E1D6FE80EDB
:1098E0001E6F0001D1EC25F001C0D5FB0B01D55155
:1098F000FF0826E1070151AD0AD03C0EF66E1D0EA1
:10990000F76E000EF86E000143EC1CF00701606B6F
:109910000B0EEA6EB00EE96E000E00010CEC08F0C2
:109920000A000900F550EE6E0009FBE10B0E0B0179
:10993000D86FB00ED76F0001F7EC14F05AD10B01BD
:10994000010EDD6FDE6B00017EEC27F0070151ADEB
:1099500009D04E0EF66E1D0EF76E000EF86E000169
:1099600043EC1CF00B0E0C011C6FC10E1B6F130E91
:109970001D6FE80E1E6F0001D1EC25F001C0D5FB74
:109980000B01D551FF0826E1070151AD0AD0620E47
:10999000F66E1D0EF76E000EF86E000143EC1CF023
:1099A0000701606B0B0EEA6EB00EE96E000E00014F
:1099B0000CEC08F00A000900F550EE6E0009FBE11E
:1099C0000B0E0B01D86FB00ED76F0001F7EC14F03F
:1099D00010D10B01C45133083EE1010EDD6FDE6B87
:1099E00000017EEC27F00B0E0C011C6FC10E1B6FEB
:1099F000130E1D6FE80E1E6F0001D1EC25F001C0A3
:109A0000D5FB0B01D551FF0826E1070151AD0AD066
:109A1000740EF66E1D0EF76E000EF86E000143EC2C
:109A20001CF00701606B0B0EEA6EB00EE96E000EC3
:109A300000010CEC08F00A000900F550EE6E000978
:109A4000FBE10B0E0B01D86FB00ED76F0001F7ECE6
:109A500014F0CFD00B01C4513008D8A4A6D0C65101
:109A60004208D8A47BD0C7515508D8A477D0020E9D
:109A700007012F6F420E2E6F0B01D66BD6510508D2
:109A80001AE3036AD651590F016E070E032203C071
:109A9000D8FB050ED625036AC10FE96E0B0E032015
:109AA000EA6EEFCFD9FBD8CBEAFF01C0E9FFD9CBF3
:109AB000EFFFD62BE3D707015F6B100E606F51AD40
:109AC0000AD0860EF66E1D0EF76E000EF86E0001BF
:109AD00043EC1CF00701070EEA6E590EE96E000117
:109AE00073D60D0EA4A8FED76D6E0A0EA4A8FED7DD
:109AF0006D6E0B0EEA6EB00EE96E000E58EC08F0BB
:109B00000A000900F550EE6E0009FBE10B01D66B6F
:109B1000D65105081AE3040ED625036AB00F016E6C
:109B20000B0E032203C0D8FB036AD651590FE96E0E
:109B3000070E0320EA6EEFCFD9FBD8CBEAFF01C0B6
:109B4000E9FFD9CBEFFFD62BE3D70B0ED86FB00EC2
:109B5000D76F0001F7EC14F026D00B01070151ADCF
:109B60000AD0900EF66E1D0EF76E000EF86E000114
:109B700043EC1CF00701110E606F0B0EEA6EB00E85
:109B8000E96E000E00016BEC08F00A000900F550C8
:109B9000EE6E0009FBE10B0E0B01D86FB00ED76F14
:109BA0000001F7EC14F025D00B01070151AD0AD0EC
:109BB000A20EF66E1D0EF76E000EF86E000143EC5D
:109BC0001CF00701606B0B0EEA6EB00EE96E000E22
:109BD00000010CEC08F00A000900F550EE6E0009D7
:109BE000FBE10B0E0B01D86FB00ED76F0001F7EC45
:109BF00014F0A4EF4FF00B01CD6B710E6725E96EE9
:109C0000090E6821EA6EEFCFCDFB010E6725CE6FFE
:109C1000000E6821CF6FE8CFBCFDCECBBBFD010E9F
:109C20000D01BE6FF40EBD6F0001D7EC1CF000C03B
:109C300067FB0B0103C068FB6551675D04E166517A
:109C4000685D01E1309CCDCB01F0000112000B01F9
:109C5000CC6B30AC06D00001CEDF01C0CCFB0B01D9
:109C6000F8D7696B00018EEF4EF00B01B56BB46B4A
:109C7000B36BB26BB76BB66BCA6BCB81CB8307018F
:109C800051AD09D00A0EF66E1E0EF76E000EF86E7C
:109C9000000143EC1CF00B01CBA3BCD0B7CBB8FD4B
:109CA000B6CBB7FD0D01BA6BFA0EB96F000158ECD7
:109CB0001CF002C0CDFB01C0CCFB0B01B151025C1A
:109CC0002BE303E1B051CC5D27E3070151AD21D077
:109CD0001E0EF66E1E0EF76E000EF86E0B0E0D01C8
:109CE000B66F000169EC1CF0100EE96EB1CBB7FD48
:109CF000B0CBB6FD82EC1CF02C0EF66E1E0EF76E8D
:109D0000000EF86E070E0D01B66F000169EC1CF035
:109D10000701000E016E81D0000199D7600E0B0182
:109D2000DD6FDE6B00017EEC27F00B0E0B01DE6FAA
:109D3000B80EDD6F0D0EDF6F070EE16FD00EE06F16
:109D4000000183EC3EF001C0CAFB0B01CA2D01D01B
:109D500001D0CB910B0EDE6FB80EDD6F0D0EDF6FF5
:109D6000EF0EE06F0001C0EC3EF00150090802E385
:109D70000B01CB910B01CBA141D0BDCBDEFB000190
:109D80006DEC25F001500F0B0B01C66FBECBDEFB57
:109D900000016DEC25F00138006EF00E0016005049
:109DA000F00B0B01CC6FBFCBDEFB00016DEC25F09F
:109DB00001500F0B0B01CC11C76FC0CBDEFB0001B4
:109DC0006DEC25F00138006EF00E00160050F00B1F
:109DD0000B01CC6FC1CBDEFB00016DEC25F0015017
:109DE0000F0B0B01CC11C86FB56BC6CBB4FBC7CB47
:109DF000B3FBC8CBB2FBB3BD01D0CB93CB81FA0E82
:109E00000D01B66F000117EC13F00B01B62BD8B49F
:109E1000B72B42D7010E016E07010001BEEF4FF0D4
:109E20000B01B06B070151A523D0000141EC1FF0DD
:109E3000090E0B01DD6FDE6B00017EEC27F00B0ECF
:109E40000B01CA6FB00EC96F050ECB6F070ECD6F39
:109E5000D00ECC6F0001C7EC2AF0012C05D0B0CB9E
:109E600077F7010E016E06D0FF0E016E03D00701D9
:109E7000FF0E016E0001E6EF4FF00B01AD6BAE6B14
:109E8000AF919D920B0EEA6E9B0EE96E006A026A1C
:109E9000120E016E0001AAEC1BF00B0EEA6E9B0E77
:109EA000E96E000EB6EC06F00A000900F550EE6E01
:109EB0000009FBE10B0E0B01D86F9B0ED76F000161
:109EC000F7EC14F00701606B080E0B01B06FFA0E8F
:109ED0000D01B66F000117EC13F00B01B02FF7D78F
:109EE0005E0EDD6FDE6B00017EEC27F0030E0C01D1
:109EF0000C6FE80E0B6F00013EEC27F001C0ADFBCC
:109F00000B01AD2D01D01CD0280EB06FFA0E0D0143
:109F1000B66F000117EC13F00B01B02FF7D75E0EF0
:109F2000DD6FDE6B00017EEC27F0030E0C010C6F81
:109F3000E80E0B6F00013EEC27F001C0ADFB0B01FA
:109F4000AD2D85D0000154D407016053D8B480D022
:109F50004C0E0B01DD6FDE6B00017EEC27F01F0E57
:109F60000C010C6F400E0B6F00013EEC27F03E0E13
:109F70000B01B16F800EB06F000177D6200E0B0180
:109F8000DD6F010EDE6F00017EEC27F0640E0D0127
:109F9000B66F000117EC13F0800E0701726F696B4A
:109FA000686F676B666F656B756B010E736F746BB3
:109FB000020E6F6F6E6B6D6B800E6A6F6C6F6B6BEA
:109FC000010E716F000107EC3BF02AD7010E0B0167
:109FD000B06F0001D4EC3BF0012C15D0010E0B0149
:109FE000B06F0001D0EC42F04F984F86400E0B014D
:109FF000C66F0C0EC76F4FC0C8FB0001C0EC11F05C
:10A0000030800B01AF810B01AFB121D0070151AD01
:10A0100009D0A20EF66E180EF76E000EF86E000153
:10A0200043EC1CF0370E0B01DD6F010EDE6F0001FB
:10A030007EEC27F04F904F92400E0B01C66F0C0E36
:10A04000C76F4FC0C8FB0001C0EC11F00B01070146
:10A05000966884CF35F0976885CF36F00B01AE6BEC
:10A06000AE5107080AE3036AAE513F0FE96E000ED6
:10A070000320EA6EEF6AAE2BF3D79D820001120037
:10A0800041EC1FF00B01FE6BFF6B00017CEC2EF02E
:10A090000B0E0B01FF6FAF0EFE6F0A0E0C01006F6F
:10A0A000070E026FD00E016F00010DEC46F0012C7F
:10A0B00004D0010E016E3DD03CD04B0E0B01FE6F63
:10A0C000FF6B00017CEC2EF0140E0D01B66F000149
:10A0D00017EC13F00B0E0B01FF6FAF0EFE6F0A0EA5
:10A0E0000C01006F070E026FD00E016F00010DEC26
:10A0F00046F0012C19D00B01B23D17D0B151030825
:10A1000014E14C0EFE6FFF6B00017CEC2EF04E0E46
:10A110000D019D6F200E9C6F000118EC2EF0012C9C
:10A1200003D0000E016E05D00B01000E016E000180
:10A1300000D012000B01D769D669000141EC1FF075
:10A14000650E0B01FE6FFF6B00017CEC2EF00B0E19
:10A150000B01FF6FD80EFE6F0A0E0C01006F130E7D
:10A16000026F880E016F00010DEC46F0012C0CD03F
:10A170000B01DF3D01D002D0DC3D04D0DACBD7FBB0
:10A18000DBCBD6FB25D0000141EC1FF0650E0B01A7
:10A19000FE6FFF6B00017CEC2EF00B0E0B01FF6FCE
:10A1A000D80EFE6F0A0E0C01006F130E026F880EA0
:10A1B000016F00010DEC46F0012C0BD00B01DF3DCF
:10A1C00001D002D0DC3D04D0DACBD7FBDBCBD6FB11
:10A1D0000001D7CB53F7D6CB52F718EF52F0040E4D
:10A1E0000B01FE6FFA0E0D01B66F000117EC13F0B4
:10A1F0000B01FE2FF7D7000141EC1FF0640E0B019D
:10A20000FE6FFF6B00017CEC2EF00B0E0B01FF6F5D
:10A21000D60EFE6F280E0C01006F070E026FD00ED7
:10A22000016F00010DEC46F0012C11D00B01FC3D3B
:10A230000DD0E751480804E1010E016E0BD006D0A5
:10A24000E751530803E1020E016E04D00001000E35
:10A25000016E0B01000196EF54F00B01B06BAF6B78
:10A26000B16BC26B900EC36FF00EC46F07012D6B04
:10A270002C6B2F6B2E6B316B306B326B0B0EEA6ECF
:10A28000C50EE96E006A026A110E016E0001AAECA9
:10A290001BF00B0EEA6EB20EE96E006A026A100E37
:10A2A000016EAAEC1BF0010E0B01FE6FFF6B0001AB
:10A2B0007CEC2EF0070151AD0AD0B60EF66E180EEA
:10A2C000F76E000EF86E000143EC1CF0070130BA87
:10A2D00032D0B0CBB8FDAFCBB7FD0D01BA6B320EAB
:10A2E000B96F000158EC1CF002C0D7FB01C0D6FBCF
:10A2F0000B01D75303E1D651C70811E2070151AD55
:10A300000AD0C60EF66E180EF76E000EF86E00013B
:10A3100043EC1CF00701000E016E47EF55F0320EC2
:10A320000D01B66F000117EC13F00B01AF2BD8B481
:10A33000B02B0701CCD730AA38D00B01C2510F087F
:10A34000D8B002D0070131D00001FAEC1CF001C0F6
:10A35000B1FB0A0E0D01B66F000117EC13F00B01F3
:10A36000C351B15D03E0C451B15D04E1C26BB1CB37
:10A37000B2FB0AD0C22B036AC251B20FE96E0B0EB8
:10A380000320EA6EB1CBEFFF070151AD0DD0B1CB89
:10A39000B7FD570E0D01B86F0001B7EC1BF0200E92
:10A3A000A4A8FED76D6E0701C6D751AD08D00A0E1E
:10A3B000A4A8FED76D6E0D0EA4A8FED76D6E0B017E
:10A3C000B25190080BE1B351380808E1B43D06D012
:10A3D000010E016E070147EF55F00B01B251F00875
:10A3E0000AE1B351380807E1B43D05D0010E016E12
:10A3F00007014DD30B01C2510408D8B021D3B4CB0F
:10A400002DF7B5CB2CF7B6CB2FF7B7CB2EF7B8CBB4
:10A4100031F7B9CB30F7BACB32F7070130510E081C
:10A42000D8A4EBD031510E08D8A4E7D0000182D6D1
:10A430000701523D05D0533D03D0010E536F526BBF
:10A440005251006E5351036E010E035C04E1005241
:10A4500000012FE00701035005E1020E005C00013E
:10A4600045E00701035005E1030E005C00013EE0FA
:10A470000701010E035C05E1010E005C00013BE0F9
:10A480000701010E035C05E1020E005C000150E0D3
:10A490000701020E035C04E10052000166E00701BF
:10A4A000030E035C05E100520001D8B47BD0070124
:10A4B00096D0070151AD0AD0D20EF66E180EF76E87
:10A4C000000EF86E000143EC1CF007010B0EEA6E63
:10A4D000C50EE96E000E0001C9EC06F00A00090085
:10A4E000F550EE6E0009FBE1070179D0010E07017E
:10A4F000536F526F0001070151AD0AD0E40EF66EA2
:10A50000180EF76E000EF86E000143EC1CF0070108
:10A510000B0EEA6EC50EE96E000E0001DCEC06F0D3
:10A520000A000900F550EE6E0009FBE1070157D063
:10A53000070151AD0AD0FC0EF66E180EF76E000E34
:10A54000F86E000143EC1CF007010B0EEA6EC50E1D
:10A55000E96E000E0001EFEC06F00A000900F5506C
:10A56000EE6E0009FBE107013AD0070151AD0AD0B8
:10A570001A0EF66E190EF76E000EF86E000143EC1F
:10A580001CF007010B0EEA6EC50EE96E000E00010D
:10A5900002EC07F00A000900F550EE6E0009FBE13D
:10A5A00007011DD0070151AD0AD02C0EF66E190E11
:10A5B000F76E000EF86E000143EC1CF007010B0E65
:10A5C000EA6EC50EE96E000E000115EC07F00A00F8
:10A5D0000900F550EE6E0009FBE1070100D00E0EF8
:10A5E000606F0B0E0B01D86FC50ED76F0001F7EC33
:10A5F00014F0000E016E07014AD22E51006E2F5149
:10A60000036E040E035C05E1020E005C000153E0E2
:10A610000701040E035C06E10D0E005C0001D8B4D6
:10A6200068D00701040E035C06E10E0E005C000119
:10A63000D8B47DD00701050E035C06E1030E005C73
:10A640000001D8B4B5D00701050E035C06E1010E88
:10A65000005C0001D8B4ACD00701040E035C06E135
:10A660000F0E005C0001D8B4E8D00701050E035CB2
:10A6700006E1050E005C0001D8B4FDD00701050E0F
:10A68000035C06E1070E005C0001D8B412D107019B
:10A69000050E035C06E1040E005C0001D8B427D16E
:10A6A0000701040E035C06E12D0E005C0001D8B426
:10A6B0003CD107019ED1010E0701606F51AD0AD058
:10A6C0003E0EF66E190EF76E000EF86E000143ECAA
:10A6D0001CF007010B0EEA6EC50EE96E000E0001BC
:10A6E00028EC07F00A000900F550EE6E0009FBE1C6
:10A6F0009DD1020E0701606F51AD0AD0500EF66E6B
:10A70000190EF76E000EF86E000143EC1CF0070105
:10A710000B0EEA6EC50EE96E000E00013BEC07F071
:10A720000A000900F550EE6E0009FBE17FD1070138
:10A730002C51400820E12D531EE10E0E606F51ADEB
:10A740000AD0620EF66E190EF76E000EF86E00015A
:10A7500043EC1CF007010B0EEA6EC50EE96E000E0D
:10A760000001C9EC06F00A000900F550EE6E000980
:10A77000FBE11DD00701030E606F51AD0AD0740ECE
:10A78000F66E190EF76E000EF86E000143EC1CF029
:10A7900007010B0EEA6EC50EE96E000E00014EECCD
:10A7A00007F00A000900F550EE6E0009FBE13ED10A
:10A7B00007012E2D25D02F51050822E12C2D20D068
:10A7C0002D531EE1090E606F51AD0AD0860EF66E54
:10A7D000190EF76E000EF86E000143EC1CF0070135
:10A7E0000B0EEA6EC50EE96E000E000161EC07F07B
:10A7F0000A000900F550EE6E0009FBE11DD00701CB
:10A80000010E606F51AD0AD0980EF66E190EF76EFC
:10A81000000EF86E000143EC1CF007010B0EEA6E0F
:10A82000C50EE96E000E000174EC07F00A00090085
:10A83000F550EE6E0009FBE1F9D0080E0701606FDC
:10A8400051AD0AD0A80EF66E190EF76E000EF86E16
:10A85000000143EC1CF007010B0EEA6EC50EE96E19
:10A86000000E000187EC07F00A000900F550EE6EBB
:10A870000009FBE1DBD0070E0701606F51AD0AD084
:10A88000BA0EF66E190EF76E000EF86E000143EC6C
:10A890001CF007010B0EEA6EC50EE96E000E0001FA
:10A8A0009AEC07F00A000900F550EE6E0009FBE192
:10A8B000BDD00F0E0701606F51AD0AD0CC0EF66E01
:10A8C000190EF76E000EF86E000143EC1CF0070144
:10A8D0000B0EEA6EC50EE96E000E0001ADEC07F03E
:10A8E0000A000900F550EE6E0009FBE19FD0040E4E
:10A8F0000701606F51AD0AD0DE0EF66E190EF76ECD
:10A90000000EF86E000143EC1CF007010B0EEA6E1E
:10A91000C50EE96E000E0001C0EC07F00A00090048
:10A92000F550EE6E0009FBE181D059D40150010AC7
:10A9300005E0030A21E0020A3DE03CD00B0E0701CE
:10A94000606F51AD0AD0F00EF66E190EF76E000E64
:10A95000F86E000143EC1CF007010B0EEA6EC50E09
:10A96000E96E000E0001D3EC07F00A000900F55073
:10A97000EE6E0009FBE13BD00A0E0701606F51AD9E
:10A980000AD00A0EF66E1A0EF76E000EF86E00016F
:10A9900043EC1CF007010B0EEA6EC50EE96E000ECB
:10A9A0000001E6EC07F00A000900F550EE6E000920
:10A9B000FBE11DD0070151AD0AD0240EF66E1A0E30
:10A9C000F76E000EF86E000143EC1CF00701110E4B
:10A9D000606F0B0EEA6EC50EE96E000E0001F9EC19
:10A9E00007F00A000900F550EE6E0009FBE11ED0E9
:10A9F000070151AD0AD0360EF66E1A0EF76E000E34
:10AA0000F86E000143EC1CF00701110E606F0B0E95
:10AA1000EA6EC50EE96E000E0001F9EC07F00A00BF
:10AA20000900F550EE6E0009FBE100D00B0E0B01A2
:10AA3000D86FC50ED76F0001F7EC14F025D00B01CD
:10AA4000070151AD0AD0480EF66E1A0EF76E000ED1
:10AA5000F86E000143EC1CF00701606B0B0EEA6E10
:10AA6000C50EE96E000E00010CEC08F00A000900AA
:10AA7000F550EE6E0009FBE10B0E0B01D86FC50E11
:10AA8000D76F0001F7EC14F0000E016E0701000112
:10AA9000120041EC1FF00B0E0B01FE6FFF6B00016B
:10AAA0007CEC2EF0140E0D01B66F000117EC13F0C4
:10AAB0000B0E0B01FF6FB10EFE6F0A0E0C01006F43
:10AAC000070E026FD00E016F00010DEC46F0012C55
:10AAD00006D00B01B43D02D0B3CB65F700011200E4
:10AAE0000B01B16B000141EC1FF00E0E0B01FE6F6C
:10AAF000FF6B00017CEC2EF00B0E0B01CA6FB10E48
:10AB0000C96F040ECB6F070ECD6FD00ECC6F000156
:10AB1000C7EC2AF0012C02D0B1CB6CF712000B016C
:10AB2000B16B000141EC1FF0070E0B01FE6FFF6BD4
:10AB300000017CEC2EF00B0E0B01CA6FB10EC96F39
:10AB4000040ECB6F070ECD6FD00ECC6F0001C7EC9B
:10AB50002AF0012C02D0B1CB6BF712000B01B16BC4
:10AB6000000141EC1FF00C0E0B01FE6FFF6B0001AA
:10AB70007CEC2EF00B0E0B01CA6FB10EC96F040EE8
:10AB8000CB6F070ECD6FD00ECC6F0001C7EC2AF053
:10AB9000012C02D0B1CB6AF712000B01B16B00019E
:10ABA00041EC1FF0040E0B01FE6FFF6B00017CEC0B
:10ABB0002EF00B0E0B01CA6FB10EC96F040ECB6FD6
:10ABC000070ECD6FD00ECC6F0001C7EC2AF0012C20
:10ABD0002ED0070160510E0827E10B01B15107018A
:10ABE000715D01E123D0640E0D01B66F000117EC19
:10ABF00013F0040E0B01FE6FFF6B00017CEC2EF0D6
:10AC00000B0E0B01CA6FB10EC96F040ECB6F070E8E
:10AC1000CD6FD00ECC6F0001C7EC2AF0012C02D012
:10AC2000B1CB71F704D00701B1CB71F7000112006D
:10AC30000B01B16B000141EC1FF0100E0B01FE6F18
:10AC4000FF6B00017CEC2EF00B0E0B01CA6FB10EF6
:10AC5000C96F040ECB6F070ECD6FD00ECC6F000105
:10AC6000C7EC2AF0012C02D0B1CB70F712000B0117
:10AC7000B16B000141EC1FF0110E0B01FE6FFF6B79
:10AC800000017CEC2EF00B0E0B01CA6FB10EC96FE8
:10AC9000040ECB6F070ECD6FD00ECC6F0001C7EC4A
:10ACA0002AF0012C02D0B1CB6FF712000B01B16B6F
:10ACB000000141EC1FF00F0E0B01FE6FFF6B000156
:10ACC0007CEC2EF00B0E0B01CA6FB10EC96F040E97
:10ACD000CB6F070ECD6FD00ECC6F0001C7EC2AF002
:10ACE000012C02D0B1CB6EF712000B01B16B000149
:10ACF00041EC1FF0070160510E083DE1180E0B01F9
:10AD0000FE6FFF6B00017CEC2EF00B0E0B01CA6F87
:10AD1000B10EC96F040ECB6F070ECD6FD00ECC6F86
:10AD20000001C7EC2AF0012C06D00B01B15107013C
:10AD3000755D01E120D0640E0D01B66F000117ECC6
:10AD400013F0180E0B01FE6FFF6B00017CEC2EF070
:10AD50000B0E0B01CA6FB10EC96F040ECB6F070E3D
:10AD6000CD6FD00ECC6F0001C7EC2AF0012C02D0C1
:10AD7000B1CB75F707010001120041EC1FF007018C
:10AD800060510E0834E1525332E1535103082FE170
:10AD9000190E0B01FE6FFF6B00017CEC2EF0140E00
:10ADA0000D01B66F000117EC13F00B0E0B01FF6FD6
:10ADB000B10EFE6F0A0E0C01006F070E026FD00E6F
:10ADC000016F00010DEC46F0012C13D00B01B43DD6
:10ADD0000FD0B351020A000103E0010A05E004D0DC
:10ADE000010E07016D6F03D007016D6B00D00B01E1
:10ADF0000001120041EC1FF0070160510E0834E120
:10AE0000525332E1535103082FE11A0E0B01FE6F2A
:10AE1000FF6B00017CEC2EF0140E0D01B66F0001EB
:10AE200017EC13F00B0E0B01FF6FB10EFE6F0A0E45
:10AE30000C01006F070E026FD00E016F00010DECC8
:10AE400046F0012C13D00B01B43D0FD0B351020AD0
:10AE5000000103E0010A05E004D0010E07016E6F56
:10AE600003D007016E6B00D00B01000112000B0133
:10AE7000B16B000141EC1FF0070160510E084AE17F
:10AE8000525348E15351030845E176510D0803E25E
:10AE900076511B0802E20E0E766F1B0E0B01FE6F41
:10AEA000FF6B00017CEC2EF00B0E0B01CA6FB10E94
:10AEB000C96F040ECB6F070ECD6FD00ECC6F0001A3
:10AEC000C7EC2AF0012C06D00B01B1510701765DC9
:10AED00001E120D0640E0D01B66F000117EC13F0F4
:10AEE0001B0E0B01FE6FFF6B00017CEC2EF00B0EB6
:10AEF0000B01CA6FB10EC96F040ECB6F070ECD6F79
:10AF0000D00ECC6F0001C7EC2AF0012C02D0B1CBDF
:10AF100076F70701000112000B01AD6BAE919D9217
:10AF20000B0EEA6E9B0EE96E006A026A120E016E4B
:10AF30000001AAEC1BF00B0EEA6E9B0EE96E000EF0
:10AF40006AEC06F00A000900F550EE6E0009FBE11C
:10AF50000B0E0B01D86F9B0ED76F0001F7EC14F0AE
:10AF60000701606B080E0B01AF6FFA0E0D01B66F93
:10AF7000000117EC13F00B01AF2FF7D7000140ECE5
:10AF800050F0015225E140EC50F0015221E10B0E4E
:10AF9000EA6E9B0EE96E006A026A120E016EAAEC5E
:10AFA0001BF00B0EEA6E9B0EE96E000E7DEC06F0B8
:10AFB0000A000900F550EE6E0009FBE10B0E0B01D3
:10AFC000D86F9B0ED76F0001F7EC14F09D8269D10A
:10AFD000080E0B01AF6FFA0E0D01B66F000117ECF2
:10AFE00013F00B01AF2FF7D700012DEC51F0012C1E
:10AFF00002D02DEC51F007016053D8B43BD151AFD2
:10B0000018D0320E0D01B66F000117EC13F0070EC9
:10B010000B01B16F540EB06F070EB36F560EB26FC7
:10B02000070EB56F580EB46F0001BCEC24F039D197
:10B030000701000107EC3BF0012C01D007D0640EA2
:10B040000D01B66F000117EC13F0F4D70701605142
:10B050000E082BE0010E0B01B06F0001D4EC3BF0A9
:10B06000012C21D0010E0B01B06F0001D0EC42F099
:10B070004F984F86400E0B01C66F0C0EC76F4FC026
:10B08000C8FB0001C0EC11F030800B01AE8107015C
:10B0900051AD0AD0360EF66E180EF76E000EF86E31
:10B0A000000143EC1CF0070145D0525312E153510B
:10B0B00002080FE1200E0B01FE6F010EFF6F000171
:10B0C0007CEC2EF007EC3BF0070164510B0801E229
:10B0D0006189030E0B01B06F0001D4EC3BF0012C31
:10B0E00026D0030E0B01B06F0001D0EC42F04F8868
:10B0F0004F86400E0B01C66F0C0EC76F4FC0C8FBCA
:10B100000001C0EC11F08A92939230800B01AE8165
:10B11000070151AD0AD04E0EF66E180EF76E000EF6
:10B12000F86E000143EC1CF0070104D000018A8294
:10B13000939207010B01AEB19CD0070151AD09D02C
:10B140006C0EF66E180EF76E000EF86E000143ECF2
:10B150001CF00001D4EC48F007EC3BF00701605113
:10B160000E0817E1960E0D01B66F000117EC13F0F3
:10B170000701525309E15351030806E14FB004D0CF
:10B18000000187DC04D00701000168EC4AF004D01C
:10B190000701000168EC4AF056EC46F007016051E7
:10B1A0000E0807E00001BEEC41F070EC40F01BD04F
:10B1B000070161A108D01E0E0B01FE6F010EFF6F8B
:10B1C00000017CEC2EF00001BEEC41F070EC40F090
:10B1D000070161A109D01C0E0B01FE6F010EFF6F6C
:10B1E00000017CEC2EF007016051090807E1000125
:10B1F00077DC95DCB3DCD1DC3BD00701605107087C
:10B2000003E060510F0807E1000112DD30DD4EDD83
:10B21000C4DC2ED0070160510E0819E100010DECCD
:10B2200047F0D6EC47F055EC48F0B4EC45F0070198
:10B23000525303E15351030804E0000156DD05D0E9
:10B24000070100019ADDD6DD12DE12D00701605140
:10B250000D080BE100010DEC47F0D6EC47F055EC82
:10B2600048F0B4EC45F004D007010001B4EC45F01F
:10B270000B010701966884CF35F0976885CF36F0CB
:10B280000B01AD6BAD5107080AE3036AAD513F0FE7
:10B29000E96E000E0320EA6EEF6AAD2BF3D79D82B4
:10B2A000000112000B0184518519800B876F84AF58
:10B2B00002D0841F842B85AF02D0851F852B85513A
:10B2C000016A845D03E284CB00F00CD0006A080EB2
:10B2D000866F843700368551005CD8B0006E013629
:10B2E000862FF7D787AF02D0011E012A0001120076
:10B2F0000B019E519EAF03D0000ED8809E55006E6C
:10B30000E8BE03D00050010803E39ECB01F038D023
:10B310009EBF01D01DD09E519EAF03D0000ED8809D
:10B320009E55006EE8BE06D000501D0803E2E20EF6
:10B33000016E26D09E519EAF03D0000ED8809E5540
:10B34000006ED89000320050FF0A010F016E18D035
:10B350009EBF16D09E51000813E29E519EAF03D0AF
:10B36000000ED8809E55006EE8BE06D000501D0825
:10B3700003E21E0E016E04D0D8909E31016E00D003
:10B380000001120001509BCB25FC640E0C01266FBE
:10B3900000017CEC25F000C09BFB0150300E08E161
:10B3A0000B019CA30FD09CB70DD09CB9200E04D0EC
:10B3B0000B019C979C999C81012601C0A6FB000172
:10B3C000C3EC13F09BCB25FC0A0E0C01266F000189
:10B3D0007CEC25F000C09BFB0150300E08E10B0116
:10B3E0009CB70BD09CA109D09CB9200E000101266E
:10B3F00001C0A6FBC3EC13F00B01300E9B279BCBC7
:10B40000A6FB0001C3EC13F01200200E0B019DA956
:10B41000300E9E6F9CCB00F09CAF07D0001E002A20
:10B4200000C09CFB2D0E9E6F9D8F01509CCB25FC78
:10B43000640E0C01266F00017CEC25F000C09CFB23
:10B44000300E01240B019F6F9CCB25FC0A0E0C01D2
:10B45000266F00017CEC25F0300E00240B01A16F5B
:10B46000300E0124A06F9ECB00F09DA702D09DAFAF
:10B470009D959DB90BD09DAF22D09DB520D000C029
:10B480009FFB9DB31CD000C0A0FB19D0300E9F5D68
:10B4900016E100C09FFB200E9E6F9DA704D09D95D6
:10B4A0009D839DAF9D93300EA05D09E100C0A0FB80
:10B4B000200E9F6F9DA7F7D79D939DAF9D919DA552
:10B4C00006D09ECBA6FB0001C3EC13F00B019DA39D
:10B4D00006D09FCBA6FB0001C3EC13F00B019DA18E
:10B4E00005D0A0CBA6FB0001C3EC13F0A1CBA6FBBB
:10B4F0000001C3EC13F012000B01A351A519800B3E
:10B50000A76FA3AF05D0A21FA31FA22BD8B4A32B54
:10B51000A5AF05D0A41FA51FA42BD8B4A52BA2515D
:10B52000A403F3CF01F0F4CF00F0A503F3500026FD
:10B53000A351A403F3500020026EA7AF05D0011E53
:10B54000021E012AD8B4022A000112000B019F6BCF
:10B550009E6BA16BA06B9DCB03F09C519DAF08D05F
:10B56000000ED8809C55006E000E9D55036E005055
:10B57000A06F03C0A1FBA15308E1A051070805E398
:10B580009DCB9FFB9CCB9EFB3FD0A15312E1A051D2
:10B590000E080FE39DCBA3FB9CCBA2FBA56B040E77
:10B5A000A46F0001A9DF02C09FFB01C09EFB2CD04D
:10B5B0000B01A15312E1A0511D080FE39DCBA3FB8A
:10B5C0009CCBA2FBA56B060EA46F000195DF02C009
:10B5D0009FFB01C09EFB18D00B019DCBA3FB9CCB16
:10B5E000A2FB9DCBA5FB9CCBA4FB000185DF02C089
:10B5F0009FFB01C09EFB0B019DBF01D005D09E1F8C
:10B600009F1F9E2BD8B49F2B0B019ECB01F09FCB8D
:10B6100002F00001ACEF61F0EACFA5FBE9CFA4FB9B
:10B620000B019EAF08D0A48FA4A9A42B9D1F9E1F21
:10B630009D2BD8B49E2B9E39F009A06FA027E20F56
:10B64000A16F320FA36F9E510F0BA127A127A32734
:10B65000E90FA26FA227A2279D390F0BA227A327CC
:10B66000A237A337A31FA3379D510F0BA327A037E2
:10B67000070E9F6F0A0EA207A327FDE3A107A227CB
:10B68000FDE3A007A127FDE39F07A027FDE30B0E25
:10B69000EA6E9F0EE96E070EA415A49DE906A41597
:10B6A00007E1A4B9E92AA4B903D0200E006E1CD08A
:10B6B000E926A30EE95CD8B4A48DEF50006E08E132
:10B6C000A4BD06D0A4B91ED0A4B702D0200E0BD0C2
:10B6D000A4AF06D02D0E006EED50A49DA49F04D003
:10B6E000A487A499300E0026EACF9EFBE9CF9DFBEC
:10B6F00000C0A6FB0001C3EC13F09ECBEAFF9DCB7C
:10B70000E9FF0B01EE50A4ADD4D7000112000900EF
:10B71000F55211E0F6CF9BFBF7CF9CFBF8CF9DFBDA
:10B72000F5CFA6FBC3EC13F09BCBF6FF9CCBF7FF4A
:10B730009DCBF8FFECD712000B01936B946B956BCC
:10B74000966B986B976B996B9A918153D8A44BEF3A
:10B750006CF0936B93510308D8A049EF6CF0036A27
:10B760009351470FE96E000E0320EA6EEF52D8B4F2
:10B770003EEF6CF0000141EC1FF00701482D44D072
:10B780000B019351030A000101E039D0020E0701B9
:10B790004D6F4C513F0803E14AC74CF701D04C2B89
:10B7A0004C51020801E24C6B4C51060DF350036AF8
:10B7B000030F016E060E032201C09BFB0B0103C0A9
:10B7C0009CFB0B0E6B6F820E6A6F6E0EF66E110E87
:10B7D000F76E000EF86E070E9D6F0001D3EC13F0AC
:10B7E0009CCBEAFF9BCBE9FFEBEC13F00B0E0B01BC
:10B7F000D86F820ED76F0001F7EC14F002D02CEF57
:10B800007BF03DEF6CF007010B019351FC0FD8B0BA
:10B810003EEF6CF0040F00012DEF7BF0070160514B
:10B8200010083FE14FB43DD00B019C6B6CC79BFBF4
:10B83000036A9351470FE96E000E0320EA6EEFCFC3
:10B840009DFB9DCB9EFB000153DD036A0150E8BECA
:10B8500003060B019B25976F03509C21986F98BF9F
:10B8600009D0985303E19751FE0804E207016C697F
:10B870000ED00B0198BF05D0985307E197510008EF
:10B8800004E307016C6B03D00B0197CB6CF7660EDA
:10B890000B01DD6F010EDE6F00017EEC27F073D22D
:10B8A000070160510E0802E081B225D24FA023D2D9
:10B8B000036A0B019351470FE96E000E0320EA6EF5
:10B8C000EFCF9BFB9BCB9EFB000112DD01500701DC
:10B8D00065250B01996F07016051090A000121E0FC
:10B8E0000E0A3FE0080AD8B467D0070AD8B48ED051
:10B8F0000A0AD8B48BD0060AD8B488D00F0AD8B4B4
:10B9000085D0050AD8B4A1D00D0AD8B402D1090A4D
:10B91000D8B4FFD0070AD8B41BD11D0AD8B45DD162
:10B9200099D10B0199BF08D09951070805E2080E7B
:10B930000701656F0DD00B0199BF03D09951010824
:10B9400005E3010E0701656F03D00B0199CB65F785
:10B950003B0E0B01FE6F010EFF6F00017CEC2EF021
:10B96000A6D10B0199BF06D09951190803E21A0E0E
:10B97000996F07D099BF03D09951010802E3010ED6
:10B98000996F99CB65F73B0EFE6F010EFF6F0001BB
:10B990007CEC2EF068EC4AF00B0199510701655DD3
:10B9A00009E0640E0D01B66F000117EC13F068ECAE
:10B9B0004AF0F2D700017BD10B0199BF06D0995113
:10B9C000190803E21A0E996F06D099BF03D0995156
:10B9D000000801E3996B99CB65F73B0EFE6F010EF2
:10B9E000FF6F00017CEC2EF068EC4AF00B019951DE
:10B9F0000701655D09E0640E0D01B66F000117ECEB
:10BA000013F068EC4AF0F2D7000151D10B0199BF55
:10BA100008D09951060805E2070E0701656F0CD0A2
:10BA20000B0199BF03D09951000804E30701656B2E
:10BA300003D00B0199CB65F73B0E0B01FE6F010E96
:10BA4000FF6F00017CEC2EF032D107015251006EE5
:10BA50005351036E030E035C04E10052000120E029
:10BA60000701020E035C04E10052000131E007010E
:10BA7000010E035C04E1005200012AE00701010EFF
:10BA8000035C05E1010E005C000122E00701010EEC
:10BA9000035C05E1020E005C00011AE0070118D00A
:10BAA0000B0199BF08D09951230805E2240E070124
:10BAB000656F0DD00B0199BF03D09951000804E3C5
:10BAC0000701656B04D00B0199CB65F7070118D00E
:10BAD0000B0199BF08D099511D0805E21E0E070100
:10BAE000656F0DD00B0199BF03D09951000804E395
:10BAF0000701656B04D00B0199CB65F7070100D0F6
:10BB00003B0E0B01FE6F010EFF6F00017CEC2EF06F
:10BB1000CED00B0199BF08D099510E0805E20F0E47
:10BB20000701656F0CD00B0199BF03D09951000834
:10BB300004E30701656B03D00B0199CB65F73B0E5E
:10BB40000B01FE6F010EFF6F00017CEC2EF0AFD0F9
:10BB50000B0199BF01D004D00701656B35D00B01F3
:10BB600099BF08D099511A0805E21A0E0701656FAE
:10BB70002BD00B0199BF03D09951080805E3080E9B
:10BB80000701656F21D00B0199BF0DD099511408A1
:10BB90000AE299BF03D09951160805E3170E070171
:10BBA000656F12D00B0199BF0DD0995117080AE2A9
:10BBB00099BF03D09951190805E31A0E0701656F63
:10BBC00003D00B0199CB65F73B0E0B01CE6F010E35
:10BBD000CF6F00014FEC1FF06AD00B019C6B72C756
:10BBE0009BFB036A9351470FE96E000E0320EA6E38
:10BBF000EFCF9DFB9DCB9EFB000178EC59F0036AD3
:10BC00000150E8BE03060B019B25976F03509C2152
:10BC1000986F98BF09D0985303E19751FE0804E24A
:10BC2000070172690ED00B0198BF05D0985307E148
:10BC30009751000804E30701726B03D00B0197CB07
:10BC400072F7500E0B01DD6F010EDE6F00017EEC0E
:10BC500027F02DD0036A0B0193513F0FE96E000EC0
:10BC60000320EA6EEFBE13D0EF50000810E2070188
:10BC700051B30BD051B509D0390E0B01FE6F010E37
:10BC8000FF6F00017CEC2EF007010FD00B010701C4
:10BC900051B30BD051B509D03A0E0B01FE6F010E16
:10BCA000FF6F00017CEC2EF00701000100D0640E54
:10BCB0000D01B66F000117EC13F007016051100879
:10BCC00004E0000168EC4AF007016051070803E056
:10BCD00060510F080FE10B0199510701655D0AE002
:10BCE000640E0D01B66F000117EC13F068EC4AF01A
:10BCF0000701F1D749D060510E083AE1525338E1BB
:10BD00005351030835E1036A0B019351470FE96E64
:10BD1000000E0320EA6EEFCF9BFB9BCB9EFB000146
:10BD200078EC59F00150070165250B01996F99BF17
:10BD300008D09951020805E2030E0701656F0CD087
:10BD40000B0199BF03D09951000804E30701656B0B
:10BD500003D00B0199CB65F73C0E0B01FE6F010E72
:10BD6000FF6F00017CEC2EF049EC55F00CD0070180
:10BD700060510E0802E081B207D06051100804E063
:10BD8000000168EC4AF007016051090A00011CE05B
:10BD9000060A46E0080A44E00F0A66E00A0A64E080
:10BDA000060A62E00F0A60E0050AD8B481D00D0AE5
:10BDB000D8B4CFD0090AD8B4CCD0070AD8B4EDD0C3
:10BDC0001D0AD8B42ED169D107016051090805E1D7
:10BDD0006551070802E2080E656F6551060DF350C4
:10BDE000036AE60F016E000E032201C09BFB0B01EC
:10BDF00003C09CFB0B0E6B6F820E6A6F780EF66EA3
:10BE0000110EF76E000EF86E0B0E9D6F0001D3EC55
:10BE100013F09CCBEAFF9BCBE9FFEBEC13F056D180
:10BE200007016551060DF350036ACA0F016E010E3A
:10BE3000032201C09BFB0B0103C09CFB0B0E6B6F2D
:10BE4000820E6A6F860EF66E110EF76E000EF86E99
:10BE50000B0E9D6F0001D3EC13F09CCBEAFF9BCB44
:10BE6000E9FFEBEC13F032D107016551060DF350F9
:10BE7000036A9E0F016E030E032201C09BFB0B01A0
:10BE800003C09CFB0B0E6B6F820E6A6F940EF66EF6
:10BE9000110EF76E000EF86E0B0E9D6F0001D3ECC5
:10BEA00013F09CCBEAFF9BCBE9FFEBEC13F00ED138
:10BEB0000701525329E15351030826E14FB024D022
:10BEC0006551070DF350036ACE0F016E030E032276
:10BED00001C09BFB0B0103C09CFB0B0E6B6F820E22
:10BEE0006A6FA20EF66E110EF76E000EF86E0A0E55
:10BEF0009D6F0001D3EC13F09CCBEAFF9BCBE9FFD5
:10BF0000EBEC13F025D007010B0E0B016B6F820ECB
:10BF10006A6FB00EF66E110EF76E000EF86E0B0E15
:10BF20009D6F0001D3EC13F065C79BFB1B0E0B014B
:10BF30009C6F0001C2EC59F0640E0B01A66F00016A
:10BF4000C3EC13F0420E0B01A66F0001C3EC13F01B
:10BF5000BDD007016551050DF350036AC90F016E8D
:10BF6000040E032201C09BFB0B0103C09CFB0B0EC4
:10BF70006B6F820E6A6FC00EF66E110EF76E000EBA
:10BF8000F86E0B0E9D6F0001D3EC13F09CCBEAFF13
:10BF90009BCBE9FFEBEC13F099D00E0E0B01956FE4
:10BFA00007016551140806E3080E655D0B01956FE6
:10BFB00015D007016551140808E26551170805E31B
:10BFC0000D0E0B01956F0AD007016551170806E2A7
:10BFD00065511A0803E30E0E0B01956F0B01955185
:10BFE000050DF350036A190F016E050E032201C0FF
:10BFF0009BFB03C09CFB0B0E6B6F820E6A6FCE0E19
:10C00000F66E110EF76E000EF86E0A0E9D6F0001AF
:10C01000D3EC13F09CCBEAFF9BCBE9FFEBEC13F0E6
:10C0200055D04FA41DD0800E0701725D0B019B6F90
:10C030000B0E6B6F820E6A6FDC0EF66E110EF76ED2
:10C04000000EF86E0C0E9D6F0001D3EC13F09BCB2D
:10C050009CFB1F0E0B019D6F000105EC5AF01CD0DC
:10C06000800E07016C5D0B019B6F0B0E6B6F820ED8
:10C070006A6FEC0EF66E110EF76E000EF86E0B0E78
:10C080009D6F0001D3EC13F09BCB9CFB1F0E0B01AB
:10C090009D6F000105EC5AF019D00B0E0B016B6F70
:10C0A000820E6A6FFA0EF66E110EF76E000EF86EC3
:10C0B0000C0E9D6F0001D3EC13F065C79BFB1B0EAC
:10C0C0000B019C6F0001C2EC59F000D00B0E0B016C
:10C0D000D86F820ED76F0001F7EC14F00B013EEF22
:10C0E0006CF0070160510E0802E081B2E0D14FB060
:10C0F00004D060511008D8A4DAD160510D0815E0C1
:10C10000036A0B019351470FE96E000E0320EA6E9C
:10C11000EFCF9BFB9BCB9EFB000178EC59F00150CD
:10C12000070164250B01996F07016051090A00019D
:10C130001FE0060A42E0080A40E0090A5DE0060A3C
:10C14000D8B4D9D0020AD8B4D6D0090AD8B4D3D03A
:10C15000010AD8B4D0D0060AD8B4CDD00F0AD8B4CA
:10C16000CAD0060AD8B4E6D01D0AD8B423D140D12B
:10C170000B0199BF08D09951150805E2160E070169
:10C18000646F0CD00B0199BF03D09951000804E3F0
:10C190000701646B03D00B0199CB64F7370E0B01D9
:10C1A000FE6F010EFF6F00017CEC2EF0640E0D019E
:10C1B000B66F000117EC13F070D10B0199BF08D0D6
:10C1C00099511B0805E21C0E0701646F0CD00B018E
:10C1D00099BF03D09951000804E30701646B03D0B1
:10C1E0000B0199CB64F7370E0B01FE6F010EFF6F49
:10C1F00000017CEC2EF051D107015251006E5351D9
:10C20000036E020E035C04E10052000120E007010E
:10C21000010E035C04E1005200014CE00701010E35
:10C22000035C05E1010E005C000144E00701010E22
:10C23000035C05E1020E005C00013CE00701030E17
:10C24000035C04E10052000135E0070133D007012F
:10C2500061A918D00B0199BF08D09951130805E2C4
:10C26000140E0701646F0DD00B0199BF03D09951D3
:10C27000000804E30701646B04D00B0199CB64F759
:10C28000070117D00B0199BF08D099510A0805E2A0
:10C290000B0E0701646F0DD00B0199BF03D09951AC
:10C2A000000804E30701646B04D00B0199CB64F729
:10C2B000070118D00B0199BF08D09951100805E269
:10C2C000110E0701646F0DD00B0199BF03D0995176
:10C2D000000804E30701646B04D00B0199CB64F7F9
:10C2E000070100D0370E0B01FE6F010EFF6F00013A
:10C2F0007CEC2EF0D2D00B0199BF08D099511008D8
:10C3000005E2110E0701646F0CD00B0199BF03D039
:10C310009951000804E30701646B03D00B0199CB2A
:10C3200064F7370E0B01FE6F010EFF6F00017CEC0E
:10C330002EF0B3D0036A0B019351470FE96E000E44
:10C340000320EA6EEFCF9BFB9D6B9BCB9CFB9CBFBE
:10C350009D070001A6EF5AF00150070162250B016D
:10C36000976F0250070163210B01986F98BF09D0A6
:10C370009851030806E2030E0701636F626911D04A
:10C380000B0198BF05D0985308E19751000805E3C9
:10C390000701636B626B05D00B0198CB63F797CBFA
:10C3A00062F7130E0B01CE6F010ECF6F00014FEC41
:10C3B0001FF073D00B0199BF01D001D0996B070119
:10C3C00061B714D00B0199BF08D0070177510B0159
:10C3D000995D03E377C764F702D099CB64F7370E12
:10C3E000DD6F010EDE6F00017EEC27F0000155D0FD
:10C3F000070151B350D051B54ED0036A0B01935190
:10C400003F0FE96E000E0320EA6EEFBE24D0EF501E
:10C41000000821E2946B036A93513F0FE96E000E0E
:10C420000320EA6EEFCF9BFB9B519BAF03D0000E26
:10C43000D8809B55006EE8BE0DD00050945D0AE296
:10C44000350EFE6F010EFF6F00017CEC2EF00B012C
:10C45000942BE1D720D0946B036A93513F0FE96E80
:10C46000000E0320EA6EEFCF9BFB9B519BAF03D0E6
:10C47000000ED8809B55006EE8BE0DD00050945D34
:10C480000AE2360EFE6F010EFF6F00017CEC2EF00B
:10C490000B01942BE1D7000100D0640E0D01B66FA3
:10C4A000000117EC13F007EC3BF009D007016051D5
:10C4B0000E0802E081B204D0000107EC3BF0070156
:10C4C0006051090A00011FE0060A41E0080A3FE046
:10C4D000090A61E0060AD8B4F8D0020AD8B4F5D047
:10C4E000080AD8B416D1010AD8B437D1070AD8B48B
:10C4F00058D10F0AD8B455D1060AD8B476D11D0A3E
:10C50000D8B48CD1D7D107016451060DF350036A1A
:10C51000500F016E000E032201C09BFB0B0103C0F4
:10C520009CFB0B0E6B6F820E6A6F0A0EF66E120E7C
:10C53000F76E000EF86E0B0E9D6F0001D3EC13F03A
:10C540009CCBEAFF9BCBE9FFEBEC13F0CCD10701CE
:10C550006451060DF350036A1C0F016E010E032295
:10C5600001C09BFB0B0103C09CFB0B0E6B6F820E8B
:10C570006A6F180EF66E120EF76E000EF86E0B0E46
:10C580009D6F0001D3EC13F09CCBEAFF9BCBE9FF3E
:10C59000EBEC13F0A8D107015251006E5351036E1A
:10C5A000020E035C04E10052000120E00701030ECB
:10C5B000035C04E10052000163E00701010E035C2B
:10C5C00004E1005200015CE00701010E035C05E19B
:10C5D000010E005C000154E00701010E035C05E15F
:10C5E000020E005C00014CE007014BD0070161A97D
:10C5F00024D06451060DF350036A200F016E030E20
:10C60000032201C09BFB0B0103C09CFB0B0E6B6F55
:10C61000820E6A6F260EF66E120EF76E000EF86E20
:10C620000B0E9D6F0001D3EC13F09CCBEAFF9BCB6C
:10C63000E9FFEBEC13F023D007016451060DF35032
:10C64000036AD80F016E020E032201C09BFB0B018F
:10C6500003C09CFB0B0E6B6F820E6A6F340EF66E7E
:10C66000120EF76E000EF86E0B0E9D6F0001D3ECEC
:10C6700013F09CCBEAFF9BCBE9FFEBEC13F024D04B
:10C6800007016451060DF350036A6C0F016E020E30
:10C69000032201C09BFB0B0103C09CFB0B0E6B6FC5
:10C6A000820E6A6F420EF66E120EF76E000EF86E74
:10C6B0000B0E9D6F0001D3EC13F09CCBEAFF9BCBDC
:10C6C000E9FFEBEC13F000D00ED107016451060D29
:10C6D000F350036A6C0F016E020E032201C09BFB34
:10C6E0000B0103C09CFB0B0E6B6F820E6A6F500E2A
:10C6F000F66E120EF76E000EF86E0B0E9D6F0001B7
:10C70000D3EC13F09CCBEAFF9BCBE9FFEBEC13F0EF
:10C71000EAD007016451060DF350036A970F016ECA
:10C72000050E032201C09BFB0B0103C09CFB0B0EFB
:10C730006B6F820E6A6F5E0EF66E120EF76E000E53
:10C74000F86E0B0E9D6F0001D3EC13F09CCBEAFF4B
:10C750009BCBE9FFEBEC13F0C6D007016451060D4B
:10C76000F350036A5D0F016E040E032201C09BFBB0
:10C770000B0103C09CFB0B0E6B6F820E6A6F6C0E7D
:10C78000F66E120EF76E000EF86E0B0E9D6F000126
:10C79000D3EC13F09CCBEAFF9BCBE9FFEBEC13F05F
:10C7A000A2D007016451060DF350036AF10F016E28
:10C7B000030E032201C09BFB0B0103C09CFB0B0E6D
:10C7C0006B6F820E6A6F7A0EF66E120EF76E000EA7
:10C7D000F86E0B0E9D6F0001D3EC13F09CCBEAFFBB
:10C7E0009BCBE9FFEBEC13F07ED00B0E0B016B6FD4
:10C7F000820E6A6F880EF66E120EF76E000EF86EDD
:10C800000A0E9D6F0001D3EC13F0020EE96E63C7B0
:10C810009EFB62C79DFB0CEC5BF065D04FA025D062
:10C820000B0E0B016B6F820E6A6F980EF66E120E76
:10C83000F76E000EF86E080E9D6F0001D3EC13F03A
:10C8400064C79BFB1B0E0B019C6F0001C2EC59F0EF
:10C85000A20EF66E120EF76E000EF86E040E0B01AD
:10C860009D6F0001D3EC13F024D00B0E0B016B6F06
:10C87000820E6A6FA80EF66E120EF76E000EF86E3C
:10C880000A0E9D6F0001D3EC13F064C79BFB1B0ED7
:10C890000B019C6F0001C2EC59F0200E0B01A66F3A
:10C8A0000001C3EC13F0200E0B01A66F0001C3ECD6
:10C8B00013F019D00B0E0B016B6F820E6A6FB80E5E
:10C8C000F66E120EF76E000EF86E0C0E9D6F0001E4
:10C8D000D3EC13F064C79BFB1B0E0B019C6F000194
:10C8E000C2EC59F000D00B0E0B01D86F820ED76F3F
:10C8F0000001F7EC14F00B013EEF6CF00701605102
:10C900000E0802E081B25FD26051090A00010EE018
:10C91000060A48E0080A46E0090AD8B47DD0030AAE
:10C92000D8B49BD11D0AD8B4D2D14BD24FB431D098
:10C93000036A0B019351470FE96E000E0320EA6E64
:10C94000EFCF9BFB9BCB9EFB000178EC59F0015095
:10C9500007016C250B01996F99BF08D099510D08FB
:10C9600005E20E0E07016C6F0CD00B0199BF03D0CE
:10C970009951000804E307016C6B03D00B0199CBBC
:10C980006CF7460E0B01FE6F010EFF6F00017CEC91
:10C990002EF0640E0D01B66F000117EC13F070EC71
:10C9A00055F010D2036A0B019351470FE96E000E48
:10C9B0000320EA6EEFCF9BFB9BCB9EFB000178EC44
:10C9C00059F00150070170250B01996F99BF08D0EC
:10C9D0009951130805E2140E0701706F0CD00B017A
:10C9E00099BF03D09951000804E30701706B03D08D
:10C9F0000B0199CB70F7480E0B01FE6F010EFF6F14
:10CA000000017CEC2EF0640E0D01B66F000117ECF6
:10CA100013F018EC56F0D6D14FA2E3D00B019C6B6B
:10CA200074C79BFB036A9351470FE96E000E032006
:10CA3000EA6EEFCF9DFB9DCB9EFB000178EC59F099
:10CA4000036A0150E8BE03060B019B25976F035054
:10CA50009C21986F07015251006E5351036E020ED4
:10CA6000035C04E10052000123E00701030E035CB4
:10CA700004E10052000138E00701010E035C05E10A
:10CA800000520001D8B479D00701010E035C06E121
:10CA9000010E005C0001D8B470D00701010E035CE8
:10CAA00006E1020E005C0001D8B467D0070165D032
:10CAB0000B0198BF05D0985307E19751000804E394
:10CAC0000701746B10D00B0198BF0AD0985303E193
:10CAD0009751CF0805E2CF0E0701746F04D00B0108
:10CAE00097CB74F7070165D00B019C6B72C79BFB5A
:10CAF000036A9351470FE96E000E0320EA6EEFCFF1
:10CB00009DFB9DCB9EFB000178EC59F0036A015020
:10CB1000E8BE03060B019B25976F03509C21986F7D
:10CB200098BF05D0985308E19751010805E3010E1D
:10CB30000701726F10D00B0198BF0AD0985303E120
:10CB40009751640805E2640E0701726F04D00B016F
:10CB500097CB72F70701510E0B01FE6F010EFF6FAD
:10CB600000017CEC2EF0640E0D01B66F000117EC95
:10CB700013F00DEC47F007011CD00B0198BF05D056
:10CB8000985307E19751000804E30701746B10D034
:10CB90000B0198BF0AD0985303E197518F0805E223
:10CBA0008F0E0701746F04D00B0197CB74F7070148
:10CBB00000D0525303E15351030811E0530E0B010F
:10CBC000FE6F010EFF6F00017CEC2EF0640E0D0174
:10CBD000B66F000117EC13F055EC48F007013BD09D
:10CBE0000001036A0B019351470FE96E000E032009
:10CBF000EA6EEFCF99FB07016E5314E10B0199BF69
:10CC00000FD0995100080CE2010E07016E6F570E0C
:10CC10000B01FE6F010EFF6F00017CEC2EF00B018B
:10CC200012D007010B0199BF03D0995100080BE303
:10CC300007016E6B580E0B01FE6F010EFF6F0001B6
:10CC40007CEC2EF00B01640E0D01B66F000117ECA9
:10CC500013F0FAEC56F00001B5D0036A0B019351C2
:10CC6000470FE96E000E0320EA6EEFCF9BFB9BCBD4
:10CC70009EFB000178EC59F00150070174250B016F
:10CC8000996F99BF03D09951000804E30701746BB1
:10CC90000DD00B0199BF08D09951020805E2020E90
:10CCA0000701746F03D00B0199CB74F7530E0B017E
:10CCB000CE6F010ECF6F00014FEC1FF0640E0D011F
:10CCC000B66F000117EC13F055EC48F07BD04FA085
:10CCD00075D04FA440D0036A0B019351470FE96E02
:10CCE000000E0320EA6EEFCF9BFB9BCB9EFB000167
:10CCF00078EC59F0036A0150E8BE03060701682585
:10CD00000B01976F0350070169210B01986F98BFC2
:10CD10000AD0985303E19751FE0805E20701696BB9
:10CD2000686910D00B0198BF05D0985307E197515F
:10CD3000000804E30701696B686B04D00701696BA5
:10CD400097CB68F72F0E0B01DD6F010EDE6F000130
:10CD50007EEC27F033D0036A0B019351470FE96E45
:10CD6000000E0320EA6EEFCF99FB6FC796FB99BFC9
:10CD700007D09951000804E207016F2B0AD00B017C
:10CD800099BF01D006D007016F076F51030801E278
:10CD90006F6B07016F51030803E2040E6F6F03D03E
:10CDA0006F5301E16F6B6F510B01965D08E0490E07
:10CDB000DD6F010EDE6F00017EEC27F00B0100013C
:10CDC00001D000D007016051090A00010DE0060AF8
:10CDD00028E0080A26E0090A54E0030AD8B4DDD0A6
:10CDE0001D0AD8B4FED077D1070E07016C5D0B0188
:10CDF0009B6F0B0E6B6F820E6A6FC80EF66E120E73
:10CE0000F76E000EF86E0C0E9D6F0001D3EC13F060
:10CE10009BCB9CFB1F0E0B019D6F000105EC5AF094
:10CE200066D1070170510A0810E10B0E0B016B6F00
:10CE3000820E6A6FD80EF66E120EF76E000EF86E46
:10CE4000000187EC5BF01CD007010A0E705D0B013E
:10CE50009B6F0B0E6B6F820E6A6FEA0EF66E120EF0
:10CE6000F76E000EF86E0C0E9D6F0001D3EC13F000
:10CE70009BCB9CFB1F0E0B019D6F000105EC5AF034
:10CE800036D14FA261D007015251006E5351036E4B
:10CE9000030E035C04E10052000120E00701020ED2
:10CEA000035C04E10052000133E00701010E035C62
:10CEB00004E1005200012CE00701010E035C05E1D2
:10CEC000010E005C000124E00701010E035C05E196
:10CED000020E005C00011CE0070134D00B0E0B01B8
:10CEE0006B6F820E6A6FFA0EF66E120EF76E000E00
:10CEF000F86E090E9D6F0001D3EC13F072C79BFB17
:10CF00001B0E0B019C6F0001C2EC59F007011AD0F7
:10CF10000B0E0B016B6F820E6A6F060EF66E130E10
:10CF2000F76E000EF86E070E9D6F0001D3EC13F044
:10CF300074C79BFB1B0E0B019C6F0001C2EC59F0E8
:10CF4000070100D028D000010701525324E15351BA
:10CF5000030821E16E5310E10B0E0B016B6F820E83
:10CF60006A6F100EF66E130EF76E000EF86E00016B
:10CF700087EC5BF00FD007010B0E0B016B6F820E7D
:10CF80006A6F220EF66E130EF76E000EF86E000139
:10CF900087EC5BF007010001AAD007017451050D71
:10CFA000F350036A880F016E050E032201C09BFB3C
:10CFB0000B0103C09CFB0B0E6B6F820E6A6F340E6D
:10CFC000F66E130EF76E000EF86E070E9D6F0001E1
:10CFD000D3EC13F09CCBEAFF9BCBE9FFEBEC13F017
:10CFE00086D04FA41DD0800E0701685D0B019B6F9A
:10CFF0000B0E6B6F820E6A6F3E0EF66E130EF76E9F
:10D00000000EF86E0C0E9D6F0001D3EC13F09BCB5D
:10D010009CFB1F0E0B019D6F000105EC5AF05AD0CE
:10D0200007016F51000A000109E0010A16E0030A36
:10D0300023E0010A30E0070A3DE04BD00B0E0B0164
:10D040006B6F820E6A6F4E0EF66E130EF76E000E49
:10D05000F86E000187EC5BF03DD00B0E0B016B6F9F
:10D06000820E6A6F600EF66E130EF76E000EF86E8B
:10D07000000187EC5BF02ED00B0E0B016B6F820E64
:10D080006A6F720EF66E130EF76E000EF86E0001E8
:10D0900087EC5BF01FD00B0E0B016B6F820E6A6F7B
:10D0A000840EF66E130EF76E000EF86E000187EC1C
:10D0B0005BF010D00B0E0B016B6F820E6A6F960E39
:10D0C000F66E130EF76E000EF86E000187EC5BF043
:10D0D00001D000D00CD00B0EEA6E820EE96E200E4D
:10D0E000006E026A110E016EAAEC1BF000D00B0E4E
:10D0F0000B01D86F820ED76F0001F7EC14F00B0113
:10D100003EEF6CF0070160510E0802E081B285D25B
:10D110006051090A00010EE0060A46E0080A44E0F0
:10D120000A0AD8B47BD0030AD8B4B2D01E0AD8B445
:10D13000B9D132D2036A0B019351470FE96E000E49
:10D140000320EA6EEFCF9BFB9BCB9EFB000178ECAC
:10D1500059F0015007016B250B01996F99BF08D059
:10D1600099510D0805E20E0E07016B6F0CD00B01F3
:10D1700099BF03D09951000804E307016B6B03D0FA
:10D180000B0199CB6BF7330E0B01FE6F010EFF6F96
:10D1900000017CEC2EF0640E0D01B66F000117EC5F
:10D1A00013F08FEC55F038D2036A0B019351470FFF
:10D1B000E96E000E0320EA6EEFCF9BFB9BCB9EFB3C
:10D1C000000178EC59F0015007016F250B01996FB0
:10D1D00099BF08D09951130805E2140E07016F6F2B
:10D1E0000CD00B0199BF03D09951000804E307014B
:10D1F0006F6B03D00B0199CB6FF7490E0B01FE6FDC
:10D20000010EFF6F00017CEC2EF0640E0D01B66F75
:10D21000000117EC13F037EC56F0FED1036A0B0156
:10D220009351470FE96E000E0320EA6EEFCF9BFB90
:10D230009BCB9EFB000178EC59F001500701732550
:10D240000B01996F99BF03D09951000804E30701BE
:10D25000736B0DD00B0199BF08D09951060805E2F8
:10D26000060E0701736F03D00B0199CB73F7520EB3
:10D270000B01CE6F010ECF6F00014FEC1FF0640E5B
:10D280000D01B66F000117EC13F0D6EC47F0C4D1D6
:10D290004FA2ADD00B019C6B73C79BFB036A9351EC
:10D2A000470FE96E000E0320EA6EEFCF9DFB9DCB8A
:10D2B0009EFB000178EC59F0036A0150E8BE0306BA
:10D2C0000B019B25976F03509C21986F07015251CA
:10D2D000006E5351036E020E035C04E10052000124
:10D2E00020E00701030E035C04E10052000135E079
:10D2F0000701010E035C04E1005200014AE007014E
:10D30000010E035C05E1010E005C000142E0070133
:10D31000010E035C05E1020E005C00013AE007012A
:10D3200038D00B0198BF05D0985307E197510008FA
:10D3300004E30701736B10D00B0198BF0AD0985318
:10D3400003E19751AF0805E2AF0E0701736F04D0F8
:10D350000B0197CB73F7070139D00B0198BF05D0AC
:10D36000985307E19751000804E30701736B10D04D
:10D370000B0198BF0AD0985303E19751640805E266
:10D38000640E0701736F04D00B0197CB73F707018D
:10D390001DD00B0198BF05D0985308E1975108089C
:10D3A00005E3080E0701736F10D00B0198BF0AD078
:10D3B000985303E197511F0805E21F0E0701736F91
:10D3C00004D00B0197CB73F7070100D0520E0B016D
:10D3D000FE6F010EFF6F00017CEC2EF0640E0D015C
:10D3E000B66F000117EC13F0D6EC47F05AD04FA0FF
:10D3F00056D00B019C6B76C79BFB036A9351470F7A
:10D40000E96E000E0320EA6EEFCF9DFB9DCB9EFBE5
:10D41000000178EC59F0036A0150E8BE03060B01E5
:10D420009B25976F03509C21986F07015251006E06
:10D430005351036E030E035C04E10052000102E04D
:10D4400007012BD00B0198BF05D0985308E19751E5
:10D450000D0805E30E0E0701766F10D00B0198BF83
:10D460000AD0985303E197511B0805E21B0E0701F0
:10D47000766F04D00B0197CB76F70701590E0B019D
:10D48000FE6F010EFF6F00017CEC2EF0640E0D01AB
:10D49000B66F000117EC13F0070100D0000137EC64
:10D4A00057F0BAD04FA442D04FA03FD0036A0B012F
:10D4B0009351470FE96E000E0320EA6EEFCF9BFBFE
:10D4C0009BCB9EFB000178EC59F0036A0150E8BE4B
:10D4D0000306070166250B01976F035007016721BB
:10D4E0000B01986F98BF0AD0985303E19751FE083B
:10D4F00005E20701676B666910D00B0198BF05D084
:10D50000985307E19751000804E30701676B666BC6
:10D5100004D00701676B97CB66F72B0E0B01DD6F0D
:10D52000010EDE6F00017EEC27F033D0036A0B01A1
:10D530009351470FE96E000E0320EA6EEFCF99FB7F
:10D540006EC796FB99BF07D09951000804E2070106
:10D550006E2B0AD00B0199BF01D006D007016E07D0
:10D560006E51010801E26E6B07016E51010803E282
:10D57000020E6E6F03D06E5301E16E6B6E510B01A4
:10D58000965D08E0470EDD6F010EDE6F00017EEC58
:10D5900027F00B01000140D0070151B33BD051B53A
:10D5A00039D0036A0B019351470FE96E000E032037
:10D5B000EA6EEFCF9BFB9BCB9EFB000178EC59F012
:10D5C0000150070171250B01996F99BF08D099513E
:10D5D0000E0805E20F0E0701716F0CD00B0199BF09
:10D5E00003D09951000804E30701716B03D00B01CC
:10D5F00099CB71F7270E0B01FE6F010EFF6F000133
:10D600007CEC2EF0640E0D01B66F000117EC13F0E8
:10D61000B4EC45F0000100D007016051090A000197
:10D620000DE0060A28E0080A26E0090A41E0030A9C
:10D63000D8B485D01D0AD8B49FD0F6D0070E070104
:10D640006B5D0B019B6F0B0E6B6F820E6A6FA80EEA
:10D65000F66E130EF76E000EF86E0D0E9D6F000144
:10D66000D3EC13F09BCB9CFB1F0E0B019D6F0001B5
:10D6700005EC5AF0F8D00A0E07016F5D0B019B6FA5
:10D680000B0E6B6F820E6A6FB80EF66E130EF76E8E
:10D69000000EF86E0C0E9D6F0001D3EC13F09BCBC7
:10D6A0009CFB1F0E0B019D6F000105EC5AF0DBD0B7
:10D6B0004FA219D00B0E0B016B6F820E6A6FC80E52
:10D6C000F66E130EF76E000EF86E090E9D6F0001D8
:10D6D000D3EC13F073C79BFB1B0E0B019C6F000177
:10D6E000C2EC59F029D00701525327E153510308E6
:10D6F00024E10E0E765D060DF350036AD80F016E1D
:10D70000060E032201C09BFB0B0103C09CFB0B0E0A
:10D710006B6F820E6A6FD40EF66E130EF76E000EEC
:10D72000F86E0A0E9D6F0001D3EC13F09CCBEAFF5C
:10D730009BCBE9FFEBEC13F00701000194D0030E43
:10D740000701735D0B019B6F0B0E6B6F820E6A6F8F
:10D75000E20EF66E130EF76E000EF86E090E9D6F58
:10D760000001D3EC13F09BCB9CFB1F0E0B019D6FB4
:10D77000000105EC5AF077D04FA41DD0800E0701B0
:10D78000665D0B019B6F0B0E6B6F820E6A6FEE0E68
:10D79000F66E130EF76E000EF86E0C0E9D6F000104
:10D7A000D3EC13F09BCB9CFB1F0E0B019D6F000174
:10D7B00005EC5AF038D007016E51000A000105E06F
:10D7C000010A12E0030A1FE02DD00B0E0B016B6F54
:10D7D000820E6A6FFE0EF66E130EF76E000EF86E76
:10D7E000000187EC5BF01FD00B0E0B016B6F820EFC
:10D7F0006A6F100EF66E140EF76E000EF86E0001D2
:10D8000087EC5BF010D00B0E0B016B6F820E6A6F12
:10D81000220EF66E140EF76E000EF86E000187EC05
:10D820005BF001D000D01FD0070151B31AD051B521
:10D8300018D00B0E0B016B6F820E6A6F340EF66EF2
:10D84000140EF76E000EF86E0C0E9D6F0001D3ECF7
:10D8500013F071C79BFB1B0E0B019C6F0001C2EC08
:10D8600059F0000100D00B0E0B01D86F820ED76F5C
:10D870000001F7EC14F00B0101D00B01036A935186
:10D880003F0FE96E000E0320EA6EEF6A932BAAEFBA
:10D890005BF02BEF7BF0040E936F93510708D8A039
:10D8A0002BEF7BF0036A9351470FE96E000E0320C4
:10D8B000EA6EEF52D8B420EF7BF0000141EC1FF08C
:10D8C0000701482D51D00B019351040A000101E0DA
:10D8D00046D0010E07014D6F4B513F0803E149C788
:10D8E0004BF718D0036A0B019351470FE96E000EF6
:10D8F0000320EA6EEFBE07D0EF50000804E20701F4
:10D900004B2B08D00B0107014B5302E04B0702D011
:10D910000E0E4B6F4B510E0801E24B6B4B510D0D30
:10D92000F350036A150F016E060E032201C09BFB24
:10D930000B0103C09CFB0B0E6B6F820E6A6F03C062
:10D94000EAFF01C0E9FF0001EBEC13F00B0E0B0145
:10D95000D86F820ED76F0001F7EC14F002D02CEFD5
:10D960007BF01FEF7BF00701040E0B01935DFC0FB2
:10D97000D8B020EF7BF0040F000141EF7BF00701EE
:10D9800060510E0802E081B203D36051090A000120
:10D990000EE0060A46E0080A44E0090AD8B47BD043
:10D9A000030AD8B456D21D0AD8B48DD2EFD2036A76
:10D9B0000B019351470FE96E000E0320EA6EEFCF83
:10D9C0009BFB9BCB9EFB000178EC59F001500701BB
:10D9D0006A250B01996F99BF08D099510D0805E28E
:10D9E0000E0E07016A6F0CD00B0199BF03D099513D
:10D9F000000804E307016A6B03D00B0199CB6AF7B7
:10DA0000400E0B01FE6F010EFF6F00017CEC2EF04B
:10DA1000640E0D01B66F000117EC13F0AEEC55F07B
:10DA2000B6D2036A0B019351470FE96E000E032033
:10DA3000EA6EEFCF9BFB9BCB9EFB000178EC59F08D
:10DA4000015007016E250B01996F99BF08D09951BC
:10DA5000130805E2140E07016E6F0CD00B0199BF7D
:10DA600003D09951000804E307016E6B03D00B014A
:10DA700099CB6EF7470E0B01FE6F010EFF6F000191
:10DA80007CEC2EF0640E0D01B66F000117EC13F064
:10DA900056EC56F07CD20701525304E1535103086F
:10DAA000D8B453D14FA2ADD00B019C6B72C79BFB76
:10DAB000036A9351470FE96E000E0320EA6EEFCF21
:10DAC0009DFB9DCB9EFB000178EC59F0036A015051
:10DAD000E8BE03060B019B25976F03509C21986FAE
:10DAE00007015251006E5351036E020E035C04E1B4
:10DAF0000052000119E00701010E035C04E100522D
:10DB000000012FE00701010E035C05E1010E005C3E
:10DB1000000127E00701010E035C05E1020E005C35
:10DB200000011FE007011ED00B0198BF05D09853DC
:10DB300008E19751010805E3010E0701726F10D04B
:10DB40000B0198BF0AD0985303E197515F0805E293
:10DB50005F0E0701726F04D00B0197CB72F70701BC
:10DB60003ED00701725180081DE20B0198BF05D01D
:10DB7000985308E19751010805E3FD0E0701726F04
:10DB800010D00B0198BF0AD0985303E19751FD08BC
:10DB900005E2FD0E0701726F04D00B0197CB72F7FF
:10DBA00007011CD00B0198BF05D0985308E197518D
:10DBB000010805E3010E0701726F10D00B0198BF39
:10DBC0000AD0985303E19751FD0805E2FD0E0701C5
:10DBD000726F04D00B0197CB72F7070100D0500E83
:10DBE0000B01FE6F010EFF6F00017CEC2EF0640E46
:10DBF0000D01B66F000117EC13F00DEC47F0A3D048
:10DC000007010B019C6B75C79BFB036A9351470F80
:10DC1000E96E000E0320EA6EEFCF9DFB9DCB9EFBCD
:10DC2000000178EC59F0036A0150E8BE03060B01CD
:10DC30009B25976F03509C21986F07015251006EEE
:10DC40005351036E020E035C04E10052000119E01F
:10DC50000701010E035C04E10052000148E00701E6
:10DC6000010E035C05E1010E005C000140E00701CC
:10DC7000010E035C05E1020E005C000138E00701C3
:10DC800036D007017551800819E20B0198BF05D005
:10DC9000985307E19751010804E3070175690DD016
:10DCA0000B0198BF07D09851000804E2070175697D
:10DCB00004D00B0197CB75F7070118D00B0198BF63
:10DCC00005D0985307E19751000804E30701756BED
:10DCD0000DD00B0198BF07D09851000804E207014E
:10DCE000756904D00B0197CB75F707011CD00B01A8
:10DCF00098BF05D0985307E19751000804E3070146
:10DD0000756B10D00B0198BF0AD0985303E197515F
:10DD10007F0805E27F0E0701756F04D00B0197CBDA
:10DD200075F7070100D0540E0B01FE6F010EFF6F57
:10DD300000017CEC2EF0640E0D01B66F000117ECB3
:10DD400013F075EC56F084D007014FA247D00B01B9
:10DD50009C6B74C79BFB036A9351470FE96E000EDF
:10DD60000320EA6EEFCF9DFB9DCB9EFB000178EC7C
:10DD700059F0036A0150E8BE03060B019B25976F1B
:10DD800003509C21986F98BF05D0985307E1975195
:10DD9000000804E30701746B0FD00B0198BF0AD091
:10DDA000985303E19751100805E2100E0701746FB4
:10DDB00003D00B0197CB74F7530E0B01FE6F010ECE
:10DDC000FF6F00017CEC2EF0640E0D01B66F0001B8
:10DDD00017EC13F055EC48F03BD00701036A0B0138
:10DDE0009351470FE96E000E0320EA6EEFCF99FBC7
:10DDF00007016D5314E10B0199BF0FD09951000831
:10DE00000CE2010E07016D6F550E0B01FE6F010E46
:10DE1000FF6F00017CEC2EF00B0112D007010B010B
:10DE200099BF03D0995100080BE307016D6B560EA3
:10DE30000B01FE6F010EFF6F00017CEC2EF00B0159
:10DE4000640E0D01B66F000117EC13F0BDEC56F037
:10DE50009ED0036A0B019351470FE96E000E032019
:10DE6000EA6EEFCF9BFB9BCB9EFB000178EC59F059
:10DE70000150070172250B01996F99BF03D0995189
:10DE8000000804E30701726B0DD00B0199BF08D0A5
:10DE900099513C0805E23C0E0701726F03D00B015B
:10DEA00099CB72F7500E0B01CE6F010ECF6F0001B0
:10DEB0004FEC1FF0640E0D01B66F000117EC13F06C
:10DEC0000DEC47F064D0036A0B019351470FE96EE4
:10DED000000E0320EA6EEFCF99FB4FA42DD04FA088
:10DEE0002AD065C796FB99BF07D09951000804E274
:10DEF0000701652B0AD00B0199BF01D006D007019D
:10DF000065076551040801E2656B07016551040866
:10DF100003E2040E656F03D0655301E1656B655143
:10DF20000B01965D08E03B0EDD6F010EDE6F000118
:10DF30007EEC27F00B0128D007016D5314E10B0193
:10DF400099BF0FD0995100080CE2010E07016D6FC7
:10DF5000410E0B01DD6F010EDE6F00017EEC27F03C
:10DF60000B0112D007010B0199BF03D09951000892
:10DF70000BE307016D6B420E0B01DD6F010EDE6FCF
:10DF800000017EEC27F00B01000101D000D0070159
:10DF90006051090A00010DE0060A28E0080A26E09F
:10DFA000090A54E0030AD8B4E7D01D0AD8B401D155
:10DFB00048D1070E07016A5D0B019B6F0B0E6B6F5B
:10DFC000820E6A6F440EF66E140EF76E000EF86E37
:10DFD0000C0E9D6F0001D3EC13F09BCB9CFB1F0E2E
:10DFE0000B019D6F000105EC5AF037D107016E510E
:10DFF0000A0810E10B0E0B016B6F820E6A6F540E54
:10E00000F66E140EF76E000EF86E000187EC5BF0F2
:10E010001CD007010A0E6E5D0B019B6F0B0E6B6F20
:10E02000820E6A6F660EF66E140EF76E000EF86EB4
:10E030000C0E9D6F0001D3EC13F09BCB9CFB1F0ECD
:10E040000B019D6F000105EC5AF007D107015253F7
:10E0500003E15351030835E04FA219D00B0E0B0119
:10E060006B6F820E6A6F760EF66E140EF76E000EF0
:10E07000F86E0B0E9D6F0001D3EC13F072C79BFB83
:10E080001B0E0B019C6F0001C2EC59F018D00B0E57
:10E090000B016B6F820E6A6F840EF66E140EF76EB4
:10E0A000000EF86E070E9D6F0001D3EC13F075C7DC
:10E0B0009BFB1B0E0B019C6F0001C2EC59F05BD067
:10E0C00007014FA238D07451100810E10B0E0B015C
:10E0D0006B6F820E6A6F8E0EF66E140EF76E000E68
:10E0E000F86E000187EC5BF024D007017451050D38
:10E0F000F350140F0B01996F0B0E6B6F820E6A6F4A
:10E100009A0EF66E140EF76E000EF86E080E9D6FE6
:10E110000001D3EC13F099CB9CFB110E0B019D6F0A
:10E12000000105EC5AF0200E0B01A66F0001C3ECB4
:10E1300013F021D007016D5310E10B0E0B016B6F33
:10E14000820E6A6FA80EF66E140EF76E000EF86E51
:10E15000000187EC5BF00FD007010B0E0B016B6F1A
:10E16000820E6A6FBA0EF66E140EF76E000EF86E1F
:10E17000000187EC5BF071D01E0E0701725D0B0190
:10E180009B6F0B0E6B6F820E6A6FCC0EF66E140EC9
:10E19000F76E000EF86E0B0E9D6F0001D3EC13F0BE
:10E1A0009BCB9CFB1F0E0B019D6F000105EC5AF0F1
:10E1B00054D04FA424D007016551060DF350036AD3
:10E1C000640F016E050E032201C09BFB0B0103C00F
:10E1D0009CFB0B0E6B6F820E6A6FDA0EF66E140EDE
:10E1E000F76E000EF86E0C0E9D6F0001D3EC13F06D
:10E1F0009CCBEAFF9BCBE9FFEBEC13F021D00701AE
:10E200006D5310E10B0E0B016B6F820E6A6FEA0EFD
:10E21000F66E140EF76E000EF86E000187EC5BF0E0
:10E220000FD007010B0E0B016B6F820E6A6FFC0E95
:10E23000F66E140EF76E000EF86E000187EC5BF0C0
:10E240000CD00B0EEA6E820EE96E200E006E026A92
:10E25000110E016EAAEC1BF000D00B0E0B01D86F53
:10E26000820ED76F0001F7EC14F00B0120EF7BF06A
:10E27000070160510E0802E081B2B4D14FB404D05E
:10E2800051A5ACD14FA0AAD151A336D0036A0B013E
:10E290009351470FE96E000E0320EA6EEFCF9BFB10
:10E2A0009BCB9EFB000178EC59F0015007016825DB
:10E2B0000B01996F99BF09D099513C0806E20701FB
:10E2C000696B3C0E686F0ED00B0199BF03D099515A
:10E2D000000804E30701696B686B04D00701696BF0
:10E2E00099CB68F72F0E0B01CE6F010ECF6F000197
:10E2F0004FEC1FF06CD1070151A579D04FA076D01B
:10E300004FA436D0036A0B019351470FE96E000EFC
:10E310000320EA6EEFCF99FB75C796FB99BF07D034
:10E320009951000804E20701752B0AD00B0199BF2F
:10E3300001D006D0070175077551020801E2756B1F
:10E3400007017551020803E2030E756F03D0755380
:10E3500001E1756B75510B01965D08E0540EDD6FA0
:10E36000010EDE6F00017EEC27F00B013ED00701AD
:10E370000B019C6B6AC79BFB036A9351470FE96EC5
:10E38000000E0320EA6EEFCF9DFB9DCB9EFB0001AC
:10E3900078EC59F0036A0150E8BE03060B019B2597
:10E3A000976F03509C21986F98BF09D0985303E151
:10E3B0009751FE0804E207016A690ED00B0198BF6D
:10E3C00005D0985307E19751000804E307016A6BF1
:10E3D00003D00B0197CB6AF7400E0B01DD6F010EE6
:10E3E000DE6F00017EEC27F00B010701F1D0036A1C
:10E3F0000B019351470FE96E000E0320EA6EEFCF39
:10E400009BFB9BCB9EFB000178EC59F0036A01500B
:10E41000E8BE0306070168250B01976F035007014B
:10E4200069210B01986F070160510E08D8A4A7D08D
:10E430005251006E5351036E020E035C04E1005210
:10E44000000122E00701030E035C04E10052000119
:10E450003FE00701010E035C05E100520001D8B462
:10E460006AD00701010E035C06E1010E005C0001A9
:10E47000D8B461D00701010E035C05E1020E005C17
:10E48000000159E0070157D00B0198BF05D0985300
:10E4900008E19751000805E30701696B686B17D025
:10E4A0000B0198BF0FD0985101080CE2FF0A03E15D
:10E4B00097517E0807E2020E0701696F7F0E686FB1
:10E4C00006D00B0198CB69F797CB68F7070156D0B8
:10E4D000070161A304D00B019A812BD00701695178
:10E4E000EF0816E2FF0A03E16851000811E20B0190
:10E4F00098AF02D007010CD0985306E1975100085D
:10E50000D8A002D0070104D007016969686911D059
:10E5100069510F080AE30B0198BF03D0070105D02A
:10E520000B010701696B686B04D098CB69F797CB37
:10E5300068F7070123D00B0198BF05D0985308E175
:10E540009751000805E30701696B686B16D00B0152
:10E5500098BF0ED0985100080BE2FF0A03E19751D3
:10E56000FE0806E2010E0701696F686906D00B011B
:10E5700098CB69F797CB68F7070100D01ED00B0145
:10E5800098BF05D0985308E19751000805E30701AB
:10E59000696B686B12D00B0198BF0AD0985303E1E6
:10E5A0009751FE0805E20701696B686906D00B0107
:10E5B00098CB69F797CB68F707010B019AB108D0A0
:10E5C0002F0EFE6F010EFF6F00017CEC2EF00B0191
:10E5D000640E0D01B66F000117EC13F00001BEECE4
:10E5E00041F0070151A322D01E0E685D006E000E9F
:10E5F0006959036E00C09BFB0B010B0E6B6F820E03
:10E600006A6F0E0EF66E150EF76E000EF86E0C0E9B
:10E610009D6F0001D3EC13F09BCB9CFB1F0E0B01F5
:10E620009D6F000105EC5AF0F0D1070151A569D0AA
:10E630004FA44AD07551000A000107E0010A14E016
:10E64000030A21E0010A2EE03CD00B0E0B016B6F98
:10E65000820E6A6F1E0EF66E150EF76E000EF86EC5
:10E66000000187EC5BF02ED00B0E0B016B6F820E5E
:10E670006A6F300EF66E150EF76E000EF86E000122
:10E6800087EC5BF01FD00B0E0B016B6F820E6A6F75
:10E69000420EF66E150EF76E000EF86E000187EC56
:10E6A0005BF010D00B0E0B016B6F820E6A6F540E75
:10E6B000F66E150EF76E000EF86E000187EC5BF03B
:10E6C00001D000D01CD00701800E6A5D0B019B6F4A
:10E6D0000B0E6B6F820E6A6F660EF66E150EF76E7E
:10E6E000000EF86E0C0E9D6F0001D3EC13F09BCB67
:10E6F0009CFB1F0E0B019D6F000105EC5AF085D1AC
:10E70000070160510E08D8A420D15251006E535118
:10E71000036E020E035C04E10052000124E00701D5
:10E72000030E035C05E100520001D8B48BD0070151
:10E73000010E035C05E100520001D8B49CD0070132
:10E74000010E035C06E1010E005C0001D8B493D019
:10E750000701010E035C06E1020E005C0001D8B463
:10E760008AD0070189D0070168513F0803E1692D6C
:10E7700001D005D0685140081BE1692D19D00B0E5E
:10E780000B016B6F820E6A6F760EF66E150EF76ECA
:10E79000000EF86E0C0E9D6F0001D3EC13F00B0110
:10E7A0009C6B1F0E9D6F000105EC5AF04AD00701CB
:10E7B0006951010826E303E168513F0822E33F0E57
:10E7C000685D0B019B6F010E070169590B019C6F7E
:10E7D0000B0E6B6F820E6A6F860EF66E150EF76E5D
:10E7E000000EF86E0C0E9D6F0001D3EC13F0100EAE
:10E7F000E96E9CCB9EFB9BCB9DFB0CEC5BF021D090
:10E800000701400E685D0B019B6F010E07016959FE
:10E810000B019C6F0B0E6B6F820E6A6F960EF66E7D
:10E82000150EF76E000EF86E0C0E9D6F0001D3EC06
:10E8300013F0100EE96E9CCB9EFB9BCB9DFB0CEC6A
:10E840005BF081D00B0E0B016B6F820E6A6FA60E10
:10E85000F66E150EF76E000EF86E0B0E9D6F000132
:10E86000D3EC13F0100EE96E69C79EFB68C79DFBE1
:10E870000CEC5BF068D00701683D02D0695304E0FE
:10E8800068531BE1692D19D00B0E0B016B6F820EC3
:10E890006A6FB60EF66E150EF76E000EF86E0C0E61
:10E8A0009D6F0001D3EC13F00B019C6B1F0E9D6F4D
:10E8B000000105EC5AF046D007016951000822E337
:10E8C000FF0E685D0B019B6F000E070169590B017C
:10E8D0009C6F0B0E6B6F820E6A6FC60EF66E150E76
:10E8E000F76E000EF86E0C0E9D6F0001D3EC13F066
:10E8F000100EE96E9CCB9EFB9BCB9DFB0CEC5BF062
:10E9000021D00701000E685D0B019B6F010E07010E
:10E9100069590B019C6F0B0E6B6F820E6A6FD60EDE
:10E92000F66E150EF76E000EF86E0C0E9D6F000160
:10E93000D3EC13F0100EE96E9CCB9EFB9BCB9DFBA2
:10E940000CEC5BF000D061D0070168517F0802E158
:10E95000695305E0685180081BE1695319E10B0E0A
:10E960000B016B6F820E6A6FE60EF66E150EF76E78
:10E97000000EF86E0C0E9D6F0001D3EC13F00B012E
:10E980009C6B1F0E9D6F000105EC5AF03ED00701F5
:10E99000695320E168517F081DE37F0E685D0B011C
:10E9A0009B6F0B0E6B6F820E6A6FF60EF66E150E76
:10E9B000F76E000EF86E0C0E9D6F0001D3EC13F095
:10E9C0009BCB9CFB1F0E0B019D6F000105EC5AF0C9
:10E9D0001CD00701800E685D0B019B6F0B0E6B6FE7
:10E9E000820E6A6F060EF66E160EF76E000EF86E49
:10E9F0000C0E9D6F0001D3EC13F09BCB9CFB1F0E04
:10EA00000B019D6F000105EC5AF00B0E0B01D86F46
:10EA1000820ED76F0001F7EC14F00B0120EF7BF0B2
:10EA2000070160510E0802E081B2A0D14FB404D0BA
:10EA300051A598D14FA096D151A336D0036A0B01AE
:10EA40009351470FE96E000E0320EA6EEFCF9BFB58
:10EA50009BCB9EFB000178EC59F001500701662525
:10EA60000B01996F99BF09D099513C0806E2070143
:10EA7000676B3C0E666F0ED00B0199BF03D09951A6
:10EA8000000804E30701676B666B04D00701676B3E
:10EA900099CB66F72B0E0B01CE6F010ECF6F0001E5
:10EAA0004FEC1FF058D1070151A565D0036A0B0147
:10EAB0009351470FE96E000E0320EA6EEFCF99FBEA
:10EAC0004FA057D04FA42BD073C796FB99BF07D048
:10EAD0009951000804E20701732B0AD00B0199BF7A
:10EAE00001D006D0070173077351010801E2736B6F
:10EAF00007017351010803E2020E736F03D07353D1
:10EB000001E1736B73510B01965D08E0520EDD6FEE
:10EB1000010EDE6F00017EEC27F00B012AD06BC7DF
:10EB200096FB99BF07D09951000804E207016B2BAF
:10EB30000AD00B0199BF01D006D007016B076B51BA
:10EB4000010801E26B6B07016B51010803E2020E41
:10EB50006B6F03D06B5301E16B6B6B510B01965DD7
:10EB600008E0330EDD6F010EDE6F00017EEC27F052
:10EB70000B01F2D00701036A0B019351470FE96EB5
:10EB8000000E0320EA6EEFCF9BFB9BCB9EFB0001A8
:10EB900078EC59F0036A0150E8BE030607016625C8
:10EBA0000B01976F0350070167210B01986F070155
:10EBB00060510E08D8A4A7D05251006E5351036E75
:10EBC000020E035C04E10052000122E00701030E83
:10EBD000035C04E1005200013FE00701010E035C09
:10EBE00005E100520001D8B46AD00701010E035CB0
:10EBF00006E1010E005C0001D8B461D00701010EEE
:10EC0000035C05E1020E005C000159E0070157D0EA
:10EC10000B0198BF05D0985308E19751000805E310
:10EC20000701676B666B17D00B0198BF0FD0985127
:10EC300001080CE2FF0A03E197517E0807E2020E89
:10EC40000701676F7F0E666F06D00B0198CB67F7E1
:10EC500097CB66F7070156D0070161A304D00B01DB
:10EC60009A812BD007016751EF0816E2FF0A03E1F2
:10EC70006651000811E20B0198AF02D007010CD0D9
:10EC8000985306E197510008D8A002D0070104D09C
:10EC900007016769666911D067510F080AE30B0124
:10ECA00098BF03D0070105D00B010701676B666BA6
:10ECB00004D098CB67F797CB66F7070123D00B01F9
:10ECC00098BF05D0985308E19751000805E3070164
:10ECD000676B666B16D00B0198BF0ED09851000879
:10ECE0000BE2FF0A03E19751FE0806E2010E07015D
:10ECF000676F666906D00B0198CB67F797CB66F70D
:10ED0000070100D01ED00B0198BF05D0985308E131
:10ED10009751000805E30701676B666B12D00B0182
:10ED200098BF0AD0985303E19751FE0805E2070106
:10ED3000676B666906D00B0198CB67F797CB66F7D0
:10ED400007010B019AB108D02B0EFE6F010EFF6F69
:10ED500000017CEC2EF00B01640E0D01B66F00017A
:10ED600017EC13F0000170EC40F0070151A322D022
:10ED70001E0E665D006E000E6759036E00C09BFBA1
:10ED80000B010B0E6B6F820E6A6F160EF66E160E6F
:10ED9000F76E000EF86E0B0E9D6F0001D3EC13F0B2
:10EDA0009BCB9CFB1F0E0B019D6F000105EC5AF0E5
:10EDB000FBD1070151A574D04FA439D07351000A7B
:10EDC000000105E0010A12E0030A1FE02DD00B0E3E
:10EDD0000B016B6F820E6A6F240EF66E160EF76EC5
:10EDE000000EF86E000187EC5BF01FD00B0E0B01DC
:10EDF0006B6F820E6A6F360EF66E160EF76E000E91
:10EE0000F86E000187EC5BF010D00B0E0B016B6FFE
:10EE1000820E6A6F480EF66E160EF76E000EF86ED2
:10EE2000000187EC5BF001D000D038D007016B51B6
:10EE3000000A000105E0010A12E0030A1FE02DD0DC
:10EE40000B0E0B016B6F820E6A6F5A0EF66E160E6A
:10EE5000F76E000EF86E000187EC5BF01FD00B0E12
:10EE60000B016B6F820E6A6F6C0EF66E160EF76EEC
:10EE7000000EF86E000187EC5BF010D00B0E0B015A
:10EE80006B6F820E6A6F7E0EF66E160EF76E000EB8
:10EE9000F86E000187EC5BF001D000D085D107014E
:10EEA00060510E08D8A420D15251006E5351036E08
:10EEB000020E035C04E10052000124E00701030E8E
:10EEC000035C05E100520001D8B48BD00701010EAC
:10EED000035C05E100520001D8B49CD00701010E8B
:10EEE000035C06E1010E005C0001D8B493D0070179
:10EEF000010E035C06E1020E005C0001D8B48AD06A
:10EF0000070189D0070166513F0803E1672D01D051
:10EF100005D0665140081BE1672D19D00B0E0B017F
:10EF20006B6F820E6A6F900EF66E160EF76E000E05
:10EF3000F86E0C0E9D6F0001D3EC13F00B019C6B6F
:10EF40001F0E9D6F000105EC5AF04AD00701675172
:10EF5000010826E303E166513F0822E33F0E665DA8
:10EF60000B019B6F010E070167590B019C6F0B0E84
:10EF70006B6F820E6A6FA00EF66E160EF76E000EA5
:10EF8000F86E0C0E9D6F0001D3EC13F0100EE96EBD
:10EF90009CCB9EFB9BCB9DFB0CEC5BF021D0070137
:10EFA000400E665D0B019B6F010E070167590B0157
:10EFB0009C6F0B0E6B6F820E6A6FB00EF66E160EA4
:10EFC000F76E000EF86E0C0E9D6F0001D3EC13F07F
:10EFD000100EE96E9CCB9EFB9BCB9DFB0CEC5BF07B
:10EFE00081D00B0E0B016B6F820E6A6FC00EF66E36
:10EFF000160EF76E000EF86E0B0E9D6F0001D3EC2F
:10F0000013F0100EE96E67C79EFB66C79DFB0CEC04
:10F010005BF068D00701663D02D0675304E0665399
:10F020001BE1672D19D00B0E0B016B6F820E6A6FFF
:10F03000D00EF66E160EF76E000EF86E0C0E9D6F6B
:10F040000001D3EC13F00B019C6B1F0E9D6F0001B0
:10F0500005EC5AF046D007016751000822E3FF0E85
:10F06000665D0B019B6F000E070167590B019C6FDA
:10F070000B0E6B6F820E6A6FE00EF66E160EF76E59
:10F08000000EF86E0C0E9D6F0001D3EC13F0100E05
:10F09000E96E9CCB9EFB9BCB9DFB0CEC5BF021D0E7
:10F0A0000701000E665D0B019B6F010E070167599A
:10F0B0000B019C6F0B0E6B6F820E6A6FF00EF66E7B
:10F0C000160EF76E000EF86E0C0E9D6F0001D3EC5D
:10F0D00013F0100EE96E9CCB9EFB9BCB9DFB0CECC2
:10F0E0005BF000D061D0070166517F0802E16753F1
:10F0F00005E0665180081BE1675319E10B0E0B0117
:10F100006B6F820E6A6F000EF66E170EF76E000EB2
:10F11000F86E0C0E9D6F0001D3EC13F00B019C6B8D
:10F120001F0E9D6F000105EC5AF03ED0070167539A
:10F1300020E166517F081DE37F0E665D0B019B6F2A
:10F140000B0E6B6F820E6A6F100EF66E170EF76E57
:10F15000000EF86E0C0E9D6F0001D3EC13F09BCBEC
:10F160009CFB1F0E0B019D6F000105EC5AF01CD09B
:10F170000701800E665D0B019B6F0B0E6B6F820E9D
:10F180006A6F200EF66E170EF76E000EF86E0C0EFC
:10F190009D6F0001D3EC13F09BCB9CFB1F0E0B016A
:10F1A0009D6F000105EC5AF00B0E0B01D86F820E1B
:10F1B000D76F0001F7EC14F00B0142D20701605148
:10F1C0000E0802E081B26CD160510E0A000110E01D
:10F1D000070AD8B48DD0060AD8B48AD0080AD8B4A1
:10F1E00087D00A0AD8B4BED01D0AD8B4F2D056D1FE
:10F1F000036A0B019351470FE96E000E0320EA6E7C
:10F20000EFCF9BFB9BCB9EFB000178EC59F00150AC
:10F21000070171250B01996F07015251006E53517F
:10F22000036E030E035C04E10052000120E00701BD
:10F23000020E035C04E10052000131E00701010EFF
:10F24000035C04E1005200012AE00701010E035CA7
:10F2500005E1010E005C000122E00701010E035CE4
:10F2600005E1020E005C00011AE0070118D00B0155
:10F2700099BF08D099511E0805E21F0E0701716F52
:10F280000DD00B0199BF03D09951000804E3070189
:10F29000716B04D00B0199CB71F7070118D00B01EA
:10F2A00099BF08D099513E0805E23F0E0701716FE2
:10F2B0000DD00B0199BF03D09951000804E3070159
:10F2C000716B04D00B0199CB71F7070100D0270EA9
:10F2D0000B01FE6F010EFF6F00017CEC2EF0640E3F
:10F2E0000D01B66F000117EC13F0CDEC55F0D7D03F
:10F2F000036A0B019351470FE96E000E0320EA6E7B
:10F30000EFCF9BFB9BCB9EFB000178EC59F00150AB
:10F31000070171250B01996F99BF08D099510E080B
:10F3200005E20F0E0701716F0CD00B0199BF03D0DE
:10F330009951000804E30701716B03D00B0199CBCD
:10F3400071F7270E0B01FE6F010EFF6F00017CECC1
:10F350002EF0640E0D01B66F000117EC13F0CDEC2A
:10F3600055F09DD0036A0B019351470FE96E000ED3
:10F370000320EA6EEFCF9BFB9BCB9EFB000178EC5A
:10F3800059F00150070171250B01996F99518008BF
:10F3900005E3800E0701716F0BD00B0199518E08A8
:10F3A00005E28E0E0701716F03D00B0199CB71F747
:10F3B000270E0B01CE6F010ECF6F00014FEC1FF037
:10F3C000640E0D01B66F000117EC13F0B4EC45F0BC
:10F3D00066D04FA060D0036A0B019351470FE96ECE
:10F3E000000E0320EA6EEFCF99FB4FA42BD074C719
:10F3F00096FB99BF07D09951000804E20701742BCE
:10F400000AD00B0199BF01D006D0070174077451CF
:10F41000010801E2746B07017451010803E2020E56
:10F42000746F03D0745301E1746B74510B01965DDA
:10F4300008E0530EDD6F010EDE6F00017EEC27F059
:10F440000B012AD071C796FB99BF07D099510008CC
:10F4500004E20701712B0AD00B0199BF01D006D03D
:10F46000070171077151010801E2716B07017151C8
:10F47000010803E2020E716F03D0715301E1716B59
:10F4800071510B01965D08E0270EDD6F010EDE6FF6
:10F4900000017EEC27F00B01000101D000D0070134
:10F4A00060510E0A00010BE0070A09E0060A07E0B6
:10F4B000080A05E00A0A1CE01D0A37E0AAD00B0E74
:10F4C0000B016B6F820E6A6F300EF66E170EF76EC1
:10F4D000000EF86E0C0E9D6F0001D3EC13F071C797
:10F4E0009BFB1B0E0B019C6F0001C2EC59F09DD0E1
:10F4F000800E0701715D0B019B6F0B0E6B6F820E0F
:10F500006A6F400EF66E170EF76E000EF86E090E5B
:10F510009D6F0001D3EC13F09BCB9CFB1F0E0B01E6
:10F520009D6F000105EC5AF080D04FA439D007013F
:10F530007451000A000105E0010A12E0030A1FE00D
:10F540002DD00B0E0B016B6F820E6A6F4C0EF66E98
:10F55000170EF76E000EF86E000187EC5BF01FD0FF
:10F560000B0E0B016B6F820E6A6F5E0EF66E170E3E
:10F57000F76E000EF86E000187EC5BF010D00B0EFA
:10F580000B016B6F820E6A6F700EF66E170EF76EC0
:10F59000000EF86E000187EC5BF001D000D038D08F
:10F5A00007017151000A000105E0010A12E0030A97
:10F5B0001FE02DD00B0E0B016B6F820E6A6F820E57
:10F5C000F66E170EF76E000EF86E000187EC5BF01A
:10F5D0001FD00B0E0B016B6F820E6A6F940EF66ECE
:10F5E000170EF76E000EF86E000187EC5BF010D07E
:10F5F0000B0E0B016B6F820E6A6FA60EF66E170E66
:10F60000F76E000EF86E000187EC5BF001D000D0C1
:10F610000CD00B0EEA6E820EE96E200E006E026AAE
:10F62000110E016EAAEC1BF000D00B0E0B01D86F6F
:10F63000820ED76F0001F7EC14F00B0101D00B0123
:10F64000036A93513F0FE96E000E0320EA6EEF6AE2
:10F65000932B4DEF6CF000011200E824F76AF736A7
:10F660007B0FF66EF60EF722000EF86EFB6E0A00A8
:10F67000F550FA6E0800F550F96E1CB8E2C0FCC8EF
:10F6800004D1E824F76AF736A30FF66EF60EF722D8
:10F69000000EF86EFB6E0A00F550FA6E0800F55089
:10F6A000F96E7ED970E220EABCF1EACFA3FBE9CF84
:10F6B000A2FB0B019C39F0099E6F9E27E20F9F6F02
:10F6C000320FA16F9C510F0B9F279F27A127E90F96
:10F6D000A06FA027A0279B390F0BA027A127A03739
:10F6E000A137A11FA1379B510F0BA1279E37070EF2
:10F6F0009D6F0A0EA007A127FDE39F07A027FDE34A
:10F700009E079F27FDE39D079E27FDE30B0EEA6EF4
:10F710009D0EE96E070EA215A29DE926A10EE95CD9
:10F72000D8B4A28DEF50006E08E1A2BD06D0A2B9F8
:10F7300016D0A2B702D0200E03D0A287A299300E15
:10F740000026EACF9CFBE9CF9BFB00C0A6FB000193
:10F75000C3EC13F09CCBEAFF9BCBE9FF0B01EE500F
:10F76000A2ADDCD7000112000B01A56BA66B0A0E3F
:10F770000D01B66F000117EC13F00B01A56BA2CBC6
:10F78000A6FB580EC66FA5CBC7FBA6CBC8FB0001D6
:10F79000C0EC11F00A0E0D01B66F000117EC13F06A
:10F7A000100E0B01A56FA4CBA6FB580EC66FA5CB00
:10F7B000C7FBA6CBC8FB0001C0EC11F00A0E0D017F
:10F7C000B66F000117EC13F0100E0B01A56FA0CB64
:10F7D000A6FB5E0EC66FA5CBC7FBA6CBC8FB000180
:10F7E000C0EC11F072EF7CF0938681A670D0040E0D
:10F7F0000B01A06FFA0E0D01B66F000117EC13F0AC
:10F800000B01A02FF7D79BCBA0FBA16BA26B9BCBCF
:10F81000A3FB000137EC1AF0640E0D01B66F000176
:10F8200017EC13F09CCBA0FB0B01A16B010EA017F2
:10F83000A16BA26FA0CBA3FB000137EC1AF0640E02
:10F840000D01B66F000117EC13F00B019DCBA0FB6F
:10F85000A16B020EA26F9DCBA3FB000137EC1AF047
:10F86000640E0D01B66F000117EC13F09ECBA0FBE8
:10F870000B01A16B010EA017A16B030EA26FA0CB11
:10F88000A3FB000137EC1AF0640E0D01B66F000106
:10F8900017EC13F00B019F517F0BA06F040EA26FAA
:10F8A000A0CBA3FB000137EC1AF0640E0D01B66F7C
:10F8B000000117EC13F00B01A06B000180EC1AF0B3
:10F8C000640E0D01B66F000117EC13F00BD09CCB4A
:10F8D000A1FB9BCBA0FB9ECBA3FB9DCBA2FB9FCB15
:10F8E000A4FB42D712000B019B51000A000104E067
:10F8F000080AD8B49CD026D19DCBA1FB0B01A26BEA
:10F90000010EA117A26BAA6AA96AA1CBA8FFA69CA7
:10F91000A69EA684F250006EF29E0F01550EA76EB1
:10F92000AA0EA76EA682A6B2FED7A6940050F21227
:10F930000B019C51A16FA26BAA6A010EA96EA1CB0B
:10F94000A8FFA69CA69EA684F250006EF29E0F0110
:10F95000550EA76EAA0EA76EA682A6B2FED7A694D3
:10F960000050F2129FCBA1FB0B01A26B010EA1175D
:10F97000A26BAA6A020EA96EA1CBA8FFA69CA69EA6
:10F98000A684F250006EF29E0F01550EA76EAA0ECD
:10F99000A76EA682A6B2FED7A6940050F2120B0163
:10F9A0009E51A16FA26BAA6A030EA96EA1CBA8FFFC
:10F9B000A69CA69EA684F250006EF29E0F01550EE4
:10F9C000A76EAA0EA76EA682A6B2FED7A694005076
:10F9D000F2120B01A0517F0BA16FAA6A040EA96E4F
:10F9E000A1CBA8FFA69CA69EA684F250006EF29E14
:10F9F0000F01550EA76EAA0EA76EA682A6B2FED75D
:10FA0000A6940050F2129CCB54F70B019D51010BB0
:10FA10000701556F9ECB56F70B019F51010B070154
:10FA2000576F0B01A0517F0B0701586F8FD09DCBF3
:10FA3000A1FB0B01A26B010EA117A26BAA6A060E15
:10FA4000A96EA1CBA8FFA69CA69EA684F250006E2C
:10FA5000F29E0F01550EA76EAA0EA76EA682A6B241
:10FA6000FED7A6940050F2120B019C51A16FA26B1D
:10FA7000AA6A070EA96EA1CBA8FFA69CA69EA68483
:10FA8000F250006EF29E0F01550EA76EAA0EA76EE1
:10FA9000A682A6B2FED7A6940050F2129FCBA1FB7D
:10FAA0000B01A26B010EA117A26BAA6A080EA96E28
:10FAB000A1CBA8FFA69CA69EA684F250006EF29E43
:10FAC0000F01550EA76EAA0EA76EA682A6B2FED78C
:10FAD000A6940050F2120B019E51A16FA26BAA6A6C
:10FAE000090EA96EA1CBA8FFA69CA69EA684F250E3
:10FAF000006EF29E0F01550EA76EAA0EA76EA6828B
:10FB0000A6B2FED7A6940050F2120B01A0517F0BB3
:10FB1000A16FAA6A0A0EA96EA1CBA8FFA69CA69EF9
:10FB2000A684F250006EF29E0F01550EA76EAA0E2B
:10FB3000A76EA682A6B2FED7A6940050F2120701C5
:10FB400005D00001000E016E04D00701010E016E08
:10FB5000000112005C0E0B01CE6FCF6B00014FEC69
:10FB60001FF0040E0701496F0B0E0B01CF6F9B0EA8
:10FB7000CE6F130ED06F070ED26FD00ED16FD36B36
:10FB800000013DEC25F0012C0AD0A3CBDEFB6DEC8F
:10FB900025F001C049F73F0E07014B6F000112002D
:10FBA000610E0B01CE6FCF6B00014FEC1FF0010E09
:10FBB00007014A6F0B0E0B01CF6F9B0ECE6F130E1A
:10FBC000D06F070ED26FD00ED16FD36B00013DEC1A
:10FBD00025F0012C16D0A3CBDEFB6DEC25F001380F
:10FBE0000B01AF6FF00EAF17A4CBDEFB00016DEC85
:10FBF00025F00B01AF51011007014A6F3F0E4C6F0A
:10FC000000011200070151AD09D05A0EF66E1A0E0E
:10FC1000F76E000EF86E000143EC1CF00B0E0D01A8
:10FC2000AD6F9D0EAC6F0D0EAE6F9CCBB0FD9BCB40
:10FC3000AFFD000168EC2CF0015222E00B019E5157
:10FC4000410A000111E0030A0FE0220A11E0580AFC
:10FC500013E0680A11E0010A0FE0030A0DE0330A1D
:10FC60000BE0030A09E009D0010E016E0BD005D0AC
:10FC7000FF0E016E07D001D000D00701CFD70001E1
:10FC8000000E016E120007016051010A000126E01A
:10FC9000030A32E00C0A3EE00D0AD8B4BBD00A0ACF
:10FCA000D8B4C6D0010AD8B4D1D00F0AD8B4DCD0A9
:10FCB000080AD8B4E7D00B0AD8B4F2D00F0AD8B4E7
:10FCC000FDD0010AD8B408D1070AD8B413D11D0A4F
:10FCD000D8B41ED1010AD8B449D148D19CCBEAFF8F
:10FCE0009BCBE9FF000E28EC07F00A000900F55055
:10FCF000EE6E0009FBE148D19CCBEAFF9BCBE9FF0C
:10FD0000000E3BEC07F00A000900F550EE6E00090A
:10FD1000FBE13AD107015251006E5351036E010EBF
:10FD2000035C04E10052000120E00701010E035CC6
:10FD300005E1010E005C000126E00701010E035CF5
:10FD400005E1020E005C00012CE00701020E035CDD
:10FD500004E10052000133E00701030E035C04E1FB
:10FD6000005200013AE0070146D09CCBEAFF9BCB52
:10FD7000E9FF000EC9EC06F00A000900F550EE6E2E
:10FD80000009FBE146D09CCBEAFF9BCBE9FF000ECC
:10FD9000DCEC06F00A000900F550EE6E0009FBE10C
:10FDA00038D09CCBEAFF9BCBE9FF000EEFEC06F0CE
:10FDB0000A000900F550EE6E0009FBE12AD09CCB49
:10FDC000EAFF9BCBE9FF000E02EC07F00A000900F6
:10FDD000F550EE6E0009FBE11CD09CCBEAFF9BCBFB
:10FDE000E9FF000E15EC07F00A000900F550EE6E71
:10FDF0000009FBE10ED09CCBEAFF9BCBE9FF000E94
:10FE000000017EEC08F00A000900F550EE6E0009D2
:10FE1000FBE1BAD09CCBEAFF9BCBE9FF000E4EEC96
:10FE200007F00A000900F550EE6E0009FBE1ACD0C6
:10FE30009CCBEAFF9BCBE9FF000E61EC07F00A00C8
:10FE40000900F550EE6E0009FBE19ED09CCBEAFF65
:10FE50009BCBE9FF000E87EC07F00A000900F55084
:10FE6000EE6E0009FBE190D09CCBEAFF9BCBE9FF53
:10FE7000000E9AEC07F00A000900F550EE6E00093A
:10FE8000FBE182D09CCBEAFF9BCBE9FF000EADECFF
:10FE900007F00A000900F550EE6E0009FBE174D08E
:10FEA0009CCBEAFF9BCBE9FF000EC0EC07F00A00F9
:10FEB0000900F550EE6E0009FBE166D09CCBEAFF2D
:10FEC0009BCBE9FF000ED3EC07F00A000900F550C8
:10FED000EE6E0009FBE158D09CCBEAFF9BCBE9FF1B
:10FEE000000EE6EC07F00A000900F550EE6E00097E
:10FEF000FBE14AD09CCBEAFF9BCBE9FF000EA3ECD1
:10FF000006F00A000900F550EE6E0009FBE13CD056
:10FF10009CCBEAFF9BCBE9FF000E58EC08F00A00EF
:10FF20000900F550EE6E0009FBE10B019D6B9D5140
:10FF300005081AE3040E9D25036A9B25016E9C515A
:10FF4000032203C09FFB036A9D51590FE96E070E00
:10FF50000320EA6EEFCFA0FB9FCBEAFF01C0E9FFD1
:10FF6000A0CBEFFF9D2BE3D700010ED09CCBEAFF87
:10FF70009BCBE9FF000EF9EC07F00A000900F550F1
:10FF8000EE6E0009FBE100D068EF90F0D4EC48F091
:10FF9000070161B507D0000107EC3BF068EC4AF0BF
:10FFA0000ED0070160510E080AE1525308E1535187
:10FFB000030805E14FB003D0000149EC55F0000102
:10FFC00056EC46F0070161B105D00001BEEC41F0EE
:10FFD00070EC40F00001B4EC45F075EF90F0B0CB60
:0EFFE000B1FBDDD3120014EF84F09FEFACF004
:020000040001F9
:100000000B01B36BB26BB153D8B40CEF80F0B151AC
:100010000308D8B010EF80F0000E016E3BEF83F0C4
:10002000B36B600EB26F200EB227000EB323010E29
:10003000B15D200DF350036AB2270350B323B351CF
:10004000036EB251B22BD8B4B32BB46F03C0B5FB5F
:10005000B5CBAAFFB4CBA9FF60C7A8FFA69CA69EFC
:10006000A684F250006EF29E0F01550EA76EAA0EE6
:10007000A76EA682A6B23AEF80F0A6940050F212C4
:100080000B01B351036EB251B22BD8B4B32BB46F82
:1000900003C0B5FBB5CBAAFFB4CBA9FF61C7A8FFCE
:1000A000A69CA69EA684F250006EF29E0F01550EED
:1000B000A76EAA0EA76EA682A6B25CEF80F0A694E9
:1000C0000050F2120B01B351036EB251B22BD8B4EF
:1000D000B32BB46F03C0B5FB63C7B6FBB5CBAAFFA8
:1000E000B4CBA9FFB6CBA8FFA69CA69EA684F250CF
:1000F000006EF29E0F01550EA76EAA0EA76EA68285
:10010000A6B280EF80F0A6940050F2120B01B3511A
:10011000036EB251B22BD8B4B32BB46F03C0B5FB8E
:1001200062C7B6FBB5CBAAFFB4CBA9FFB6CBA8FF7D
:10013000A69CA69EA684F250006EF29E0F01550E5C
:10014000A76EAA0EA76EA682A6B2A4EF80F0A69410
:100150000050F2120B01B351036EB251B22BD8B45E
:10016000B32BB46F03C0B5FBB5CBAAFFB4CBA9FFCB
:1001700064C7A8FFA69CA69EA684F250006EF29EBD
:100180000F01550EA76EAA0EA76EA682A6B2C6EFE5
:1001900080F0A6940050F2120B01B351036EB251DD
:1001A000B22BD8B4B32BB46F03C0B5FBB5CBAAFF49
:1001B000B4CBA9FF65C7A8FFA69CA69EA684F25053
:1001C000006EF29E0F01550EA76EAA0EA76EA682B4
:1001D000A6B2E8EF80F0A6940050F2120B01B351E2
:1001E000036EB251B22BD8B4B32BB46F03C0B5FBBE
:1001F00067C7B6FBB5CBAAFFB4CBA9FFB6CBA8FFA8
:10020000A69CA69EA684F250006EF29E0F01550E8B
:10021000A76EAA0EA76EA682A6B20CEF81F0A694D6
:100220000050F2120B01B351036EB251B22BD8B48D
:10023000B32BB46F03C0B5FB66C7B6FBB5CBAAFF43
:10024000B4CBA9FFB6CBA8FFA69CA69EA684F2506D
:10025000006EF29E0F01550EA76EAA0EA76EA68223
:10026000A6B230EF81F0A6940050F2120B01B35108
:10027000036EB251B22BD8B4B32BB46F03C0B5FB2D
:1002800069C7B6FBB5CBAAFFB4CBA9FFB6CBA8FF15
:10029000A69CA69EA684F250006EF29E0F01550EFB
:1002A000A76EAA0EA76EA682A6B254EF81F0A694FE
:1002B0000050F2120B01B351036EB251B22BD8B4FD
:1002C000B32BB46F03C0B5FB68C7B6FBB5CBAAFFB1
:1002D000B4CBA9FFB6CBA8FFA69CA69EA684F250DD
:1002E000006EF29E0F01550EA76EAA0EA76EA68293
:1002F000A6B278EF81F0A6940050F2120B01B35130
:10030000036EB251B22BD8B4B32BB46F03C0B5FB9C
:10031000B5CBAAFFB4CBA9FF6AC7A8FFA69CA69E2F
:10032000A684F250006EF29E0F01550EA76EAA0E23
:10033000A76EA682A6B29AEF81F0A6940050F212A0
:100340000B01B351036EB251B22BD8B4B32BB46FBF
:1003500003C0B5FBB5CBAAFFB4CBA9FF6BC7A8FF01
:10036000A69CA69EA684F250006EF29E0F01550E2A
:10037000A76EAA0EA76EA682A6B2BCEF81F0A694C5
:100380000050F2120B01B351036EB251B22BD8B42C
:10039000B32BB46F03C0B5FBB5CBAAFFB4CBA9FF99
:1003A0006CC7A8FFA69CA69EA684F250006EF29E83
:1003B0000F01550EA76EAA0EA76EA682A6B2DEEF9B
:1003C00081F0A6940050F2120B01B351036EB251AA
:1003D000B22BD8B4B32BB46F03C0B5FBB5CBAAFF17
:1003E000B4CBA9FF6DC7A8FFA69CA69EA684F25019
:1003F000006EF29E0F01550EA76EAA0EA76EA68282
:10040000A6B200EF82F0A6940050F2120B01B35195
:10041000036EB251B22BD8B4B32BB46F03C0B5FB8B
:10042000B5CBAAFFB4CBA9FF6EC7A8FFA69CA69E1A
:10043000A684F250006EF29E0F01550EA76EAA0E12
:10044000A76EA682A6B222EF82F0A6940050F21206
:100450000B01B351036EB251B22BD8B4B32BB46FAE
:1004600003C0B5FBB5CBAAFFB4CBA9FF6FC7A8FFEC
:10047000A69CA69EA684F250006EF29E0F01550E19
:10048000A76EAA0EA76EA682A6B244EF82F0A6942B
:100490000050F2120B01B351036EB251B22BD8B41B
:1004A000B32BB46F03C0B5FBB5CBAAFFB4CBA9FF88
:1004B00070C7A8FFA69CA69EA684F250006EF29E6E
:1004C0000F01550EA76EAA0EA76EA682A6B266EF02
:1004D00082F0A6940050F2120B01B351036EB25198
:1004E000B22BD8B4B32BB46F03C0B5FBB5CBAAFF06
:1004F000B4CBA9FF71C7A8FFA69CA69EA684F25004
:10050000006EF29E0F01550EA76EAA0EA76EA68270
:10051000A6B288EF82F0A6940050F2120B01B351FC
:10052000036EB251B22BD8B4B32BB46F03C0B5FB7A
:10053000B5CBAAFFB4CBA9FF72C7A8FFA69CA69E05
:10054000A684F250006EF29E0F01550EA76EAA0E01
:10055000A76EA682A6B2AAEF82F0A6940050F2126D
:100560000B01B351036EB251B22BD8B4B32BB46F9D
:1005700003C0B5FBB5CBAAFFB4CBA9FF73C7A8FFD7
:10058000A69CA69EA684F250006EF29E0F01550E08
:10059000A76EAA0EA76EA682A6B2CCEF82F0A69492
:1005A0000050F2120B01B351036EB251B22BD8B40A
:1005B000B32BB46F03C0B5FBB5CBAAFFB4CBA9FF77
:1005C00074C7A8FFA69CA69EA684F250006EF29E59
:1005D0000F01550EA76EAA0EA76EA682A6B2EEEF69
:1005E00082F0A6940050F2120B01B351036EB25187
:1005F000B22BD8B4B32BB46F03C0B5FBB5CBAAFFF5
:10060000B4CBA9FF75C7A8FFA69CA69EA684F250EE
:10061000006EF29E0F01550EA76EAA0EA76EA6825F
:10062000A6B210EF83F0A6940050F2120B01B35162
:10063000036EB251B22BD8B4B32BB46F03C0B5FB69
:10064000B5CBAAFFB4CBA9FF76C7A8FFA69CA69EF0
:10065000A684F250006EF29E0F01550EA76EAA0EF0
:10066000A76EA682A6B232EF83F0A6940050F212D3
:10067000010E016E0B010001C1EF83F007EC3BF0AE
:10068000070160510E08D8A458EF83F05253D8A444
:1006900058EF83F053510308D8A458EF83F04FB0BC
:1006A00058EF83F0000149EC55F05BEF83F0070150
:1006B000000168EC4AF0D4EC48F056EC46F0BEEC91
:1006C00041F070EC40F0070160510908D8A475EFC3
:1006D00083F0000170EC55F08FEC55F0AEEC55F066
:1006E000CDEC55F08FEF83F0070160510708D8B4C7
:1006F0007FEF83F060510F08D8A48CEF83F00001E6
:1007000018EC56F037EC56F056EC56F0CDEC55F0B0
:1007100007016D6B90EF83F00001B4EC45F0070129
:1007200060510D08D8B49AEF83F060510E08D8A438
:10073000A2EF83F000010DEC47F0D6EC47F055EC4A
:1007400048F0070160510E08D8A4BDEF83F0525362
:10075000D8A4B0EF83F053510308D8B4B6EF83F0B8
:10076000000175EC56F0BDEF83F00701000137EC96
:1007700057F0BDEC56F0FAEC56F0B0CBB1FB0001EF
:100780003FD4012CCAEF83F0010E016ECEEF83F04F
:10079000CEEF83F0000E016ECEEF83F012000B015E
:1007A000B36BB26BB153D8B4DBEF83F0B151030834
:1007B000D8B0DFEF83F0000E016E11EF84F0B36B61
:1007C000600EB26F200EB227000EB323010EB15D92
:1007D000200DF350036AB2270350B323B351036EC5
:1007E000B251B22BD8B4B32BB46F03C0B5FBB5CBA9
:1007F000AAFFB4CBA9FFA86AA69CA69EA684F25025
:10080000006EF29E0F01550EA76EAA0EA76EA6826D
:10081000A6B208EF84F0A6940050F212010E016E09
:100820000B010001F2EF7FF00B01926B936B946B65
:10083000966B956B986B976B996B9A919A939A9527
:1008400081A025EF84F0A4EF96F0400E9B6F9C6B87
:1008500000013AEC12F001C092FBFF0E0B01921B5B
:10086000929F400E9B6F010E9C6F00013AEC12F0BC
:1008700001C051F7070151AD6AEF84F0B80EF66E72
:10088000170EF76E000EF86E090E0D01B66F00011F
:1008900069EC1CF051C7B7FD570E0D01B86F000190
:1008A000B7EC1BF0200EA4A853EF84F06D6E92CB32
:1008B000B7FD570E0D01B86F0001B7EC1BF00A0E23
:1008C000A4A860EF84F06D6E0D0EA4A865EF84F00F
:1008D0006D6E070151AF89EF87F0938681A678EF9F
:1008E00084F0010E0B01986F97697CEF84F007018B
:1008F0000B01986B7F0E976F92515F0B010A0001FD
:10090000D8B495EF84F0030AD8B4A8EF84F0420A73
:10091000D8B4BBEF84F0500AD8B4ACEF85F0180A15
:10092000D8B49DEF86F086EF87F04FB09BEF84F050
:100930004F809CEF84F04F90400E0B01C66F0C0E61
:10094000C76F4FC0C8FB0001C0EC11F086EF87F005
:100950004FB2AEEF84F04F82AFEF84F04F92400E73
:100960000B01C66F0C0EC76F4FC0C8FB0001C0EC77
:1009700011F086EF87F00B019A9355C796FB54C789
:1009800095FB96510108D8B0C9EF84F0010E966F1F
:1009900095694F884FB275EF85F09AB341EF85F0B6
:1009A000400E9B6F9C6B00013AEC12F001C092FB71
:1009B000FF0E0B01921B5F0E921792514008D8A4B4
:1009C0003EEF85F04FB0F9EF84F0952BD8B4962B1D
:1009D0009851965DD8A0F7EF84F0D8A4F5EF84F095
:1009E0009551975DD8B0F7EF84F0966B956B0BEF50
:1009F00085F09553D8A401EF85F09653D8B407EF4E
:100A000085F09551D8B4960795070BEF85F098CBF4
:100A100096FB97CB95FB0B0E6B6F810E6A6FCC0E1E
:100A2000F66E170EF76E000EF86E090E9D6F000140
:100A3000D3EC13F0100EE96E96CB9CFB95CB9BFB91
:100A400055EC7BF0200E0B01A66F0001C3EC13F0F8
:100A50000B0E0B01D86F810ED76F0001F7EC14F06D
:100A6000020E0B019B6F960E0D01B66F000117EC85
:100A700013F00B019B2FF7D73FEF85F09A83CDEF53
:100A800084F09553D8A449EF85F09653D8B475EF08
:100A900085F096510108D8A075EF85F096CB55F7F3
:100AA00095CB54F755C79CFB54C79BFB57C79EFB80
:100AB00056C79DFB58C79FFB0001F4EC7BF0320E3C
:100AC0000D01B66F000117EC13F00B019B6B55C7BE
:100AD0009DFB54C79CFB57C79FFB56C79EFB58C73F
:100AE000A0FB000173EC7CF00B01070EB16F540EFC
:100AF000B06F070EB36F560EB26F070EB56F580E7C
:100B0000B46F0001BCEC24F00B0E0B016B6F810E77
:100B10006A6FDA0EF66E170EF76E000EF86E090E9B
:100B20009D6F0001D3EC13F0100EE96E55C79CFBCE
:100B300054C79BFB55EC7BF0200E0B01A66F000108
:100B4000C3EC13F00B0E0B01D86F810ED76F0001B1
:100B5000F7EC14F086EF87F00B019A9357C796FBDA
:100B600056C795FB96510108D8B0BAEF85F0010E33
:100B7000966F95694F884FB266EF86F09AB332EF61
:100B800086F0400E9B6F9C6B00013AEC12F001C0A6
:100B900092FBFF0E0B01921B5F0E921792511008F1
:100BA000D8A42FEF86F04FB0EAEF85F0952BD8B49C
:100BB000962B9851965DD8A0E8EF85F0D8A4E6EF83
:100BC00085F09551975DD8B0E8EF85F0966B956B01
:100BD000FCEF85F09553D8A4F2EF85F09653D8B486
:100BE000F8EF85F09551D8B496079507FCEF85F09E
:100BF00098CB96FB97CB95FB0B0E6B6F810E6A6FB4
:100C0000E80EF66E170EF76E000EF86E090E9D6F69
:100C10000001D3EC13F0100EE96E96CB9CFB95CB44
:100C20009BFB55EC7BF0200E0B01A66F0001C3EC83
:100C300013F00B0E0B01D86F810ED76F0001F7EC8C
:100C400014F0020E0B019B6F960E0D01B66F0001A2
:100C500017EC13F00B019B2FF7D730EF86F09A8338
:100C6000BEEF85F09553D8A43AEF86F09653D8B4EA
:100C700066EF86F096510108D8A066EF86F096CB15
:100C800057F795CB56F755C79CFB54C79BFB57C7E7
:100C90009EFB56C79DFB58C79FFB0001F4EC7BF001
:100CA000320E0D01B66F000117EC13F00B019B6BB8
:100CB00055C79DFB54C79CFB57C79FFB56C79EFB60
:100CC00058C7A0FB000173EC7CF00B01070EB16F5D
:100CD000540EB06F070EB36F560EB26F070EB56F9E
:100CE000580EB46F0001BCEC24F00B0E0B016B6FBF
:100CF000810E6A6FF60EF66E170EF76E000EF86E26
:100D0000090E9D6F0001D3EC13F0100EE96E57C76A
:100D10009CFB56C79BFB55EC7BF0200E0B01A66F8E
:100D20000001C3EC13F00B0E0B01D86F810ED76FCF
:100D30000001F7EC14F086EF87F00B019A93966BA5
:100D400058C795FB9653D8A4ABEF86F095517F0812
:100D5000D8B0AEEF86F0966B7F0E956F4F864FB290
:100D60004FEF87F09AB321EF87F0400E9B6F9C6B9B
:100D700000013AEC12F001C092FBFF0E0B01921B36
:100D80005F0E921792510808D8A41EEF87F04FB05B
:100D9000DAEF86F0952BD8B4962B9653D8A4D6EFDD
:100DA00086F095517F08D8B0D8EF86F0966B956B9A
:100DB000EBEF86F09553D8A4E2EF86F09653D8B4C3
:100DC000E8EF86F09551D8B496079507EBEF86F0DB
:100DD000966B7F0E956F0B0E6B6F810E6A6F040E14
:100DE000F66E180EF76E000EF86E090E9D6F00017C
:100DF000D3EC13F095CB9BFB1B0E0B019C6F0001FA
:100E0000C2EC59F0200E0B01A66F0001C3EC13F0E9
:100E10000B0E0B01D86F810ED76F0001F7EC14F0A9
:100E2000020E0B019B6F960E0D01B66F000117ECC1
:100E300013F00B019B2FF7D71FEF87F09A83B2EFC8
:100E400086F09553D8B44FEF87F095517F08D8A01E
:100E50004FEF87F095CB58F755C79CFB54C79BFBCA
:100E600057C79EFB56C79DFB58C79FFB0001F4EC7C
:100E70007BF0320E0D01B66F000117EC13F00B0181
:100E80009B6B55C79DFB54C79CFB57C79FFB56C721
:100E90009EFB58C7A0FB000173EC7CF00B01070E12
:100EA000B16F540EB06F070EB36F560EB26F070ED0
:100EB000B56F580EB46F0001BCEC24F00B0E0B01A3
:100EC0006B6F810E6A6F120EF66E180EF76E000EC3
:100ED000F86E090E9D6F0001D3EC13F058C79BFB11
:100EE0001B0E0B019C6F0001C2EC59F0200E0B0190
:100EF000A66F0001C3EC13F00B0E0B01D86F810E2F
:100F0000D76F0001F7EC14F086EF87F00B01A4EF28
:100F100096F00B019251200B2008D8A41FEF88F007
:100F200007016053D8B413EF88F060510E08D8B4AD
:100F3000A3EF87F081A2A3EF87F00B019A918A9229
:100F40009392A5EF87F00B019A819251200B200814
:100F5000D8A4D8EF87F04FAAD6EF87F04F9A400E6B
:100F6000C66F0C0EC76F4FC0C8FB0001C0EC11F07C
:100F7000070151B3CAEF87F051B5CAEF87F0410EB0
:100F80000B01FE6F010EFF6F00017CEC2EF0D4EF21
:100F900087F0070151A3D5EF87F0410E0B01CE6F0B
:100FA000CF6B00014FEC1FF007010B0102EF88F03F
:100FB0004FBA02EF88F04F8A400EC66F0C0EC76F13
:100FC0004FC0C8FB0001C0EC11F0070151B3F7EFAF
:100FD00087F051B5F7EF87F0420E0B01FE6F010E5F
:100FE000FF6F00017CEC2EF001EF88F0070151A3A8
:100FF00002EF88F0420E0B01CE6FCF6B00014FEC79
:101000001FF00701070160510E08D8B411EF88F0F6
:101010000B019AA103D0070111EF88F08A82939205
:1010200007011CEF88F00B0192512008D8A41BEF98
:1010300088F0A4EF96F007014DEF88F00B014FBA4E
:101040004EEF88F04F8A400EC66F0C0EC76F4FC030
:10105000C8FB0001C0EC11F007016053D8B44DEF9C
:1010600088F051B342EF88F051B542EF88F0420E5C
:101070000B01FE6F010EFF6F00017CEC2EF04CEFB8
:1010800088F0070151A34DEF88F0420E0B01CE6F9F
:10109000CF6B00014FEC1FF007010B015F0E9217A1
:1010A000070160510E08D8B4C2EF88F081A2C2EFE8
:1010B00088F00B019251400B4008D8B472EF88F0D1
:1010C000070151B567EF88F00B01A4EF96F00B0113
:1010D0009251040B0408D8B470EF88F0A4EF96F096
:1010E000C1EF88F007016053D8A4C2EF88F08A925C
:1010F00093920B0EEA6E810EE96E200E006E026A6C
:10110000110E016E0001AAEC1BF00B0E0B01D86F43
:10111000810ED76F0001F7EC14F0070151A397EF90
:1011200088F00001EAEC4AF0A3EF88F0070151A52E
:10113000A0EF88F000013DEC4FF0A3EF88F007012D
:1011400000018CEC57F007016053D8A4C2EF88F07F
:101150008A8293920B0EEA6E810EE96E200E006E6B
:10116000026A110E016E0001AAEC1BF00B0E0B01BE
:10117000D86F810ED76F0001F7EC14F00B01A4EFCC
:1011800096F00701482D85EF89F00B019251000A76
:101190000001D8B4DAEF88F0010AD8B4DCEF88F0A7
:1011A000030AD8B435EF89F0060AD8B435EF89F0D0
:1011B0007EEF89F082EF89F007014D51010A0001AD
:1011C000D8B4E9EF88F0030AD8B40CEF89F02FEF18
:1011D00089F05D0E0B01CE6F010ECF6F00014FEC59
:1011E0001FF0AAEC7DF00B0EEA6E810EE96E000E88
:1011F000F7EC03F00A000900F550EE6E0009D8A4E0
:10120000FBEF88F00B0E0B01D86F810ED76F00013A
:10121000F7EC14F033EF89F0620E0B01CE6F010E84
:10122000CF6F00014FEC1FF0D0EC7DF00B0EEA6E9B
:10123000810EE96E000E0AEC04F00A000900F55078
:10124000EE6E0009D8A41EEF89F00B0E0B01D86FCB
:10125000810ED76F0001F7EC14F033EF89F00B012A
:10126000A4EF96F0000182EF89F00701486B0B01B3
:10127000936B93510708D8A058EF89F04FB244EF11
:1012800089F04F8245EF89F04F92400EC66F0C0EE9
:10129000C76F4FC0C8FB0001C0EC11F0FA0E0D0182
:1012A000B66F000117EC13F00B01932B39EF89F0A7
:1012B0004F828A929392400EC66F0C0EC76F4FC03A
:1012C000C8FB0001C0EC11F00B0EEA6E810EE96E56
:1012D000000E1DEC04F00A000900F550EE6E000946
:1012E000D8A46CEF89F00B0E0B01D86F810ED76F6D
:1012F0000001F7EC14F00B01A4EF96F00B01A4EF42
:1013000096F00001A4EF96F007010B019251000A3C
:101310000001D8B4B6EF89F0010AD8B4B8EF89F06B
:10132000030AD8B42AEF8BF0060AD8B4CAEF8EF0BD
:10133000440AD8B439EF90F0480AD8B46CEF91F071
:10134000180AD8B4D0EF92F0400AD8B428EF94F03D
:10135000180AD8B4D1EF94F0500AD8B475EF95F0CC
:101360001E0AD8B4E8EF95F06EEF96F0A4EF96F071
:101370000B0EEA6E810EE96E200E006E026A110EEF
:10138000016EAAEC1BF00B0E0B01D86F810ED76F0C
:101390000001F7EC14F04FB0A0EF8AF04F80070186
:1013A00051A3E8EF89F0210E0B01CE6F010ECF6F34
:1013B00000014FEC1FF0640E0D01B66F000117EC39
:1013C00013F007EC3BF068EC4AF06BEF8AF0070192
:1013D00051A537EF8AF04E6B61A7F2EF89F0619764
:1013E0000AEF8AF04E6B670E0B01DD6FDE6B0001BA
:1013F0007EEC27F0030E0C010C6FE80E0B6F000162
:101400003EEC27F001C099FB0B01992D0BEF8AF000
:10141000070161870B01070161B735EF8AF0000111
:1014200007EC3BF0640E0D01B66F000117EC13F0F2
:10143000210E0B01DD6F010EDE6F00017EEC27F047
:10144000D9EC3EF001C099FB0B019953D8A42DEFC4
:101450008AF04FB22DEF8AF04F82370EDD6F010E0A
:10146000DE6F00017EEC27F007016CEF8AF060511F
:101470000E08D8A45EEF8AF0210E0B01FE6F010E5C
:10148000FF6F00017CEC2EF0640E0D01B66F0001C1
:1014900017EC13F007EC3BF068EC4AF007015253ED
:1014A000D8A45CEF8AF053510308D8A45CEF8AF00B
:1014B000000137EC57F007016CEF8AF0000107ECF0
:1014C0003BF068EC4AF0210E0B01FE6F010EFF6F3E
:1014D00000017CEC2EF0070151A586EF8AF061A790
:1014E00086EF8AF04F900B0EEA6E810EE96E000EC9
:1014F000000130EC04F00A000900F550EE6E00091E
:10150000D8A47CEF8AF096EF8AF007010B0EEA6E02
:10151000810EE96E000E000143EC04F00A000900A0
:10152000F550EE6E0009D8A48FEF8AF00B0E0B0178
:10153000D86F810ED76F0001F7EC14F01DEF8BF020
:101540004F90070151A3B0EF8AF0200E0B01CE6F30
:10155000010ECF6F00014FEC1FF006EF8BF007017B
:1015600051A5E4EF8AF04E6B4F92000107EC3BF07F
:10157000800E0701726F696B686F676B666F656BD2
:10158000756B010E736F746B020E6F6F800E6A6F56
:101590006B6B010E716F200E0B01DD6F010EDE6FA4
:1015A00000017EEC27F0640E0D01B66F000117EC10
:1015B00013F0370E0B01DD6F010EDE6F00017EECC4
:1015C00027F006EF8BF00701200E0B01FE6F010ED6
:1015D000FF6F00017CEC2EF007EC3BF0070160513F
:1015E0000E08D8A403EF8BF05253D8A403EF8BF06E
:1015F00053510308D8A403EF8BF0000149EC55F0D8
:1016000006EF8BF00701000168EC4AF00B0EEA6E62
:10161000810EE96E000E56EC04F00A000900F55048
:10162000EE6E0009D8A40EEF8BF00B0E0B01D86FF5
:10163000810ED76F0001F7EC14F0400E0B01C66F5E
:101640000C0EC76F4FC0C8FB0001C0EC11F030900A
:10165000A4EF96F0070160510E08D8B480EF8DF02A
:1016600051B5E7EF8CF04FA416EF8CF04FA2E3EFEB
:101670008BF04F920B0EEA6E810EE96E000E0001A8
:1016800069EC04F00A000900F550EE6E0009D8A4D8
:1016900043EF8BF00B0E0B01D86F810ED76F00015B
:1016A000F7EC14F0070151B371EF8BF01D0E0B0135
:1016B000FE6F010EFF6F00017CEC2EF01F0E0B0180
:1016C000FE6FFF6B00017CEC2EF00B019A85030E80
:1016D0009C6FE80E9B6F000102EC7EF0E0EF8BF058
:1016E00007011D0E0B01CE6FCF6B00014FEC1FF0F9
:1016F0003A0E0C01D36F980ED26FD46B000118EC28
:101700001FF0012CC9EF8BF01F0E0B01CE6FCF6BBA
:1017100000014FEC1FF03A0E0C01D36F980ED26F00
:10172000D46B000118EC1FF0012CB0EF8BF00B0E06
:10173000EA6E810EE96E000E7CEC04F00A000900EE
:10174000F550EE6E0009D8A49FEF8BF00B0E0B0145
:10175000D86F810ED76F0001F7EC14F0C7EF8BF054
:101760000B0EEA6E810EE96E000E8FEC04F00A009B
:101770000900F550EE6E0009D8A4B8EF8BF00B0EFF
:101780000B01D86F810ED76F0001F7EC14F0E0EF7A
:101790008BF00B0EEA6E810EE96E000EA2EC04F0E7
:1017A0000A000900F550EE6E0009D8A4D1EF8BF0C5
:1017B0000B0E0B01D86F810ED76F0001F7EC14F000
:1017C00013EF8CF007014F8251B3FBEF8BF0619365
:1017D00060510E08D8B4F2EF8BF00001BEEC41F07E
:1017E00070EC40F01E0E0B01FE6F010EFF6F00014A
:1017F0007CEC2EF007010B0EEA6E810EE96E000EF6
:101800000001B5EC04F00A000900F550EE6E000985
:10181000D8A404EF8CF00B0E0B01D86F810ED76F9C
:101820000001F7EC14F0D9EF8CF007014F924F84D0
:1018300051B326EF8CF01E0E0B01FE6F010EFF6FF1
:1018400000017CEC2EF02EEF8CF007011E0E0B0138
:10185000CE6F010ECF6F00014FEC1FF00B0EEA6E42
:10186000810EE96E000E69EC04F00A000900F550E3
:10187000EE6E0009D8A436EF8CF00B0E0B01D86F7A
:10188000810ED76F0001F7EC14F00A0E0D01B66F50
:10189000000117EC13F0070151B36AEF8CF01D0E35
:1018A0000B01FE6F010EFF6F00017CEC2EF01F0E8E
:1018B0000B01FE6FFF6B00017CEC2EF00B019A8593
:1018C000030E9C6FE80E9B6F000102EC7EF0D9EFD7
:1018D0008CF007011D0E0B01CE6FCF6B00014FEC9A
:1018E0001FF03A0E0C01D36F980ED26FD46B00012B
:1018F00018EC1FF0012CC2EF8CF01F0E0B01CE6F05
:10190000CF6B00014FEC1FF03A0E0C01D36F980E15
:10191000D26FD46B000118EC1FF0012CA9EF8CF0F2
:101920000B0EEA6E810EE96E000E7CEC04F00A00EC
:101930000900F550EE6E0009D8A498EF8CF00B0E5C
:101940000B01D86F810ED76F0001F7EC14F0C0EFD8
:101950008CF00B0EEA6E810EE96E000E8FEC04F037
:101960000A000900F550EE6E0009D8A4B1EF8CF022
:101970000B0E0B01D86F810ED76F0001F7EC14F03E
:10198000D9EF8CF00B0EEA6E810EE96E000EA2EC20
:1019900004F00A000900F550EE6E0009D8A4CAEF61
:1019A0008CF00B0E0B01D86F810ED76F0001F7EC96
:1019B00014F0400E0B01C66F0C0EC76F4FC0C8FB72
:1019C0000001C0EC11F030907DEF8DF007014FA0C9
:1019D00065EF8DF04FB210EF8DF04F821D0E0B01B1
:1019E000DD6F010EDE6F00017EEC27F00B0EEA6E5C
:1019F000810EE96E000EC8EC04F00A000900F550F3
:101A0000EE6E0009D8A4FEEF8CF00B0E0B01D86F20
:101A1000810ED76F0001F7EC14F057EF8DF007013E
:101A20001C0E0B01DD6FDE6B00017EEC27F0030E58
:101A30000C010C6FE80E0B6F00013EEC27F001C0AB
:101A400099FB0B01992D39EF8DF04F920B0EEA6E39
:101A5000810EE96E000E0001DBEC04F00A000900C3
:101A6000F550EE6E0009D8A42FEF8DF04FEF8DF0FA
:101A70000B011D0EDD6F010EDE6F00017EEC27F005
:101A80000B0EEA6E810EE96E000EC8EC04F00A003F
:101A90000900F550EE6E0009D8A448EF8DF00B0E4A
:101AA0000B01D86F810ED76F0001F7EC14F0400ED8
:101AB0000B01C66F0C0EC76F4FC0C8FB0001C0EC16
:101AC00011F030907DEF8DF007010B0EEA6E810E64
:101AD000E96E000E0001EEEC04F00A000900F5507A
:101AE000EE6E0009D8A46EEF8DF00B0E0B01D86FCF
:101AF000810ED76F0001F7EC14F07BEF8EF0070139
:101B00000B019A93946B4FB289EF8DF04F828AEF5D
:101B10008DF04F92400EC66F0C0EC76F4FC0C8FBC2
:101B20000001C0EC11F007015253D8A400EF8EF071
:101B300053510308D8A400EF8EF00B019AB300EFC5
:101B40008EF09AB5FEEF8DF0400E9B6F9C6B0001FE
:101B50003AEC12F001C092FBFF0E0B01921B5F0EDC
:101B6000921792510208D8A4FDEF8DF094511E08EF
:101B7000D8B0F3EF8DF01D0EFE6FFF6B00017CEC13
:101B80002EF0030E0B019C6FE80E9B6F000102EC20
:101B90007EF04FB4D7EF8DF04F84400E0B01C66F2F
:101BA0000C0EC76F4FC0C8FB0001C0EC11F00B0E4C
:101BB000EA6E810EE96E000E01EC05F00A000900E4
:101BC000F550EE6E0009D8A4DFEF8DF00B0E0B017F
:101BD000D86F810ED76F0001F7EC14F00B019A85D6
:101BE0009A83FBEF8DF0280E0D01B66F000117EC04
:101BF00013F00B01942BFEEF8DF09A839EEF8DF086
:101C00000B019AB57CEF8EF04FB23FEF8EF00701DB
:101C10005253D8A411EF8EF053510308D8B424EFD7
:101C20008EF00B0EEA6E810EE96E000E000114ECD0
:101C300005F00A000900F550EE6E0009D8A41AEF6D
:101C40008EF034EF8EF007010B0EEA6E810EE96E16
:101C5000000E000127EC05F00A000900F550EE6EB9
:101C60000009D8A42DEF8EF00B0E0B01D86F810E5A
:101C7000D76F0001F7EC14F07BEF8EF00B0107013A
:101C800061A363EF8EF061930001BEEC41F070EC54
:101C900040F01E0E0B01FE6F010EFF6F00017CEC89
:101CA0002EF00B0EEA6E810EE96E000EB5EC04F01C
:101CB0000A000900F550EE6E0009D8A459EF8EF025
:101CC00073EF8EF007010B0EEA6E810EE96E000EC7
:101CD00000013AEC05F00A000900F550EE6E00092B
:101CE000D8A46CEF8EF00B0E0B01D86F810ED76F5E
:101CF0000001F7EC14F00B019AA5C7EF8EF09A9350
:101D00009AB3C7EF8EF030BA9FEF8EF04FB28CEFE0
:101D10008EF04F828DEF8EF04F92400EC66F0C0EFC
:101D2000C76F4FC0C8FB0001C0EC11F0FA0E0D01E7
:101D3000B66F000117EC13F0C4EF8EF00B019A831D
:101D40004F92400EC66F0C0EC76F4FC0C8FB00010C
:101D5000C0EC11F0070161830B0EEA6E810EE96E93
:101D6000000E00014DEC05F00A000900F550EE6E82
:101D70000009D8A4B5EF8EF00B0E0B01D86F810EC1
:101D8000D76F0001F7EC14F00B0180EF8EF000012B
:101D9000A4EF96F00B0EEA6E810EE96E200E006E37
:101DA000026A110E016EAAEC1BF00B0E0B01D86F2C
:101DB000810ED76F0001F7EC14F04FB499EF8FF05C
:101DC0004F84070160510908D8A4EBEF8EF00001A1
:101DD00070EC55F0070160510E08D8B4F6EF8EF0A4
:101DE0000001BEEC41F070EC40F0070151A314EF8C
:101DF0008FF01E0E0B01CE6F010ECF6F00014FEC66
:101E00001FF02B0E0B01CE6F010ECF6F00014FECB8
:101E10001FF02F0E0B01CE6F010ECF6F00014FECA4
:101E20001FF079EF8FF0070151A532EF8FF00B0E05
:101E3000EA6E810EE96E000E00013AEC05F00A0030
:101E40000900F550EE6E0009D8A420EF8FF00B0EBC
:101E50000B01D86F810ED76F0001F7EC14F079EF0A
:101E60008FF007011E0E0B01FE6F010EFF6F0001C8
:101E70007CEC2EF0070160510E08D8A445EF8FF0DE
:101E80000001BEEC41F070EC40F02B0E0B01FE6F38
:101E9000010EFF6F00017CEC2EF0070160510E086F
:101EA000D8A45FEF8FF05253D8A45FEF8FF0535157
:101EB0000308D8A45FEF8FF0000139EC41F02F0E3A
:101EC0000B01FE6F010EFF6F00017CEC2EF007018D
:101ED00060510E08D8A47AEF8FF05253D8A47AEF4D
:101EE0008FF053510308D8A47AEF8FF000014BEC28
:101EF00042F0070151B596EF8FF00B0EEA6E810E9E
:101F0000E96E000E0001B5EC04F00A000900F5507E
:101F1000EE6E0009D8A486EF8FF00B0E0B01D86F80
:101F2000810ED76F0001F7EC14F007011CEF90F061
:101F300000014F94070151B5A5EF8FF04F820001CA
:101F4000BEEC41F070EC40F0070151A3CAEF8FF0F6
:101F5000676B1E0E666F2B0E0B01CE6F010ECF6FDF
:101F600000014FEC1FF00701696B1E0E686F2F0E0A
:101F70000B01CE6F010ECF6F00014FEC1FF01C0E56
:101F80000B01CE6F010ECF6F00014FEC1FF0F1EF90
:101F90008FF0070151A5E8EF8FF00B0EEA6E810E6E
:101FA000E96E000E000127EC05F00A000900F5506B
:101FB000EE6E0009D8A4D6EF8FF00B0E0B01D86F90
:101FC000810ED76F0001F7EC14F0F1EF8FF00701ED
:101FD00061931C0E0B01FE6F010EFF6F00017CEC84
:101FE0002EF0070160510908D8A400EF90F0460ECA
:101FF0000B01FE6F010EFF6F00017CEC2EF007015C
:1020000051B51CEF90F00B0EEA6E810EE96E000EDA
:10201000000160EC05F00A000900F550EE6E0009C1
:10202000D8A40CEF90F00B0E0B01D86F810ED76F78
:102030000001F7EC14F00701400E0B01C66F0C0E07
:10204000C76F4FC0C8FB0001C0EC11F0070151B5CC
:1020500036EF90F060510E08D8B436EF90F00001E2
:10206000BEEC41F070EC40F0309007010001A4EFAD
:1020700096F0400E0B01926F070160510E08D8B424
:1020800078EF90F081B25DEF90F08A8293920B0E20
:10209000EA6E810EE96E006A026A110E016E00019D
:1020A000AAEC1BF00B0E0B01D86F810ED76F00014D
:1020B000F7EC14F075EF90F007018A929392476B5A
:1020C0000B0E0B019C6F810E9B6F000143EF7EF0A6
:1020D0000B0E0B01D86F810ED76F0001F7EC14F0D7
:1020E00007014E6B0001C6EF7FF058EF91F007013A
:1020F0000B019A93946B4F884F869AB3EBEF90F055
:10210000400E9B6F9C6B00013AEC12F001C092FBF9
:10211000FF0E0B01921B5F0E921792514008D8A43C
:10212000E8EF90F094511E08D8B0DEEF90F0030E67
:10213000B06F00013EEC83F00B01936B93510708E5
:10214000D8A0B6EF90F081B2AAEF90F08A82939275
:10215000ACEF90F08A929392FA0E0D01B66F0001E7
:1021600017EC13F00B01932B9EEF90F08A92939251
:10217000400EC66F0C0EC76F4FC0C8FB0001C0EC0D
:1021800011F030800B0EEA6E810EE96E000E73ECDA
:1021900005F00A000900F550EE6E0009D8A4CAEF58
:1021A00090F00B0E0B01D86F810ED76F0001F7EC8A
:1021B00014F00B01A4EF96F0E6EF90F0280E0D015D
:1021C000B66F000117EC13F00B01942BE9EF90F0C0
:1021D0009A837DEF90F092511808D8B459EF91F09E
:1021E00092515008D8B459EF91F092514808D8B4A0
:1021F00059EF91F081B202EF91F08A829392309080
:1022000059EF91F04F884F86030EB06F0001D4EC68
:102210003BF0012C38EF91F0400E0B01C66F0C0E15
:10222000C76F4FC0C8FB0001C0EC11F08A929392B7
:10223000030E0B01B06F0001D0EC42F030800B0EAA
:10224000EA6E810EE96E000E86EC05F00A000900C8
:10225000F550EE6E0009D8A427EF91F00B0E0B019C
:10226000D86F810ED76F0001F7EC14F058EF91F0A2
:102270008A8293920B0EEA6E810EE96E000E99EC43
:1022800005F00A000900F550EE6E0009D8A442EFEF
:1022900091F00B0E0B01D86F810ED76F0001F7EC98
:1022A00014F03090320E0D01B66F000117EC13F0F0
:1022B0000B0192511808D8B46BEF91F0925150086D
:1022C000D8B46BEF91F092514808D8B46BEF91F00D
:1022D0000001A4EF96F000010B019A93946B4F88D4
:1022E000070160510E08D8A478EF91F08A8293928A
:1022F0000B019AB30DEF92F0400E9B6F9C6B0001A7
:102300003AEC12F001C092FBFF0E0B01921B5F0E24
:10231000921792510808D8A40AEF92F094511E081F
